:0400000000000000FC
:0400010000000000FB
:0400020000000000FA
:0400030000000000F9
:0400040000000000F8
:0400050000000000F7
:0400060000000000F6
:0400070000000000F5
:0400080000000000F4
:0400090000000000F3
:04000A0000000000F2
:04000B0000000000F1
:04000C0000000000F0
:04000D0000000000EF
:04000E0000000000EE
:04000F0000000000ED
:0400100000000000EC
:0400110000000000EB
:0400120000000000EA
:0400130000000000E9
:0400140000000000E8
:0400150000000000E7
:0400160000000000E6
:0400170000000000E5
:0400180000000000E4
:0400190000000000E3
:04001A0000000000E2
:04001B0000000000E1
:04001C0000000000E0
:04001D0000000000DF
:04001E0000000000DE
:04001F0000000000DD
:0400200000000000DC
:0400210000000000DB
:0400220000000000DA
:0400230000000000D9
:0400240000000000D8
:0400250000000000D7
:0400260000000000D6
:0400270000000000D5
:0400280000000000D4
:0400290000000000D3
:04002A0000000000D2
:04002B0000000000D1
:04002C0000000000D0
:04002D0000000000CF
:04002E0000000000CE
:04002F0000000000CD
:0400300000000000CC
:0400310000000000CB
:0400320000000000CA
:0400330000000000C9
:0400340000000000C8
:0400350000000000C7
:0400360000000000C6
:0400370000000000C5
:0400380000000000C4
:0400390000000000C3
:04003A0000000000C2
:04003B0000000000C1
:04003C0000000000C0
:04003D0000000000BF
:04003E0000000000BE
:04003F0000000000BD
:0400400000000000BC
:0400410000000000BB
:0400420000000000BA
:0400430000000000B9
:0400440000000000B8
:0400450000000000B7
:0400460000000000B6
:0400470000000000B5
:0400480000000000B4
:0400490000000000B3
:04004A0000000000B2
:04004B0000000000B1
:04004C0000000000B0
:04004D0000000000AF
:04004E0000000000AE
:04004F0000000000AD
:0400500000000000AC
:0400510000000000AB
:0400520000000000AA
:0400530000000000A9
:0400540000000000A8
:0400550000000000A7
:0400560000000000A6
:0400570000000000A5
:0400580000000000A4
:0400590000000000A3
:04005A0000000000A2
:04005B0000000000A1
:04005C0000000000A0
:04005D00000000009F
:04005E00000000009E
:04005F00000000009D
:04006000000000009C
:04006100000000009B
:04006200000000009A
:040063000000000099
:040064000000000098
:040065000000000097
:040066000000000096
:040067000000000095
:040068000000000094
:040069000000000093
:04006A000000000092
:04006B000000000091
:04006C000000000090
:04006D00000000008F
:04006E00000000008E
:04006F00000000008D
:04007000000000008C
:04007100000000008B
:04007200000000008A
:040073000000000089
:040074000000000088
:040075000000000087
:040076000000000086
:040077000000000085
:040078000000000084
:040079000000000083
:04007A000000000082
:04007B000000000081
:04007C000000000080
:04007D00000000007F
:04007E00000000007E
:04007F00000000007D
:04008000000000007C
:04008100000000007B
:04008200000000007A
:040083000000000079
:040084000000000078
:040085000000000077
:040086000000000076
:040087000000000075
:040088000000000074
:040089000000000073
:04008A000000000072
:04008B000000000071
:04008C000000000070
:04008D00000000006F
:04008E00000000006E
:04008F00000000006D
:04009000000000006C
:04009100000000006B
:04009200000000006A
:040093000000000069
:040094000000000068
:040095000000000067
:040096000000000066
:040097000000000065
:040098000000000064
:040099000000000063
:04009A000000000062
:04009B000000000061
:04009C000000000060
:04009D00000000005F
:04009E00000000005E
:04009F00000000005D
:0400A000000000005C
:0400A100000000005B
:0400A200000000005A
:0400A3000000000059
:0400A4000000000058
:0400A5000000000057
:0400A6000000000056
:0400A7000000000055
:0400A8000000000054
:0400A9000000000053
:0400AA000000000052
:0400AB000000000051
:0400AC000000000050
:0400AD00000000004F
:0400AE00000000004E
:0400AF00000000004D
:0400B000000000004C
:0400B100000000004B
:0400B200000000004A
:0400B3000000000049
:0400B4000000000048
:0400B5000000000047
:0400B6000000000046
:0400B7000000000045
:0400B8000000000044
:0400B9000000000043
:0400BA000000000042
:0400BB000000000041
:0400BC000000000040
:0400BD00000000003F
:0400BE00000000003E
:0400BF00000000003D
:0400C000000000003C
:0400C100000000003B
:0400C200000000003A
:0400C3000000000039
:0400C4000000000038
:0400C5000000000037
:0400C6000000000036
:0400C7000000000035
:0400C8000000000034
:0400C9000000000033
:0400CA000000000032
:0400CB000000000031
:0400CC000000000030
:0400CD00000000002F
:0400CE00000000002E
:0400CF00000000002D
:0400D000000000002C
:0400D100000000002B
:0400D200000000002A
:0400D3000000000029
:0400D4000000000028
:0400D5000000000027
:0400D6000000000026
:0400D7000000000025
:0400D8000000000024
:0400D9000000000023
:0400DA000000000022
:0400DB000000000021
:0400DC000000000020
:0400DD00000000001F
:0400DE00000000001E
:0400DF00000000001D
:0400E000000000001C
:0400E100000000001B
:0400E200000000001A
:0400E3000000000019
:0400E4000000000018
:0400E5000000000017
:0400E6000000000016
:0400E7000000000015
:0400E8000000000014
:0400E9000000000013
:0400EA000000000012
:0400EB000000000011
:0400EC000000000010
:0400ED00000000000F
:0400EE00000000000E
:0400EF00000000000D
:0400F000000000000C
:0400F100000000000B
:0400F200000000000A
:0400F3000000000009
:0400F4000000000008
:0400F5000000000007
:0400F6000000000006
:0400F7000000000005
:0400F8000000000004
:0400F9000000000003
:0400FA000000000002
:0400FB000000000001
:0400FC000000000000
:0400FD0000000000FF
:0400FE0000000000FE
:0400FF0000000000FD
:0401000000000000FB
:0401010000000000FA
:0401020000000000F9
:0401030000000000F8
:0401040000000000F7
:0401050000000000F6
:0401060000000000F5
:0401070000000000F4
:0401080000000000F3
:0401090000000000F2
:04010A0000000000F1
:04010B0000000000F0
:04010C0000000000EF
:04010D0000000000EE
:04010E0000000000ED
:04010F0000000000EC
:0401100000000000EB
:0401110000000000EA
:0401120000000000E9
:0401130000000000E8
:0401140000000000E7
:0401150000000000E6
:0401160000000000E5
:0401170000000000E4
:0401180000000000E3
:0401190000000000E2
:04011A0000000000E1
:04011B0000000000E0
:04011C0000000000DF
:04011D0000000000DE
:04011E0000000000DD
:04011F0000000000DC
:0401200000000000DB
:0401210000000000DA
:0401220000000000D9
:0401230000000000D8
:0401240000000000D7
:0401250000000000D6
:0401260000000000D5
:0401270000000000D4
:0401280000000000D3
:0401290000000000D2
:04012A0000000000D1
:04012B0000000000D0
:04012C0000000000CF
:04012D0000000000CE
:04012E0000000000CD
:04012F0000000000CC
:0401300000000000CB
:0401310000000000CA
:0401320000000000C9
:0401330000000000C8
:0401340000000000C7
:0401350000000000C6
:0401360000000000C5
:0401370000000000C4
:0401380000000000C3
:0401390000000000C2
:04013A0000000000C1
:04013B0000000000C0
:04013C0000000000BF
:04013D0000000000BE
:04013E0000000000BD
:04013F0000000000BC
:0401400000000000BB
:0401410000000000BA
:0401420000000000B9
:0401430000000000B8
:0401440000000000B7
:0401450000000000B6
:0401460000000000B5
:0401470000000000B4
:0401480000000000B3
:0401490000000000B2
:04014A0000000000B1
:04014B0000000000B0
:04014C0000000000AF
:04014D0000000000AE
:04014E0000000000AD
:04014F0000000000AC
:0401500000000000AB
:0401510000000000AA
:0401520000000000A9
:0401530000000000A8
:0401540000000000A7
:0401550000000000A6
:0401560000000000A5
:0401570000000000A4
:0401580000000000A3
:0401590000000000A2
:04015A0000000000A1
:04015B0000000000A0
:04015C00000000009F
:04015D00000000009E
:04015E00000000009D
:04015F00000000009C
:04016000000000009B
:04016100000000009A
:040162000000000099
:040163000000000098
:040164000000000097
:040165000000000096
:040166000000000095
:040167000000000094
:040168000000000093
:040169000000000092
:04016A000000000091
:04016B000000000090
:04016C00000000008F
:04016D00000000008E
:04016E00000000008D
:04016F00000000008C
:04017000000000008B
:04017100000000008A
:040172000000000089
:040173000000000088
:040174000000000087
:040175000000000086
:040176000000000085
:040177000000000084
:040178000000000083
:040179000000000082
:04017A000000000081
:04017B000000000080
:04017C00000000007F
:04017D00000000007E
:04017E00000000007D
:04017F00000000007C
:04018000000000007B
:04018100000000007A
:040182000000000079
:040183000000000078
:040184000000000077
:040185000000000076
:040186000000000075
:040187000000000074
:040188000000000073
:040189000000000072
:04018A000000000071
:04018B000000000070
:04018C00000000006F
:04018D00000000006E
:04018E00000000006D
:04018F00000000006C
:04019000000000006B
:04019100000000006A
:040192000000000069
:040193000000000068
:040194000000000067
:040195000000000066
:040196000000000065
:040197000000000064
:040198000000000063
:040199000000000062
:04019A000000000061
:04019B000000000060
:04019C00000000005F
:04019D00000000005E
:04019E00000000005D
:04019F00000000005C
:0401A000000000005B
:0401A100000000005A
:0401A2000000000059
:0401A3000000000058
:0401A4000000000057
:0401A5000000000056
:0401A6000000000055
:0401A7000000000054
:0401A8000000000053
:0401A9000000000052
:0401AA000000000051
:0401AB000000000050
:0401AC00000000004F
:0401AD00000000004E
:0401AE00000000004D
:0401AF00000000004C
:0401B000000000004B
:0401B100000000004A
:0401B2000000000049
:0401B3000000000048
:0401B4000000000047
:0401B5000000000046
:0401B6000000000045
:0401B7000000000044
:0401B8000000000043
:0401B9000000000042
:0401BA000000000041
:0401BB000000000040
:0401BC00000000003F
:0401BD00000000003E
:0401BE00000000003D
:0401BF00000000003C
:0401C000000000003B
:0401C100000000003A
:0401C2000000000039
:0401C3000000000038
:0401C4000000000037
:0401C5000000000036
:0401C6000000000035
:0401C7000000000034
:0401C8000000000033
:0401C9000000000032
:0401CA000000000031
:0401CB000000000030
:0401CC00000000002F
:0401CD00000000002E
:0401CE00000000002D
:0401CF00000000002C
:0401D000000000002B
:0401D100000000002A
:0401D2000000000029
:0401D3000000000028
:0401D4000000000027
:0401D5000000000026
:0401D6000000000025
:0401D7000000000024
:0401D8000000000023
:0401D9000000000022
:0401DA000000000021
:0401DB000000000020
:0401DC00000000001F
:0401DD00000000001E
:0401DE00000000001D
:0401DF00000000001C
:0401E000000000001B
:0401E100000000001A
:0401E2000000000019
:0401E3000000000018
:0401E4000000000017
:0401E5000000000016
:0401E6000000000015
:0401E7000000000014
:0401E8000000000013
:0401E9000000000012
:0401EA000000000011
:0401EB000000000010
:0401EC00000000000F
:0401ED00000000000E
:0401EE00000000000D
:0401EF00000000000C
:0401F000000000000B
:0401F100000000000A
:0401F2000000000009
:0401F3000000000008
:0401F4000000000007
:0401F5000000000006
:0401F6000000000005
:0401F7000000000004
:0401F8000000000003
:0401F9000000000002
:0401FA000000000001
:0401FB000000000000
:0401FC0000000000FF
:0401FD0000000000FE
:0401FE0000000000FD
:0401FF0000000000FC
:0402000000000000FA
:0402010000000000F9
:0402020000000000F8
:0402030000000000F7
:0402040000000000F6
:0402050000000000F5
:0402060000000000F4
:0402070000000000F3
:0402080000000000F2
:0402090000000000F1
:04020A0000000000F0
:04020B0000000000EF
:04020C0000000000EE
:04020D0000000000ED
:04020E0000000000EC
:04020F0000000000EB
:0402100000000000EA
:0402110000000000E9
:0402120000000000E8
:0402130000000000E7
:0402140000000000E6
:0402150000000000E5
:0402160000000000E4
:0402170000000000E3
:0402180000000000E2
:0402190000000000E1
:04021A0000000000E0
:04021B0000000000DF
:04021C0000000000DE
:04021D0000000000DD
:04021E0000000000DC
:04021F0000000000DB
:0402200000000000DA
:0402210000000000D9
:0402220000000000D8
:0402230000000000D7
:0402240000000000D6
:0402250000000000D5
:0402260000000000D4
:0402270000000000D3
:0402280000000000D2
:0402290000000000D1
:04022A0000000000D0
:04022B0000000000CF
:04022C0000000000CE
:04022D0000000000CD
:04022E0000000000CC
:04022F0000000000CB
:0402300000000000CA
:0402310000000000C9
:0402320000000000C8
:0402330000000000C7
:0402340000000000C6
:0402350000000000C5
:0402360000000000C4
:0402370000000000C3
:0402380000000000C2
:0402390000000000C1
:04023A0000000000C0
:04023B0000000000BF
:04023C0000000000BE
:04023D0000000000BD
:04023E0000000000BC
:04023F0000000000BB
:0402400000000000BA
:0402410000000000B9
:0402420000000000B8
:0402430000000000B7
:0402440000000000B6
:0402450000000000B5
:0402460000000000B4
:0402470000000000B3
:0402480000000000B2
:0402490000000000B1
:04024A0000000000B0
:04024B0000000000AF
:04024C0000000000AE
:04024D0000000000AD
:04024E0000000000AC
:04024F0000000000AB
:0402500000000000AA
:0402510000000000A9
:0402520000000000A8
:0402530000000000A7
:0402540000000000A6
:0402550000000000A5
:0402560000000000A4
:0402570000000000A3
:0402580000000000A2
:0402590000000000A1
:04025A0000000000A0
:04025B00000000009F
:04025C00000000009E
:04025D00000000009D
:04025E00000000009C
:04025F00000000009B
:04026000000000009A
:040261000000000099
:040262000000000098
:040263000000000097
:040264000000000096
:040265000000000095
:040266000000000094
:040267000000000093
:040268000000000092
:040269000000000091
:04026A000000000090
:04026B00000000008F
:04026C00000000008E
:04026D00000000008D
:04026E00000000008C
:04026F00000000008B
:04027000000000008A
:040271000000000089
:040272000000000088
:040273000000000087
:040274000000000086
:040275000000000085
:040276000000000084
:040277000000000083
:040278000000000082
:040279000000000081
:04027A000000000080
:04027B00000000007F
:04027C00000000007E
:04027D00000000007D
:04027E00000000007C
:04027F00000000007B
:04028000000000007A
:040281000000000079
:040282000000000078
:040283000000000077
:040284000000000076
:040285000000000075
:040286000000000074
:040287000000000073
:040288000000000072
:040289000000000071
:04028A000000000070
:04028B00000000006F
:04028C00000000006E
:04028D00000000006D
:04028E00000000006C
:04028F00000000006B
:04029000000000006A
:040291000000000069
:040292000000000068
:040293000000000067
:040294000000000066
:040295000000000065
:040296000000000064
:040297000000000063
:040298000000000062
:040299000000000061
:04029A000000000060
:04029B00000000005F
:04029C00000000005E
:04029D00000000005D
:04029E00000000005C
:04029F00000000005B
:0402A000000000005A
:0402A1000000000059
:0402A2000000000058
:0402A3000000000057
:0402A4000000000056
:0402A5000000000055
:0402A6000000000054
:0402A7000000000053
:0402A8000000000052
:0402A9000000000051
:0402AA000000000050
:0402AB00000000004F
:0402AC00000000004E
:0402AD00000000004D
:0402AE00000000004C
:0402AF00000000004B
:0402B000000000004A
:0402B1000000000049
:0402B2000000000048
:0402B3000000000047
:0402B4000000000046
:0402B5000000000045
:0402B6000000000044
:0402B7000000000043
:0402B8000000000042
:0402B9000000000041
:0402BA000000000040
:0402BB00000000003F
:0402BC00000000003E
:0402BD00000000003D
:0402BE00000000003C
:0402BF00000000003B
:0402C000000000003A
:0402C1000000000039
:0402C2000000000038
:0402C3000000000037
:0402C4000000000036
:0402C5000000000035
:0402C6000000000034
:0402C7000000000033
:0402C8000000000032
:0402C9000000000031
:0402CA000000000030
:0402CB00000000002F
:0402CC00000000002E
:0402CD00000000002D
:0402CE00000000002C
:0402CF00000000002B
:0402D000000000002A
:0402D1000000000029
:0402D2000000000028
:0402D3000000000027
:0402D4000000000026
:0402D5000000000025
:0402D6000000000024
:0402D7000000000023
:0402D8000000000022
:0402D9000000000021
:0402DA000000000020
:0402DB00000000001F
:0402DC00000000001E
:0402DD00000000001D
:0402DE00000000001C
:0402DF00000000001B
:0402E000000000001A
:0402E1000000000019
:0402E2000000000018
:0402E3000000000017
:0402E4000000000016
:0402E5000000000015
:0402E6000000000014
:0402E7000000000013
:0402E8000000000012
:0402E9000000000011
:0402EA000000000010
:0402EB00000000000F
:0402EC00000000000E
:0402ED00000000000D
:0402EE00000000000C
:0402EF00000000000B
:0402F000000000000A
:0402F1000000000009
:0402F2000000000008
:0402F3000000000007
:0402F4000000000006
:0402F5000000000005
:0402F6000000000004
:0402F7000000000003
:0402F8000000000002
:0402F9000000000001
:0402FA000000000000
:0402FB0000000000FF
:0402FC0000000000FE
:0402FD0000000000FD
:0402FE0000000000FC
:0402FF0000000000FB
:0403000000000000F9
:0403010000000000F8
:0403020000000000F7
:0403030000000000F6
:0403040000000000F5
:0403050000000000F4
:0403060000000000F3
:0403070000000000F2
:0403080000000000F1
:0403090000000000F0
:04030A0000000000EF
:04030B0000000000EE
:04030C0000000000ED
:04030D0000000000EC
:04030E0000000000EB
:04030F0000000000EA
:0403100000000000E9
:0403110000000000E8
:0403120000000000E7
:0403130000000000E6
:0403140000000000E5
:0403150000000000E4
:0403160000000000E3
:0403170000000000E2
:0403180000000000E1
:0403190000000000E0
:04031A0000000000DF
:04031B0000000000DE
:04031C0000000000DD
:04031D0000000000DC
:04031E0000000000DB
:04031F0000000000DA
:0403200000000000D9
:0403210000000000D8
:0403220000000000D7
:0403230000000000D6
:0403240000000000D5
:0403250000000000D4
:0403260000000000D3
:0403270000000000D2
:0403280000000000D1
:0403290000000000D0
:04032A0000000000CF
:04032B0000000000CE
:04032C0000000000CD
:04032D0000000000CC
:04032E0000000000CB
:04032F0000000000CA
:0403300000000000C9
:0403310000000000C8
:0403320000000000C7
:0403330000000000C6
:0403340000000000C5
:0403350000000000C4
:0403360000000000C3
:0403370000000000C2
:0403380000000000C1
:0403390000000000C0
:04033A0000000000BF
:04033B0000000000BE
:04033C0000000000BD
:04033D0000000000BC
:04033E0000000000BB
:04033F0000000000BA
:0403400000000000B9
:0403410000000000B8
:0403420000000000B7
:0403430000000000B6
:0403440000000000B5
:0403450000000000B4
:0403460000000000B3
:0403470000000000B2
:0403480000000000B1
:0403490000000000B0
:04034A0000000000AF
:04034B0000000000AE
:04034C0000000000AD
:04034D0000000000AC
:04034E0000000000AB
:04034F0000000000AA
:0403500000000000A9
:0403510000000000A8
:0403520000000000A7
:0403530000000000A6
:0403540000000000A5
:0403550000000000A4
:0403560000000000A3
:0403570000000000A2
:0403580000000000A1
:0403590000000000A0
:04035A00000000009F
:04035B00000000009E
:04035C00000000009D
:04035D00000000009C
:04035E00000000009B
:04035F00000000009A
:040360000000000099
:040361000000000098
:040362000000000097
:040363000000000096
:040364000000000095
:040365000000000094
:040366000000000093
:040367000000000092
:040368000000000091
:040369000000000090
:04036A00000000008F
:04036B00000000008E
:04036C00000000008D
:04036D00000000008C
:04036E00000000008B
:04036F00000000008A
:040370000000000089
:040371000000000088
:040372000000000087
:040373000000000086
:040374000000000085
:040375000000000084
:040376000000000083
:040377000000000082
:040378000000000081
:040379000000000080
:04037A00000000007F
:04037B00000000007E
:04037C00000000007D
:04037D00000000007C
:04037E00000000007B
:04037F00000000007A
:040380000000000079
:040381000000000078
:040382000000000077
:040383000000000076
:040384000000000075
:040385000000000074
:040386000000000073
:040387000000000072
:040388000000000071
:040389000000000070
:04038A00000000006F
:04038B00000000006E
:04038C00000000006D
:04038D00000000006C
:04038E00000000006B
:04038F00000000006A
:040390000000000069
:040391000000000068
:040392000000000067
:040393000000000066
:040394000000000065
:040395000000000064
:040396000000000063
:040397000000000062
:040398000000000061
:040399000000000060
:04039A00000000005F
:04039B00000000005E
:04039C00000000005D
:04039D00000000005C
:04039E00000000005B
:04039F00000000005A
:0403A0000000000059
:0403A1000000000058
:0403A2000000000057
:0403A3000000000056
:0403A4000000000055
:0403A5000000000054
:0403A6000000000053
:0403A7000000000052
:0403A8000000000051
:0403A9000000000050
:0403AA00000000004F
:0403AB00000000004E
:0403AC00000000004D
:0403AD00000000004C
:0403AE00000000004B
:0403AF00000000004A
:0403B0000000000049
:0403B1000000000048
:0403B2000000000047
:0403B3000000000046
:0403B4000000000045
:0403B5000000000044
:0403B6000000000043
:0403B7000000000042
:0403B8000000000041
:0403B9000000000040
:0403BA00000000003F
:0403BB00000000003E
:0403BC00000000003D
:0403BD00000000003C
:0403BE00000000003B
:0403BF00000000003A
:0403C0000000000039
:0403C1000000000038
:0403C2000000000037
:0403C3000000000036
:0403C4000000000035
:0403C5000000000034
:0403C6000000000033
:0403C7000000000032
:0403C8000000000031
:0403C9000000000030
:0403CA00000000002F
:0403CB00000000002E
:0403CC00000000002D
:0403CD00000000002C
:0403CE00000000002B
:0403CF00000000002A
:0403D0000000000029
:0403D1000000000028
:0403D2000000000027
:0403D3000000000026
:0403D4000000000025
:0403D5000000000024
:0403D6000000000023
:0403D7000000000022
:0403D8000000000021
:0403D9000000000020
:0403DA00000000001F
:0403DB00000000001E
:0403DC00000000001D
:0403DD00000000001C
:0403DE00000000001B
:0403DF00000000001A
:0403E0000000000019
:0403E1000000000018
:0403E2000000000017
:0403E3000000000016
:0403E4000000000015
:0403E5000000000014
:0403E6000000000013
:0403E7000000000012
:0403E8000000000011
:0403E9000000000010
:0403EA00000000000F
:0403EB00000000000E
:0403EC00000000000D
:0403ED00000000000C
:0403EE00000000000B
:0403EF00000000000A
:0403F0000000000009
:0403F1000000000008
:0403F2000000000007
:0403F3000000000006
:0403F4000000000005
:0403F5000000000004
:0403F6000000000003
:0403F7000000000002
:0403F8000000000001
:0403F9000000000000
:0403FA0000000000FF
:0403FB0000000000FE
:0403FC0000000000FD
:0403FD0000000000FC
:0403FE0000000000FB
:0403FF0000000000FA
:0404000000000000F8
:0404010000000000F7
:0404020000000000F6
:0404030000000000F5
:0404040000000000F4
:0404050000000000F3
:0404060000000000F2
:0404070000000000F1
:0404080000000000F0
:0404090000000000EF
:04040A0000000000EE
:04040B0000000000ED
:04040C0000000000EC
:04040D0000000000EB
:04040E0000000000EA
:04040F0000000000E9
:0404100000000000E8
:0404110000000000E7
:0404120000000000E6
:0404130000000000E5
:0404140000000000E4
:0404150000000000E3
:0404160000000000E2
:0404170000000000E1
:0404180000000000E0
:0404190000000000DF
:04041A0000000000DE
:04041B0000000000DD
:04041C0000000000DC
:04041D0000000000DB
:04041E0000000000DA
:04041F0000000000D9
:0404200000000000D8
:0404210000000000D7
:0404220000000000D6
:0404230000000000D5
:0404240000000000D4
:0404250000000000D3
:0404260000000000D2
:0404270000000000D1
:0404280000000000D0
:0404290000000000CF
:04042A0000000000CE
:04042B0000000000CD
:04042C0000000000CC
:04042D0000000000CB
:04042E0000000000CA
:04042F0000000000C9
:0404300000000000C8
:0404310000000000C7
:0404320000000000C6
:0404330000000000C5
:0404340000000000C4
:0404350000000000C3
:0404360000000000C2
:0404370000000000C1
:0404380000000000C0
:0404390000000000BF
:04043A0000000000BE
:04043B0000000000BD
:04043C0000000000BC
:04043D0000000000BB
:04043E0000000000BA
:04043F0000000000B9
:0404400000000000B8
:0404410000000000B7
:0404420000000000B6
:0404430000000000B5
:0404440000000000B4
:0404450000000000B3
:0404460000000000B2
:0404470000000000B1
:0404480000000000B0
:0404490000000000AF
:04044A0000000000AE
:04044B0000000000AD
:04044C0000000000AC
:04044D0000000000AB
:04044E0000000000AA
:04044F0000000000A9
:0404500000000000A8
:0404510000000000A7
:0404520000000000A6
:0404530000000000A5
:0404540000000000A4
:0404550000000000A3
:0404560000000000A2
:0404570000000000A1
:0404580000000000A0
:04045900000000009F
:04045A00000000009E
:04045B00000000009D
:04045C00000000009C
:04045D00000000009B
:04045E00000000009A
:04045F000000000099
:040460000000000098
:040461000000000097
:040462000000000096
:040463000000000095
:040464000000000094
:040465000000000093
:040466000000000092
:040467000000000091
:040468000000000090
:04046900000000008F
:04046A00000000008E
:04046B00000000008D
:04046C00000000008C
:04046D00000000008B
:04046E00000000008A
:04046F000000000089
:040470000000000088
:040471000000000087
:040472000000000086
:040473000000000085
:040474000000000084
:040475000000000083
:040476000000000082
:040477000000000081
:040478000000000080
:04047900000000007F
:04047A00000000007E
:04047B00000000007D
:04047C00000000007C
:04047D00000000007B
:04047E00000000007A
:04047F000000000079
:040480000000000078
:040481000000000077
:040482000000000076
:040483000000000075
:040484000000000074
:040485000000000073
:040486000000000072
:040487000000000071
:040488000000000070
:04048900000000006F
:04048A00000000006E
:04048B00000000006D
:04048C00000000006C
:04048D00000000006B
:04048E00000000006A
:04048F000000000069
:040490000000000068
:040491000000000067
:040492000000000066
:040493000000000065
:040494000000000064
:040495000000000063
:040496000000000062
:040497000000000061
:040498000000000060
:04049900000000005F
:04049A00000000005E
:04049B00000000005D
:04049C00000000005C
:04049D00000000005B
:04049E00000000005A
:04049F000000000059
:0404A0000000000058
:0404A1000000000057
:0404A2000000000056
:0404A3000000000055
:0404A4000000000054
:0404A5000000000053
:0404A6000000000052
:0404A7000000000051
:0404A8000000000050
:0404A900000000004F
:0404AA00000000004E
:0404AB00000000004D
:0404AC00000000004C
:0404AD00000000004B
:0404AE00000000004A
:0404AF000000000049
:0404B0000000000048
:0404B1000000000047
:0404B2000000000046
:0404B3000000000045
:0404B4000000000044
:0404B5000000000043
:0404B6000000000042
:0404B7000000000041
:0404B8000000000040
:0404B900000000003F
:0404BA00000000003E
:0404BB00000000003D
:0404BC00000000003C
:0404BD00000000003B
:0404BE00000000003A
:0404BF000000000039
:0404C0000000000038
:0404C1000000000037
:0404C2000000000036
:0404C3000000000035
:0404C4000000000034
:0404C5000000000033
:0404C6000000000032
:0404C7000000000031
:0404C8000000000030
:0404C900000000002F
:0404CA00000000002E
:0404CB00000000002D
:0404CC00000000002C
:0404CD00000000002B
:0404CE00000000002A
:0404CF000000000029
:0404D0000000000028
:0404D1000000000027
:0404D2000000000026
:0404D3000000000025
:0404D4000000000024
:0404D5000000000023
:0404D6000000000022
:0404D7000000000021
:0404D8000000000020
:0404D900000000001F
:0404DA00000000001E
:0404DB00000000001D
:0404DC00000000001C
:0404DD00000000001B
:0404DE00000000001A
:0404DF000000000019
:0404E0000000000018
:0404E1000000000017
:0404E2000000000016
:0404E3000000000015
:0404E4000000000014
:0404E5000000000013
:0404E6000000000012
:0404E7000000000011
:0404E8000000000010
:0404E900000000000F
:0404EA00000000000E
:0404EB00000000000D
:0404EC00000000000C
:0404ED00000000000B
:0404EE00000000000A
:0404EF000000000009
:0404F0000000000008
:0404F1000000000007
:0404F2000000000006
:0404F3000000000005
:0404F4000000000004
:0404F5000000000003
:0404F6000000000002
:0404F7000000000001
:0404F8000000000000
:0404F90000000000FF
:0404FA0000000000FE
:0404FB0000000000FD
:0404FC0000000000FC
:0404FD0000000000FB
:0404FE0000000000FA
:0404FF0000000000F9
:0405000000000000F7
:0405010000000000F6
:0405020000000000F5
:0405030000000000F4
:0405040000000000F3
:0405050000000000F2
:0405060000000000F1
:0405070000000000F0
:0405080000000000EF
:0405090000000000EE
:04050A0000000000ED
:04050B0000000000EC
:04050C0000000000EB
:04050D0000000000EA
:04050E0000000000E9
:04050F0000000000E8
:0405100000000000E7
:0405110000000000E6
:0405120000000000E5
:0405130000000000E4
:0405140000000000E3
:0405150000000000E2
:0405160000000000E1
:0405170000000000E0
:0405180000000000DF
:0405190000000000DE
:04051A0000000000DD
:04051B0000000000DC
:04051C0000000000DB
:04051D0000000000DA
:04051E0000000000D9
:04051F0000000000D8
:0405200000000000D7
:0405210000000000D6
:0405220000000000D5
:0405230000000000D4
:0405240000000000D3
:0405250000000000D2
:0405260000000000D1
:0405270000000000D0
:0405280000000000CF
:0405290000000000CE
:04052A0000000000CD
:04052B0000000000CC
:04052C0000000000CB
:04052D0000000000CA
:04052E0000000000C9
:04052F0000000000C8
:0405300000000000C7
:0405310000000000C6
:0405320000000000C5
:0405330000000000C4
:0405340000000000C3
:0405350000000000C2
:0405360000000000C1
:0405370000000000C0
:0405380000000000BF
:0405390000000000BE
:04053A0000000000BD
:04053B0000000000BC
:04053C0000000000BB
:04053D0000000000BA
:04053E0000000000B9
:04053F0000000000B8
:0405400000000000B7
:0405410000000000B6
:0405420000000000B5
:0405430000000000B4
:0405440000000000B3
:0405450000000000B2
:0405460000000000B1
:0405470000000000B0
:0405480000000000AF
:0405490000000000AE
:04054A0000000000AD
:04054B0000000000AC
:04054C0000000000AB
:04054D0000000000AA
:04054E0000000000A9
:04054F0000000000A8
:0405500000000000A7
:0405510000000000A6
:0405520000000000A5
:0405530000000000A4
:0405540000000000A3
:0405550000000000A2
:0405560000000000A1
:0405570000000000A0
:04055800000000009F
:04055900000000009E
:04055A00000000009D
:04055B00000000009C
:04055C00000000009B
:04055D00000000009A
:04055E000000000099
:04055F000000000098
:040560000000000097
:040561000000000096
:040562000000000095
:040563000000000094
:040564000000000093
:040565000000000092
:040566000000000091
:040567000000000090
:04056800000000008F
:04056900000000008E
:04056A00000000008D
:04056B00000000008C
:04056C00000000008B
:04056D00000000008A
:04056E000000000089
:04056F000000000088
:040570000000000087
:040571000000000086
:040572000000000085
:040573000000000084
:040574000000000083
:040575000000000082
:040576000000000081
:040577000000000080
:04057800000000007F
:04057900000000007E
:04057A00000000007D
:04057B00000000007C
:04057C00000000007B
:04057D00000000007A
:04057E000000000079
:04057F000000000078
:040580000000000077
:040581000000000076
:040582000000000075
:040583000000000074
:040584000000000073
:040585000000000072
:040586000000000071
:040587000000000070
:04058800000000006F
:04058900000000006E
:04058A00000000006D
:04058B00000000006C
:04058C00000000006B
:04058D00000000006A
:04058E000000000069
:04058F000000000068
:040590000000000067
:040591000000000066
:040592000000000065
:040593000000000064
:040594000000000063
:040595000000000062
:040596000000000061
:040597000000000060
:04059800000000005F
:04059900000000005E
:04059A00000000005D
:04059B00000000005C
:04059C00000000005B
:04059D00000000005A
:04059E000000000059
:04059F000000000058
:0405A0000000000057
:0405A1000000000056
:0405A2000000000055
:0405A3000000000054
:0405A4000000000053
:0405A5000000000052
:0405A6000000000051
:0405A7000000000050
:0405A800000000004F
:0405A900000000004E
:0405AA00000000004D
:0405AB00000000004C
:0405AC00000000004B
:0405AD00000000004A
:0405AE000000000049
:0405AF000000000048
:0405B0000000000047
:0405B1000000000046
:0405B2000000000045
:0405B3000000000044
:0405B4000000000043
:0405B5000000000042
:0405B6000000000041
:0405B7000000000040
:0405B800000000003F
:0405B900000000003E
:0405BA00000000003D
:0405BB00000000003C
:0405BC00000000003B
:0405BD00000000003A
:0405BE000000000039
:0405BF000000000038
:0405C0000000000037
:0405C1000000000036
:0405C2000000000035
:0405C3000000000034
:0405C4000000000033
:0405C5000000000032
:0405C6000000000031
:0405C7000000000030
:0405C800000000002F
:0405C900000000002E
:0405CA00000000002D
:0405CB00000000002C
:0405CC00000000002B
:0405CD00000000002A
:0405CE000000000029
:0405CF000000000028
:0405D0000000000027
:0405D1000000000026
:0405D2000000000025
:0405D3000000000024
:0405D4000000000023
:0405D5000000000022
:0405D6000000000021
:0405D7000000000020
:0405D800000000001F
:0405D900000000001E
:0405DA00000000001D
:0405DB00000000001C
:0405DC00000000001B
:0405DD00000000001A
:0405DE000000000019
:0405DF000000000018
:0405E0000000000017
:0405E1000000000016
:0405E2000000000015
:0405E3000000000014
:0405E4000000000013
:0405E5000000000012
:0405E6000000000011
:0405E7000000000010
:0405E800000000000F
:0405E900000000000E
:0405EA00000000000D
:0405EB00000000000C
:0405EC00000000000B
:0405ED00000000000A
:0405EE000000000009
:0405EF000000000008
:0405F0000000000007
:0405F1000000000006
:0405F2000000000005
:0405F3000000000004
:0405F4000000000003
:0405F5000000000002
:0405F6000000000001
:0405F7000000000000
:0405F80000000000FF
:0405F90000000000FE
:0405FA0000000000FD
:0405FB0000000000FC
:0405FC0000000000FB
:0405FD0000000000FA
:0405FE0000000000F9
:0405FF0000000000F8
:0406000000000000F6
:0406010000000000F5
:0406020000000000F4
:0406030000000000F3
:0406040000000000F2
:0406050000000000F1
:0406060000000000F0
:0406070000000000EF
:0406080000000000EE
:0406090000000000ED
:04060A0000000000EC
:04060B0000000000EB
:04060C0000000000EA
:04060D0000000000E9
:04060E0000000000E8
:04060F0000000000E7
:0406100000000000E6
:0406110000000000E5
:0406120000000000E4
:0406130000000000E3
:0406140000000000E2
:0406150000000000E1
:0406160000000000E0
:0406170000000000DF
:0406180000000000DE
:0406190000000000DD
:04061A0000000000DC
:04061B0000000000DB
:04061C0000000000DA
:04061D0000000000D9
:04061E0000000000D8
:04061F0000000000D7
:0406200000000000D6
:0406210000000000D5
:0406220000000000D4
:0406230000000000D3
:0406240000000000D2
:0406250000000000D1
:0406260000000000D0
:0406270000000000CF
:0406280000000000CE
:0406290000000000CD
:04062A0000000000CC
:04062B0000000000CB
:04062C0000000000CA
:04062D0000000000C9
:04062E0000000000C8
:04062F0000000000C7
:0406300000000000C6
:0406310000000000C5
:0406320000000000C4
:0406330000000000C3
:0406340000000000C2
:0406350000000000C1
:0406360000000000C0
:0406370000000000BF
:0406380000000000BE
:0406390000000000BD
:04063A0000000000BC
:04063B0000000000BB
:04063C0000000000BA
:04063D0000000000B9
:04063E0000000000B8
:04063F0000000000B7
:0406400000000000B6
:0406410000000000B5
:0406420000000000B4
:0406430000000000B3
:0406440000000000B2
:0406450000000000B1
:0406460000000000B0
:0406470000000000AF
:0406480000000000AE
:0406490000000000AD
:04064A0000000000AC
:04064B0000000000AB
:04064C0000000000AA
:04064D0000000000A9
:04064E0000000000A8
:04064F0000000000A7
:0406500000000000A6
:0406510000000000A5
:0406520000000000A4
:0406530000000000A3
:0406540000000000A2
:0406550000000000A1
:0406560000000000A0
:04065700000000009F
:04065800000000009E
:04065900000000009D
:04065A00000000009C
:04065B00000000009B
:04065C00000000009A
:04065D000000000099
:04065E000000000098
:04065F000000000097
:040660000000000096
:040661000000000095
:040662000000000094
:040663000000000093
:040664000000000092
:040665000000000091
:040666000000000090
:04066700000000008F
:04066800000000008E
:04066900000000008D
:04066A00000000008C
:04066B00000000008B
:04066C00000000008A
:04066D000000000089
:04066E000000000088
:04066F000000000087
:040670000000000086
:040671000000000085
:040672000000000084
:040673000000000083
:040674000000000082
:040675000000000081
:040676000000000080
:04067700000000007F
:04067800000000007E
:04067900000000007D
:04067A00000000007C
:04067B00000000007B
:04067C00000000007A
:04067D000000000079
:04067E000000000078
:04067F000000000077
:040680000000000076
:040681000000000075
:040682000000000074
:040683000000000073
:040684000000000072
:040685000000000071
:040686000000000070
:04068700000000006F
:04068800000000006E
:04068900000000006D
:04068A00000000006C
:04068B00000000006B
:04068C00000000006A
:04068D000000000069
:04068E000000000068
:04068F000000000067
:040690000000000066
:040691000000000065
:040692000000000064
:040693000000000063
:040694000000000062
:040695000000000061
:040696000000000060
:04069700000000005F
:04069800000000005E
:04069900000000005D
:04069A00000000005C
:04069B00000000005B
:04069C00000000005A
:04069D000000000059
:04069E000000000058
:04069F000000000057
:0406A0000000000056
:0406A1000000000055
:0406A2000000000054
:0406A3000000000053
:0406A4000000000052
:0406A5000000000051
:0406A6000000000050
:0406A700000000004F
:0406A800000000004E
:0406A900000000004D
:0406AA00000000004C
:0406AB00000000004B
:0406AC00000000004A
:0406AD000000000049
:0406AE000000000048
:0406AF000000000047
:0406B0000000000046
:0406B1000000000045
:0406B2000000000044
:0406B3000000000043
:0406B4000000000042
:0406B5000000000041
:0406B6000000000040
:0406B700000000003F
:0406B800000000003E
:0406B900000000003D
:0406BA00000000003C
:0406BB00000000003B
:0406BC00000000003A
:0406BD000000000039
:0406BE000000000038
:0406BF000000000037
:0406C0000000000036
:0406C1000000000035
:0406C2000000000034
:0406C3000000000033
:0406C4000000000032
:0406C5000000000031
:0406C6000000000030
:0406C700000000002F
:0406C800000000002E
:0406C900000000002D
:0406CA00000000002C
:0406CB00000000002B
:0406CC00000000002A
:0406CD000000000029
:0406CE000000000028
:0406CF000000000027
:0406D0000000000026
:0406D1000000000025
:0406D2000000000024
:0406D3000000000023
:0406D4000000000022
:0406D5000000000021
:0406D6000000000020
:0406D700000000001F
:0406D800000000001E
:0406D900000000001D
:0406DA00000000001C
:0406DB00000000001B
:0406DC00000000001A
:0406DD000000000019
:0406DE000000000018
:0406DF000000000017
:0406E0000000000016
:0406E1000000000015
:0406E2000000000014
:0406E3000000000013
:0406E4000000000012
:0406E5000000000011
:0406E6000000000010
:0406E700000000000F
:0406E800000000000E
:0406E900000000000D
:0406EA00000000000C
:0406EB00000000000B
:0406EC00000000000A
:0406ED000000000009
:0406EE000000000008
:0406EF000000000007
:0406F0000000000006
:0406F1000000000005
:0406F2000000000004
:0406F3000000000003
:0406F4000000000002
:0406F5000000000001
:0406F6000000000000
:0406F70000000000FF
:0406F80000000000FE
:0406F90000000000FD
:0406FA0000000000FC
:0406FB0000000000FB
:0406FC0000000000FA
:0406FD0000000000F9
:0406FE0000000000F8
:0406FF0000000000F7
:0407000000000000F5
:0407010000000000F4
:0407020000000000F3
:0407030000000000F2
:0407040000000000F1
:0407050000000000F0
:0407060000000000EF
:0407070000000000EE
:0407080000000000ED
:0407090000000000EC
:04070A0000000000EB
:04070B0000000000EA
:04070C0000000000E9
:04070D0000000000E8
:04070E0000000000E7
:04070F0000000000E6
:0407100000000000E5
:0407110000000000E4
:0407120000000000E3
:0407130000000000E2
:0407140000000000E1
:0407150000000000E0
:0407160000000000DF
:0407170000000000DE
:0407180000000000DD
:0407190000000000DC
:04071A0000000000DB
:04071B0000000000DA
:04071C0000000000D9
:04071D0000000000D8
:04071E0000000000D7
:04071F0000000000D6
:0407200000000000D5
:0407210000000000D4
:0407220000000000D3
:0407230000000000D2
:0407240000000000D1
:0407250000000000D0
:0407260000000000CF
:0407270000000000CE
:0407280000000000CD
:0407290000000000CC
:04072A0000000000CB
:04072B0000000000CA
:04072C0000000000C9
:04072D0000000000C8
:04072E0000000000C7
:04072F0000000000C6
:0407300000000000C5
:0407310000000000C4
:0407320000000000C3
:0407330000000000C2
:0407340000000000C1
:0407350000000000C0
:0407360000000000BF
:0407370000000000BE
:0407380000000000BD
:0407390000000000BC
:04073A0000000000BB
:04073B0000000000BA
:04073C0000000000B9
:04073D0000000000B8
:04073E0000000000B7
:04073F0000000000B6
:0407400000000000B5
:0407410000000000B4
:0407420000000000B3
:0407430000000000B2
:0407440000000000B1
:0407450000000000B0
:0407460000000000AF
:0407470000000000AE
:0407480000000000AD
:0407490000000000AC
:04074A0000000000AB
:04074B0000000000AA
:04074C0000000000A9
:04074D0000000000A8
:04074E0000000000A7
:04074F0000000000A6
:0407500000000000A5
:0407510000000000A4
:0407520000000000A3
:0407530000000000A2
:0407540000000000A1
:0407550000000000A0
:04075600000000009F
:04075700000000009E
:04075800000000009D
:04075900000000009C
:04075A00000000009B
:04075B00000000009A
:04075C000000000099
:04075D000000000098
:04075E000000000097
:04075F000000000096
:040760000000000095
:040761000000000094
:040762000000000093
:040763000000000092
:040764000000000091
:040765000000000090
:04076600000000008F
:04076700000000008E
:04076800000000008D
:04076900000000008C
:04076A00000000008B
:04076B00000000008A
:04076C000000000089
:04076D000000000088
:04076E000000000087
:04076F000000000086
:040770000000000085
:040771000000000084
:040772000000000083
:040773000000000082
:040774000000000081
:040775000000000080
:04077600000000007F
:04077700000000007E
:04077800000000007D
:04077900000000007C
:04077A00000000007B
:04077B00000000007A
:04077C000000000079
:04077D000000000078
:04077E000000000077
:04077F000000000076
:040780000000000075
:040781000000000074
:040782000000000073
:040783000000000072
:040784000000000071
:040785000000000070
:04078600000000006F
:04078700000000006E
:04078800000000006D
:04078900000000006C
:04078A00000000006B
:04078B00000000006A
:04078C000000000069
:04078D000000000068
:04078E000000000067
:04078F000000000066
:040790000000000065
:040791000000000064
:040792000000000063
:040793000000000062
:040794000000000061
:040795000000000060
:04079600000000005F
:04079700000000005E
:04079800000000005D
:04079900000000005C
:04079A00000000005B
:04079B00000000005A
:04079C000000000059
:04079D000000000058
:04079E000000000057
:04079F000000000056
:0407A0000000000055
:0407A1000000000054
:0407A2000000000053
:0407A3000000000052
:0407A4000000000051
:0407A5000000000050
:0407A600000000004F
:0407A700000000004E
:0407A800000000004D
:0407A900000000004C
:0407AA00000000004B
:0407AB00000000004A
:0407AC000000000049
:0407AD000000000048
:0407AE000000000047
:0407AF000000000046
:0407B0000000000045
:0407B1000000000044
:0407B2000000000043
:0407B3000000000042
:0407B4000000000041
:0407B5000000000040
:0407B600000000003F
:0407B700000000003E
:0407B800000000003D
:0407B900000000003C
:0407BA00000000003B
:0407BB00000000003A
:0407BC000000000039
:0407BD000000000038
:0407BE000000000037
:0407BF000000000036
:0407C0000000000035
:0407C1000000000034
:0407C2000000000033
:0407C3000000000032
:0407C4000000000031
:0407C5000000000030
:0407C600000000002F
:0407C700000000002E
:0407C800000000002D
:0407C900000000002C
:0407CA00000000002B
:0407CB00000000002A
:0407CC000000000029
:0407CD000000000028
:0407CE000000000027
:0407CF000000000026
:0407D0000000000025
:0407D1000000000024
:0407D2000000000023
:0407D3000000000022
:0407D4000000000021
:0407D5000000000020
:0407D600000000001F
:0407D700000000001E
:0407D800000000001D
:0407D900000000001C
:0407DA00000000001B
:0407DB00000000001A
:0407DC000000000019
:0407DD000000000018
:0407DE000000000017
:0407DF000000000016
:0407E0000000000015
:0407E1000000000014
:0407E2000000000013
:0407E3000000000012
:0407E4000000000011
:0407E5000000000010
:0407E600000000000F
:0407E700000000000E
:0407E800000000000D
:0407E900000000000C
:0407EA00000000000B
:0407EB00000000000A
:0407EC000000000009
:0407ED000000000008
:0407EE000000000007
:0407EF000000000006
:0407F0000000000005
:0407F1000000000004
:0407F2000000000003
:0407F3000000000002
:0407F4000000000001
:0407F5000000000000
:0407F60000000000FF
:0407F70000000000FE
:0407F80000000000FD
:0407F90000000000FC
:0407FA0000000000FB
:0407FB0000000000FA
:0407FC0000000000F9
:0407FD0000000000F8
:0407FE0000000000F7
:0407FF0000000000F6
:0408000000000000F4
:0408010000000000F3
:0408020000000000F2
:0408030000000000F1
:0408040000000000F0
:0408050000000000EF
:0408060000000000EE
:0408070000000000ED
:0408080000000000EC
:0408090000000000EB
:04080A0000000000EA
:04080B0000000000E9
:04080C0000000000E8
:04080D0000000000E7
:04080E0000000000E6
:04080F0000000000E5
:0408100000000000E4
:0408110000000000E3
:0408120000000000E2
:0408130000000000E1
:0408140000000000E0
:0408150000000000DF
:0408160000000000DE
:0408170000000000DD
:0408180000000000DC
:0408190000000000DB
:04081A0000000000DA
:04081B0000000000D9
:04081C0000000000D8
:04081D0000000000D7
:04081E0000000000D6
:04081F0000000000D5
:0408200000000000D4
:0408210000000000D3
:0408220000000000D2
:0408230000000000D1
:0408240000000000D0
:0408250000000000CF
:0408260000000000CE
:0408270000000000CD
:0408280000000000CC
:0408290000000000CB
:04082A0000000000CA
:04082B0000000000C9
:04082C0000000000C8
:04082D0000000000C7
:04082E0000000000C6
:04082F0000000000C5
:0408300000000000C4
:0408310000000000C3
:0408320000000000C2
:0408330000000000C1
:0408340000000000C0
:0408350000000000BF
:0408360000000000BE
:0408370000000000BD
:0408380000000000BC
:0408390000000000BB
:04083A0000000000BA
:04083B0000000000B9
:04083C0000000000B8
:04083D0000000000B7
:04083E0000000000B6
:04083F0000000000B5
:0408400000000000B4
:0408410000000000B3
:0408420000000000B2
:0408430000000000B1
:0408440000000000B0
:0408450000000000AF
:0408460000000000AE
:0408470000000000AD
:0408480000000000AC
:0408490000000000AB
:04084A0000000000AA
:04084B0000000000A9
:04084C0000000000A8
:04084D0000000000A7
:04084E0000000000A6
:04084F0000000000A5
:0408500000000000A4
:0408510000000000A3
:0408520000000000A2
:0408530000000000A1
:0408540000000000A0
:04085500000000009F
:04085600000000009E
:04085700000000009D
:04085800000000009C
:04085900000000009B
:04085A00000000009A
:04085B000000000099
:04085C000000000098
:04085D000000000097
:04085E000000000096
:04085F000000000095
:040860000000000094
:040861000000000093
:040862000000000092
:040863000000000091
:040864000000000090
:04086500000000008F
:04086600000000008E
:04086700000000008D
:04086800000000008C
:04086900000000008B
:04086A00000000008A
:04086B000000000089
:04086C000000000088
:04086D000000000087
:04086E000000000086
:04086F000000000085
:040870000000000084
:040871000000000083
:040872000000000082
:040873000000000081
:040874000000000080
:04087500000000007F
:04087600000000007E
:04087700000000007D
:04087800000000007C
:04087900000000007B
:04087A00000000007A
:04087B000000000079
:04087C000000000078
:04087D000000000077
:04087E000000000076
:04087F000000000075
:040880000000000074
:040881000000000073
:040882000000000072
:040883000000000071
:040884000000000070
:04088500000000006F
:04088600000000006E
:04088700000000006D
:04088800000000006C
:04088900000000006B
:04088A00000000006A
:04088B000000000069
:04088C000000000068
:04088D000000000067
:04088E000000000066
:04088F000000000065
:040890000000000064
:040891000000000063
:040892000000000062
:040893000000000061
:040894000000000060
:04089500000000005F
:04089600000000005E
:04089700000000005D
:04089800000000005C
:04089900000000005B
:04089A00000000005A
:04089B000000000059
:04089C000000000058
:04089D000000000057
:04089E000000000056
:04089F000000000055
:0408A0000000000054
:0408A1000000000053
:0408A2000000000052
:0408A3000000000051
:0408A4000000000050
:0408A500000000004F
:0408A600000000004E
:0408A700000000004D
:0408A800000000004C
:0408A900000000004B
:0408AA00000000004A
:0408AB000000000049
:0408AC000000000048
:0408AD000000000047
:0408AE000000000046
:0408AF000000000045
:0408B0000000000044
:0408B1000000000043
:0408B2000000000042
:0408B3000000000041
:0408B4000000000040
:0408B500000000003F
:0408B600000000003E
:0408B700000000003D
:0408B800000000003C
:0408B900000000003B
:0408BA00000000003A
:0408BB000000000039
:0408BC000000000038
:0408BD000000000037
:0408BE000000000036
:0408BF000000000035
:0408C0000000000034
:0408C1000000000033
:0408C2000000000032
:0408C3000000000031
:0408C4000000000030
:0408C500000000002F
:0408C600000000002E
:0408C700000000002D
:0408C800000000002C
:0408C900000000002B
:0408CA00000000002A
:0408CB000000000029
:0408CC000000000028
:0408CD000000000027
:0408CE000000000026
:0408CF000000000025
:0408D0000000000024
:0408D1000000000023
:0408D2000000000022
:0408D3000000000021
:0408D4000000000020
:0408D500000000001F
:0408D600000000001E
:0408D700000000001D
:0408D800000000001C
:0408D900000000001B
:0408DA00000000001A
:0408DB000000000019
:0408DC000000000018
:0408DD000000000017
:0408DE000000000016
:0408DF000000000015
:0408E0000000000014
:0408E1000000000013
:0408E2000000000012
:0408E3000000000011
:0408E4000000000010
:0408E500000000000F
:0408E600000000000E
:0408E700000000000D
:0408E800000000000C
:0408E900000000000B
:0408EA00000000000A
:0408EB000000000009
:0408EC000000000008
:0408ED000000000007
:0408EE000000000006
:0408EF000000000005
:0408F0000000000004
:0408F1000000000003
:0408F2000000000002
:0408F3000000000001
:0408F4000000000000
:0408F50000000000FF
:0408F60000000000FE
:0408F70000000000FD
:0408F80000000000FC
:0408F90000000000FB
:0408FA0000000000FA
:0408FB0000000000F9
:0408FC0000000000F8
:0408FD0000000000F7
:0408FE0000000000F6
:0408FF0000000000F5
:0409000000000000F3
:0409010000000000F2
:0409020000000000F1
:0409030000000000F0
:0409040000000000EF
:0409050000000000EE
:0409060000000000ED
:0409070000000000EC
:0409080000000000EB
:0409090000000000EA
:04090A0000000000E9
:04090B0000000000E8
:04090C0000000000E7
:04090D0000000000E6
:04090E0000000000E5
:04090F0000000000E4
:0409100000000000E3
:0409110000000000E2
:0409120000000000E1
:0409130000000000E0
:0409140000000000DF
:0409150000000000DE
:0409160000000000DD
:0409170000000000DC
:0409180000000000DB
:0409190000000000DA
:04091A0000000000D9
:04091B0000000000D8
:04091C0000000000D7
:04091D0000000000D6
:04091E0000000000D5
:04091F0000000000D4
:0409200000000000D3
:0409210000000000D2
:0409220000000000D1
:0409230000000000D0
:0409240000000000CF
:0409250000000000CE
:0409260000000000CD
:0409270000000000CC
:0409280000000000CB
:0409290000000000CA
:04092A0000000000C9
:04092B0000000000C8
:04092C0000000000C7
:04092D0000000000C6
:04092E0000000000C5
:04092F0000000000C4
:0409300000000000C3
:0409310000000000C2
:0409320000000000C1
:0409330000000000C0
:0409340000000000BF
:0409350000000000BE
:0409360000000000BD
:0409370000000000BC
:0409380000000000BB
:0409390000000000BA
:04093A0000000000B9
:04093B0000000000B8
:04093C0000000000B7
:04093D0000000000B6
:04093E0000000000B5
:04093F0000000000B4
:0409400000000000B3
:0409410000000000B2
:0409420000000000B1
:0409430000000000B0
:0409440000000000AF
:0409450000000000AE
:0409460000000000AD
:0409470000000000AC
:0409480000000000AB
:0409490000000000AA
:04094A0000000000A9
:04094B0000000000A8
:04094C0000000000A7
:04094D0000000000A6
:04094E0000000000A5
:04094F0000000000A4
:0409500000000000A3
:0409510000000000A2
:0409520000000000A1
:0409530000000000A0
:04095400000000009F
:04095500000000009E
:04095600000000009D
:04095700000000009C
:04095800000000009B
:04095900000000009A
:04095A000000000099
:04095B000000000098
:04095C000000000097
:04095D000000000096
:04095E000000000095
:04095F000000000094
:040960000000000093
:040961000000000092
:040962000000000091
:040963000000000090
:04096400000000008F
:04096500000000008E
:04096600000000008D
:04096700000000008C
:04096800000000008B
:04096900000000008A
:04096A000000000089
:04096B000000000088
:04096C000000000087
:04096D000000000086
:04096E000000000085
:04096F000000000084
:040970000000000083
:040971000000000082
:040972000000000081
:040973000000000080
:04097400000000007F
:04097500000000007E
:04097600000000007D
:04097700000000007C
:04097800000000007B
:04097900000000007A
:04097A000000000079
:04097B000000000078
:04097C000000000077
:04097D000000000076
:04097E000000000075
:04097F000000000074
:040980000000000073
:040981000000000072
:040982000000000071
:040983000000000070
:04098400000000006F
:04098500000000006E
:04098600000000006D
:04098700000000006C
:04098800000000006B
:04098900000000006A
:04098A000000000069
:04098B000000000068
:04098C000000000067
:04098D000000000066
:04098E000000000065
:04098F000000000064
:040990000000000063
:040991000000000062
:040992000000000061
:040993000000000060
:04099400000000005F
:04099500000000005E
:04099600000000005D
:04099700000000005C
:04099800000000005B
:04099900000000005A
:04099A000000000059
:04099B000000000058
:04099C000000000057
:04099D000000000056
:04099E000000000055
:04099F000000000054
:0409A0000000000053
:0409A1000000000052
:0409A2000000000051
:0409A3000000000050
:0409A400000000004F
:0409A500000000004E
:0409A600000000004D
:0409A700000000004C
:0409A800000000004B
:0409A900000000004A
:0409AA000000000049
:0409AB000000000048
:0409AC000000000047
:0409AD000000000046
:0409AE000000000045
:0409AF000000000044
:0409B0000000000043
:0409B1000000000042
:0409B2000000000041
:0409B3000000000040
:0409B400000000003F
:0409B500000000003E
:0409B600000000003D
:0409B700000000003C
:0409B800000000003B
:0409B900000000003A
:0409BA000000000039
:0409BB000000000038
:0409BC000000000037
:0409BD000000000036
:0409BE000000000035
:0409BF000000000034
:0409C0000000000033
:0409C1000000000032
:0409C2000000000031
:0409C3000000000030
:0409C400000000002F
:0409C500000000002E
:0409C600000000002D
:0409C700000000002C
:0409C800000000002B
:0409C900000000002A
:0409CA000000000029
:0409CB000000000028
:0409CC000000000027
:0409CD000000000026
:0409CE000000000025
:0409CF000000000024
:0409D0000000000023
:0409D1000000000022
:0409D2000000000021
:0409D3000000000020
:0409D400000000001F
:0409D500000000001E
:0409D600000000001D
:0409D700000000001C
:0409D800000000001B
:0409D900000000001A
:0409DA000000000019
:0409DB000000000018
:0409DC000000000017
:0409DD000000000016
:0409DE000000000015
:0409DF000000000014
:0409E0000000000013
:0409E1000000000012
:0409E2000000000011
:0409E3000000000010
:0409E400000000000F
:0409E500000000000E
:0409E600000000000D
:0409E700000000000C
:0409E800000000000B
:0409E900000000000A
:0409EA000000000009
:0409EB000000000008
:0409EC000000000007
:0409ED000000000006
:0409EE000000000005
:0409EF000000000004
:0409F0000000000003
:0409F1000000000002
:0409F2000000000001
:0409F3000000000000
:0409F40000000000FF
:0409F50000000000FE
:0409F60000000000FD
:0409F70000000000FC
:0409F80000000000FB
:0409F90000000000FA
:0409FA0000000000F9
:0409FB0000000000F8
:0409FC0000000000F7
:0409FD0000000000F6
:0409FE0000000000F5
:0409FF0000000000F4
:040A000000000000F2
:040A010000000000F1
:040A020000000000F0
:040A030000000000EF
:040A040000000000EE
:040A050000000000ED
:040A060000000000EC
:040A070000000000EB
:040A080000000000EA
:040A090000000000E9
:040A0A0000000000E8
:040A0B0000000000E7
:040A0C0000000000E6
:040A0D0000000000E5
:040A0E0000000000E4
:040A0F0000000000E3
:040A100000000000E2
:040A110000000000E1
:040A120000000000E0
:040A130000000000DF
:040A140000000000DE
:040A150000000000DD
:040A160000000000DC
:040A170000000000DB
:040A180000000000DA
:040A190000000000D9
:040A1A0000000000D8
:040A1B0000000000D7
:040A1C0000000000D6
:040A1D0000000000D5
:040A1E0000000000D4
:040A1F0000000000D3
:040A200000000000D2
:040A210000000000D1
:040A220000000000D0
:040A230000000000CF
:040A240000000000CE
:040A250000000000CD
:040A260000000000CC
:040A270000000000CB
:040A280000000000CA
:040A290000000000C9
:040A2A0000000000C8
:040A2B0000000000C7
:040A2C0000000000C6
:040A2D0000000000C5
:040A2E0000000000C4
:040A2F0000000000C3
:040A300000000000C2
:040A310000000000C1
:040A320000000000C0
:040A330000000000BF
:040A340000000000BE
:040A350000000000BD
:040A360000000000BC
:040A370000000000BB
:040A380000000000BA
:040A390000000000B9
:040A3A0000000000B8
:040A3B0000000000B7
:040A3C0000000000B6
:040A3D0000000000B5
:040A3E0000000000B4
:040A3F0000000000B3
:040A400000000000B2
:040A410000000000B1
:040A420000000000B0
:040A430000000000AF
:040A440000000000AE
:040A450000000000AD
:040A460000000000AC
:040A470000000000AB
:040A480000000000AA
:040A490000000000A9
:040A4A0000000000A8
:040A4B0000000000A7
:040A4C0000000000A6
:040A4D0000000000A5
:040A4E0000000000A4
:040A4F0000000000A3
:040A500000000000A2
:040A510000000000A1
:040A520000000000A0
:040A5300000000009F
:040A5400000000009E
:040A5500000000009D
:040A5600000000009C
:040A5700000000009B
:040A5800000000009A
:040A59000000000099
:040A5A000000000098
:040A5B000000000097
:040A5C000000000096
:040A5D000000000095
:040A5E000000000094
:040A5F000000000093
:040A60000000000092
:040A61000000000091
:040A62000000000090
:040A6300000000008F
:040A6400000000008E
:040A6500000000008D
:040A6600000000008C
:040A6700000000008B
:040A6800000000008A
:040A69000000000089
:040A6A000000000088
:040A6B000000000087
:040A6C000000000086
:040A6D000000000085
:040A6E000000000084
:040A6F000000000083
:040A70000000000082
:040A71000000000081
:040A72000000000080
:040A7300000000007F
:040A7400000000007E
:040A7500000000007D
:040A7600000000007C
:040A7700000000007B
:040A7800000000007A
:040A79000000000079
:040A7A000000000078
:040A7B000000000077
:040A7C000000000076
:040A7D000000000075
:040A7E000000000074
:040A7F000000000073
:040A80000000000072
:040A81000000000071
:040A82000000000070
:040A8300000000006F
:040A8400000000006E
:040A8500000000006D
:040A8600000000006C
:040A8700000000006B
:040A8800000000006A
:040A89000000000069
:040A8A000000000068
:040A8B000000000067
:040A8C000000000066
:040A8D000000000065
:040A8E000000000064
:040A8F000000000063
:040A90000000000062
:040A91000000000061
:040A92000000000060
:040A9300000000005F
:040A9400000000005E
:040A9500000000005D
:040A9600000000005C
:040A9700000000005B
:040A9800000000005A
:040A99000000000059
:040A9A000000000058
:040A9B000000000057
:040A9C000000000056
:040A9D000000000055
:040A9E000000000054
:040A9F000000000053
:040AA0000000000052
:040AA1000000000051
:040AA2000000000050
:040AA300000000004F
:040AA400000000004E
:040AA500000000004D
:040AA600000000004C
:040AA700000000004B
:040AA800000000004A
:040AA9000000000049
:040AAA000000000048
:040AAB000000000047
:040AAC000000000046
:040AAD000000000045
:040AAE000000000044
:040AAF000000000043
:040AB0000000000042
:040AB1000000000041
:040AB2000000000040
:040AB300000000003F
:040AB400000000003E
:040AB500000000003D
:040AB600000000003C
:040AB700000000003B
:040AB800000000003A
:040AB9000000000039
:040ABA000000000038
:040ABB000000000037
:040ABC000000000036
:040ABD000000000035
:040ABE000000000034
:040ABF000000000033
:040AC0000000000032
:040AC1000000000031
:040AC2000000000030
:040AC300000000002F
:040AC400000000002E
:040AC500000000002D
:040AC600000000002C
:040AC700000000002B
:040AC800000000002A
:040AC9000000000029
:040ACA000000000028
:040ACB000000000027
:040ACC000000000026
:040ACD000000000025
:040ACE000000000024
:040ACF000000000023
:040AD0000000000022
:040AD1000000000021
:040AD2000000000020
:040AD300000000001F
:040AD400000000001E
:040AD500000000001D
:040AD600000000001C
:040AD700000000001B
:040AD800000000001A
:040AD9000000000019
:040ADA000000000018
:040ADB000000000017
:040ADC000000000016
:040ADD000000000015
:040ADE000000000014
:040ADF000000000013
:040AE0000000000012
:040AE1000000000011
:040AE2000000000010
:040AE300000000000F
:040AE400000000000E
:040AE500000000000D
:040AE600000000000C
:040AE700000000000B
:040AE800000000000A
:040AE9000000000009
:040AEA000000000008
:040AEB000000000007
:040AEC000000000006
:040AED000000000005
:040AEE000000000004
:040AEF000000000003
:040AF0000000000002
:040AF1000000000001
:040AF2000000000000
:040AF30000000000FF
:040AF40000000000FE
:040AF50000000000FD
:040AF60000000000FC
:040AF70000000000FB
:040AF80000000000FA
:040AF90000000000F9
:040AFA0000000000F8
:040AFB0000000000F7
:040AFC0000000000F6
:040AFD0000000000F5
:040AFE0000000000F4
:040AFF0000000000F3
:040B000000000000F1
:040B010000000000F0
:040B020000000000EF
:040B030000000000EE
:040B040000000000ED
:040B050000000000EC
:040B060000000000EB
:040B070000000000EA
:040B080000000000E9
:040B090000000000E8
:040B0A0000000000E7
:040B0B0000000000E6
:040B0C0000000000E5
:040B0D0000000000E4
:040B0E0000000000E3
:040B0F0000000000E2
:040B100000000000E1
:040B110000000000E0
:040B120000000000DF
:040B130000000000DE
:040B140000000000DD
:040B150000000000DC
:040B160000000000DB
:040B170000000000DA
:040B180000000000D9
:040B190000000000D8
:040B1A0000000000D7
:040B1B0000000000D6
:040B1C0000000000D5
:040B1D0000000000D4
:040B1E0000000000D3
:040B1F0000000000D2
:040B200000000000D1
:040B210000000000D0
:040B220000000000CF
:040B230000000000CE
:040B240000000000CD
:040B250000000000CC
:040B260000000000CB
:040B270000000000CA
:040B280000000000C9
:040B290000000000C8
:040B2A0000000000C7
:040B2B0000000000C6
:040B2C0000000000C5
:040B2D0000000000C4
:040B2E0000000000C3
:040B2F0000000000C2
:040B300000000000C1
:040B310000000000C0
:040B320000000000BF
:040B330000000000BE
:040B340000000000BD
:040B350000000000BC
:040B360000000000BB
:040B370000000000BA
:040B380000000000B9
:040B390000000000B8
:040B3A0000000000B7
:040B3B0000000000B6
:040B3C0000000000B5
:040B3D0000000000B4
:040B3E0000000000B3
:040B3F0000000000B2
:040B400000000000B1
:040B410000000000B0
:040B420000000000AF
:040B430000000000AE
:040B440000000000AD
:040B450000000000AC
:040B460000000000AB
:040B470000000000AA
:040B480000000000A9
:040B490000000000A8
:040B4A0000000000A7
:040B4B0000000000A6
:040B4C0000000000A5
:040B4D0000000000A4
:040B4E0000000000A3
:040B4F0000000000A2
:040B500000000000A1
:040B510000000000A0
:040B5200000000009F
:040B5300000000009E
:040B5400000000009D
:040B5500000000009C
:040B5600000000009B
:040B5700000000009A
:040B58000000000099
:040B59000000000098
:040B5A000000000097
:040B5B000000000096
:040B5C000000000095
:040B5D000000000094
:040B5E000000000093
:040B5F000000000092
:040B60000000000091
:040B61000000000090
:040B6200000000008F
:040B6300000000008E
:040B6400000000008D
:040B6500000000008C
:040B6600000000008B
:040B6700000000008A
:040B68000000000089
:040B69000000000088
:040B6A000000000087
:040B6B000000000086
:040B6C000000000085
:040B6D000000000084
:040B6E000000000083
:040B6F000000000082
:040B70000000000081
:040B71000000000080
:040B7200000000007F
:040B7300000000007E
:040B7400000000007D
:040B7500000000007C
:040B7600000000007B
:040B7700000000007A
:040B78000000000079
:040B79000000000078
:040B7A000000000077
:040B7B000000000076
:040B7C000000000075
:040B7D000000000074
:040B7E000000000073
:040B7F000000000072
:040B80000000000071
:040B81000000000070
:040B8200000000006F
:040B8300000000006E
:040B8400000000006D
:040B8500000000006C
:040B8600000000006B
:040B8700000000006A
:040B88000000000069
:040B89000000000068
:040B8A000000000067
:040B8B000000000066
:040B8C000000000065
:040B8D000000000064
:040B8E000000000063
:040B8F000000000062
:040B90000000000061
:040B91000000000060
:040B9200000000005F
:040B9300000000005E
:040B9400000000005D
:040B9500000000005C
:040B9600000000005B
:040B9700000000005A
:040B98000000000059
:040B99000000000058
:040B9A000000000057
:040B9B000000000056
:040B9C000000000055
:040B9D000000000054
:040B9E000000000053
:040B9F000000000052
:040BA0000000000051
:040BA1000000000050
:040BA200000000004F
:040BA300000000004E
:040BA400000000004D
:040BA500000000004C
:040BA600000000004B
:040BA700000000004A
:040BA8000000000049
:040BA9000000000048
:040BAA000000000047
:040BAB000000000046
:040BAC000000000045
:040BAD000000000044
:040BAE000000000043
:040BAF000000000042
:040BB0000000000041
:040BB1000000000040
:040BB200000000003F
:040BB300000000003E
:040BB400000000003D
:040BB500000000003C
:040BB600000000003B
:040BB700000000003A
:040BB8000000000039
:040BB9000000000038
:040BBA000000000037
:040BBB000000000036
:040BBC000000000035
:040BBD000000000034
:040BBE000000000033
:040BBF000000000032
:040BC0000000000031
:040BC1000000000030
:040BC200000000002F
:040BC300000000002E
:040BC400000000002D
:040BC500000000002C
:040BC600000000002B
:040BC700000000002A
:040BC8000000000029
:040BC9000000000028
:040BCA000000000027
:040BCB000000000026
:040BCC000000000025
:040BCD000000000024
:040BCE000000000023
:040BCF000000000022
:040BD0000000000021
:040BD1000000000020
:040BD200000000001F
:040BD300000000001E
:040BD400000000001D
:040BD500000000001C
:040BD600000000001B
:040BD700000000001A
:040BD8000000000019
:040BD9000000000018
:040BDA000000000017
:040BDB000000000016
:040BDC000000000015
:040BDD000000000014
:040BDE000000000013
:040BDF000000000012
:040BE0000000000011
:040BE1000000000010
:040BE200000000000F
:040BE300000000000E
:040BE400000000000D
:040BE500000000000C
:040BE600000000000B
:040BE700000000000A
:040BE8000000000009
:040BE9000000000008
:040BEA000000000007
:040BEB000000000006
:040BEC000000000005
:040BED000000000004
:040BEE000000000003
:040BEF000000000002
:040BF0000000000001
:040BF1000000000000
:040BF20000000000FF
:040BF30000000000FE
:040BF40000000000FD
:040BF50000000000FC
:040BF60000000000FB
:040BF70000000000FA
:040BF80000000000F9
:040BF90000000000F8
:040BFA0000000000F7
:040BFB0000000000F6
:040BFC0000000000F5
:040BFD0000000000F4
:040BFE0000000000F3
:040BFF0000000000F2
:040C000000000000F0
:040C010000000000EF
:040C020000000000EE
:040C030000000000ED
:040C040000000000EC
:040C050000000000EB
:040C060000000000EA
:040C070000000000E9
:040C080000000000E8
:040C090000000000E7
:040C0A0000000000E6
:040C0B0000000000E5
:040C0C0000000000E4
:040C0D0000000000E3
:040C0E0000000000E2
:040C0F0000000000E1
:040C100000000000E0
:040C110000000000DF
:040C120000000000DE
:040C130000000000DD
:040C140000000000DC
:040C150000000000DB
:040C160000000000DA
:040C170000000000D9
:040C180000000000D8
:040C190000000000D7
:040C1A0000000000D6
:040C1B0000000000D5
:040C1C0000000000D4
:040C1D0000000000D3
:040C1E0000000000D2
:040C1F0000000000D1
:040C200000000000D0
:040C210000000000CF
:040C220000000000CE
:040C230000000000CD
:040C240000000000CC
:040C250000000000CB
:040C260000000000CA
:040C270000000000C9
:040C280000000000C8
:040C290000000000C7
:040C2A0000000000C6
:040C2B0000000000C5
:040C2C0000000000C4
:040C2D0000000000C3
:040C2E0000000000C2
:040C2F0000000000C1
:040C300000000000C0
:040C310000000000BF
:040C320000000000BE
:040C330000000000BD
:040C340000000000BC
:040C350000000000BB
:040C360000000000BA
:040C370000000000B9
:040C380000000000B8
:040C390000000000B7
:040C3A0000000000B6
:040C3B0000000000B5
:040C3C0000000000B4
:040C3D0000000000B3
:040C3E0000000000B2
:040C3F0000000000B1
:040C400000000000B0
:040C410000000000AF
:040C420000000000AE
:040C430000000000AD
:040C440000000000AC
:040C450000000000AB
:040C460000000000AA
:040C470000000000A9
:040C480000000000A8
:040C490000000000A7
:040C4A0000000000A6
:040C4B0000000000A5
:040C4C0000000000A4
:040C4D0000000000A3
:040C4E0000000000A2
:040C4F0000000000A1
:040C500000000000A0
:040C5100000000009F
:040C5200000000009E
:040C5300000000009D
:040C5400000000009C
:040C5500000000009B
:040C5600000000009A
:040C57000000000099
:040C58000000000098
:040C59000000000097
:040C5A000000000096
:040C5B000000000095
:040C5C000000000094
:040C5D000000000093
:040C5E000000000092
:040C5F000000000091
:040C60000000000090
:040C6100000000008F
:040C6200000000008E
:040C6300000000008D
:040C6400000000008C
:040C6500000000008B
:040C6600000000008A
:040C67000000000089
:040C68000000000088
:040C69000000000087
:040C6A000000000086
:040C6B000000000085
:040C6C000000000084
:040C6D000000000083
:040C6E000000000082
:040C6F000000000081
:040C70000000000080
:040C7100000000007F
:040C7200000000007E
:040C7300000000007D
:040C7400000000007C
:040C7500000000007B
:040C7600000000007A
:040C77000000000079
:040C78000000000078
:040C79000000000077
:040C7A000000000076
:040C7B000000000075
:040C7C000000000074
:040C7D000000000073
:040C7E000000000072
:040C7F000000000071
:040C80000000000070
:040C8100000000006F
:040C8200000000006E
:040C8300000000006D
:040C8400000000006C
:040C8500000000006B
:040C8600000000006A
:040C87000000000069
:040C88000000000068
:040C89000000000067
:040C8A000000000066
:040C8B000000000065
:040C8C000000000064
:040C8D000000000063
:040C8E000000000062
:040C8F000000000061
:040C90000000000060
:040C9100000000005F
:040C9200000000005E
:040C9300000000005D
:040C9400000000005C
:040C9500000000005B
:040C9600000000005A
:040C97000000000059
:040C98000000000058
:040C99000000000057
:040C9A000000000056
:040C9B000000000055
:040C9C000000000054
:040C9D000000000053
:040C9E000000000052
:040C9F000000000051
:040CA0000000000050
:040CA100000000004F
:040CA200000000004E
:040CA300000000004D
:040CA400000000004C
:040CA500000000004B
:040CA600000000004A
:040CA7000000000049
:040CA8000000000048
:040CA9000000000047
:040CAA000000000046
:040CAB000000000045
:040CAC000000000044
:040CAD000000000043
:040CAE000000000042
:040CAF000000000041
:040CB0000000000040
:040CB100000000003F
:040CB200000000003E
:040CB300000000003D
:040CB400000000003C
:040CB500000000003B
:040CB600000000003A
:040CB7000000000039
:040CB8000000000038
:040CB9000000000037
:040CBA000000000036
:040CBB000000000035
:040CBC000000000034
:040CBD000000000033
:040CBE000000000032
:040CBF000000000031
:040CC0000000000030
:040CC100000000002F
:040CC200000000002E
:040CC300000000002D
:040CC400000000002C
:040CC500000000002B
:040CC600000000002A
:040CC7000000000029
:040CC8000000000028
:040CC9000000000027
:040CCA000000000026
:040CCB000000000025
:040CCC000000000024
:040CCD000000000023
:040CCE000000000022
:040CCF000000000021
:040CD0000000000020
:040CD100000000001F
:040CD200000000001E
:040CD300000000001D
:040CD400000000001C
:040CD500000000001B
:040CD600000000001A
:040CD7000000000019
:040CD8000000000018
:040CD9000000000017
:040CDA000000000016
:040CDB000000000015
:040CDC000000000014
:040CDD000000000013
:040CDE000000000012
:040CDF000000000011
:040CE0000000000010
:040CE100000000000F
:040CE200000000000E
:040CE300000000000D
:040CE400000000000C
:040CE500000000000B
:040CE600000000000A
:040CE7000000000009
:040CE8000000000008
:040CE9000000000007
:040CEA000000000006
:040CEB000000000005
:040CEC000000000004
:040CED000000000003
:040CEE000000000002
:040CEF000000000001
:040CF0000000000000
:040CF10000000000FF
:040CF20000000000FE
:040CF30000000000FD
:040CF40000000000FC
:040CF50000000000FB
:040CF60000000000FA
:040CF70000000000F9
:040CF80000000000F8
:040CF90000000000F7
:040CFA0000000000F6
:040CFB0000000000F5
:040CFC0000000000F4
:040CFD0000000000F3
:040CFE0000000000F2
:040CFF0000000000F1
:040D000000000000EF
:040D010000000000EE
:040D020000000000ED
:040D030000000000EC
:040D040000000000EB
:040D050000000000EA
:040D060000000000E9
:040D070000000000E8
:040D080000000000E7
:040D090000000000E6
:040D0A0000000000E5
:040D0B0000000000E4
:040D0C0000000000E3
:040D0D0000000000E2
:040D0E0000000000E1
:040D0F0000000000E0
:040D100000000000DF
:040D110000000000DE
:040D120000000000DD
:040D130000000000DC
:040D140000000000DB
:040D150000000000DA
:040D160000000000D9
:040D170000000000D8
:040D180000000000D7
:040D190000000000D6
:040D1A0000000000D5
:040D1B0000000000D4
:040D1C0000000000D3
:040D1D0000000000D2
:040D1E0000000000D1
:040D1F0000000000D0
:040D200000000000CF
:040D210000000000CE
:040D220000000000CD
:040D230000000000CC
:040D240000000000CB
:040D250000000000CA
:040D260000000000C9
:040D270000000000C8
:040D280000000000C7
:040D290000000000C6
:040D2A0000000000C5
:040D2B0000000000C4
:040D2C0000000000C3
:040D2D0000000000C2
:040D2E0000000000C1
:040D2F0000000000C0
:040D300000000000BF
:040D310000000000BE
:040D320000000000BD
:040D330000000000BC
:040D340000000000BB
:040D350000000000BA
:040D360000000000B9
:040D370000000000B8
:040D380000000000B7
:040D390000000000B6
:040D3A0000000000B5
:040D3B0000000000B4
:040D3C0000000000B3
:040D3D0000000000B2
:040D3E0000000000B1
:040D3F0000000000B0
:040D400000000000AF
:040D410000000000AE
:040D420000000000AD
:040D430000000000AC
:040D440000000000AB
:040D450000000000AA
:040D460000000000A9
:040D470000000000A8
:040D480000000000A7
:040D490000000000A6
:040D4A0000000000A5
:040D4B0000000000A4
:040D4C0000000000A3
:040D4D0000000000A2
:040D4E0000000000A1
:040D4F0000000000A0
:040D5000000000009F
:040D5100000000009E
:040D5200000000009D
:040D5300000000009C
:040D5400000000009B
:040D5500000000009A
:040D56000000000099
:040D57000000000098
:040D58000000000097
:040D59000000000096
:040D5A000000000095
:040D5B000000000094
:040D5C000000000093
:040D5D000000000092
:040D5E000000000091
:040D5F000000000090
:040D6000000000008F
:040D6100000000008E
:040D6200000000008D
:040D6300000000008C
:040D6400000000008B
:040D6500000000008A
:040D66000000000089
:040D67000000000088
:040D68000000000087
:040D69000000000086
:040D6A000000000085
:040D6B000000000084
:040D6C000000000083
:040D6D000000000082
:040D6E000000000081
:040D6F000000000080
:040D7000000000007F
:040D7100000000007E
:040D7200000000007D
:040D7300000000007C
:040D7400000000007B
:040D7500000000007A
:040D76000000000079
:040D77000000000078
:040D78000000000077
:040D79000000000076
:040D7A000000000075
:040D7B000000000074
:040D7C000000000073
:040D7D000000000072
:040D7E000000000071
:040D7F000000000070
:040D8000000000006F
:040D8100000000006E
:040D8200000000006D
:040D8300000000006C
:040D8400000000006B
:040D8500000000006A
:040D86000000000069
:040D87000000000068
:040D88000000000067
:040D89000000000066
:040D8A000000000065
:040D8B000000000064
:040D8C000000000063
:040D8D000000000062
:040D8E000000000061
:040D8F000000000060
:040D9000000000005F
:040D9100000000005E
:040D9200000000005D
:040D9300000000005C
:040D9400000000005B
:040D9500000000005A
:040D96000000000059
:040D97000000000058
:040D98000000000057
:040D99000000000056
:040D9A000000000055
:040D9B000000000054
:040D9C000000000053
:040D9D000000000052
:040D9E000000000051
:040D9F000000000050
:040DA000000000004F
:040DA100000000004E
:040DA200000000004D
:040DA300000000004C
:040DA400000000004B
:040DA500000000004A
:040DA6000000000049
:040DA7000000000048
:040DA8000000000047
:040DA9000000000046
:040DAA000000000045
:040DAB000000000044
:040DAC000000000043
:040DAD000000000042
:040DAE000000000041
:040DAF000000000040
:040DB000000000003F
:040DB100000000003E
:040DB200000000003D
:040DB300000000003C
:040DB400000000003B
:040DB500000000003A
:040DB6000000000039
:040DB7000000000038
:040DB8000000000037
:040DB9000000000036
:040DBA000000000035
:040DBB000000000034
:040DBC000000000033
:040DBD000000000032
:040DBE000000000031
:040DBF000000000030
:040DC000000000002F
:040DC100000000002E
:040DC200000000002D
:040DC300000000002C
:040DC400000000002B
:040DC500000000002A
:040DC6000000000029
:040DC7000000000028
:040DC8000000000027
:040DC9000000000026
:040DCA000000000025
:040DCB000000000024
:040DCC000000000023
:040DCD000000000022
:040DCE000000000021
:040DCF000000000020
:040DD000000000001F
:040DD100000000001E
:040DD200000000001D
:040DD300000000001C
:040DD400000000001B
:040DD500000000001A
:040DD6000000000019
:040DD7000000000018
:040DD8000000000017
:040DD9000000000016
:040DDA000000000015
:040DDB000000000014
:040DDC000000000013
:040DDD000000000012
:040DDE000000000011
:040DDF000000000010
:040DE000000000000F
:040DE100000000000E
:040DE200000000000D
:040DE300000000000C
:040DE400000000000B
:040DE500000000000A
:040DE6000000000009
:040DE7000000000008
:040DE8000000000007
:040DE9000000000006
:040DEA000000000005
:040DEB000000000004
:040DEC000000000003
:040DED000000000002
:040DEE000000000001
:040DEF000000000000
:040DF00000000000FF
:040DF10000000000FE
:040DF20000000000FD
:040DF30000000000FC
:040DF40000000000FB
:040DF50000000000FA
:040DF60000000000F9
:040DF70000000000F8
:040DF80000000000F7
:040DF90000000000F6
:040DFA0000000000F5
:040DFB0000000000F4
:040DFC0000000000F3
:040DFD0000000000F2
:040DFE0000000000F1
:040DFF0000000000F0
:040E000000000000EE
:040E010000000000ED
:040E020000000000EC
:040E030000000000EB
:040E040000000000EA
:040E050000000000E9
:040E060000000000E8
:040E070000000000E7
:040E080000000000E6
:040E090000000000E5
:040E0A0000000000E4
:040E0B0000000000E3
:040E0C0000000000E2
:040E0D0000000000E1
:040E0E0000000000E0
:040E0F0000000000DF
:040E100000000000DE
:040E110000000000DD
:040E120000000000DC
:040E130000000000DB
:040E140000000000DA
:040E150000000000D9
:040E160000000000D8
:040E170000000000D7
:040E180000000000D6
:040E190000000000D5
:040E1A0000000000D4
:040E1B0000000000D3
:040E1C0000000000D2
:040E1D0000000000D1
:040E1E0000000000D0
:040E1F0000000000CF
:040E200000000000CE
:040E210000000000CD
:040E220000000000CC
:040E230000000000CB
:040E240000000000CA
:040E250000000000C9
:040E260000000000C8
:040E270000000000C7
:040E280000000000C6
:040E290000000000C5
:040E2A0000000000C4
:040E2B0000000000C3
:040E2C0000000000C2
:040E2D0000000000C1
:040E2E0000000000C0
:040E2F0000000000BF
:040E300000000000BE
:040E310000000000BD
:040E320000000000BC
:040E330000000000BB
:040E340000000000BA
:040E350000000000B9
:040E360000000000B8
:040E370000000000B7
:040E380000000000B6
:040E390000000000B5
:040E3A0000000000B4
:040E3B0000000000B3
:040E3C0000000000B2
:040E3D0000000000B1
:040E3E0000000000B0
:040E3F0000000000AF
:040E400000000000AE
:040E410000000000AD
:040E420000000000AC
:040E430000000000AB
:040E440000000000AA
:040E450000000000A9
:040E460000000000A8
:040E470000000000A7
:040E480000000000A6
:040E490000000000A5
:040E4A0000000000A4
:040E4B0000000000A3
:040E4C0000000000A2
:040E4D0000000000A1
:040E4E0000000000A0
:040E4F00000000009F
:040E5000000000009E
:040E5100000000009D
:040E5200000000009C
:040E5300000000009B
:040E5400000000009A
:040E55000000000099
:040E56000000000098
:040E57000000000097
:040E58000000000096
:040E59000000000095
:040E5A000000000094
:040E5B000000000093
:040E5C000000000092
:040E5D000000000091
:040E5E000000000090
:040E5F00000000008F
:040E6000000000008E
:040E6100000000008D
:040E6200000000008C
:040E6300000000008B
:040E6400000000008A
:040E65000000000089
:040E66000000000088
:040E67000000000087
:040E68000000000086
:040E69000000000085
:040E6A000000000084
:040E6B000000000083
:040E6C000000000082
:040E6D000000000081
:040E6E000000000080
:040E6F00000000007F
:040E7000000000007E
:040E7100000000007D
:040E7200000000007C
:040E7300000000007B
:040E7400000000007A
:040E75000000000079
:040E76000000000078
:040E77000000000077
:040E78000000000076
:040E79000000000075
:040E7A000000000074
:040E7B000000000073
:040E7C000000000072
:040E7D000000000071
:040E7E000000000070
:040E7F00000000006F
:040E8000000000006E
:040E8100000000006D
:040E8200000000006C
:040E8300000000006B
:040E8400000000006A
:040E85000000000069
:040E86000000000068
:040E87000000000067
:040E88000000000066
:040E89000000000065
:040E8A000000000064
:040E8B000000000063
:040E8C000000000062
:040E8D000000000061
:040E8E000000000060
:040E8F00000000005F
:040E9000000000005E
:040E9100000000005D
:040E9200000000005C
:040E9300000000005B
:040E9400000000005A
:040E95000000000059
:040E96000000000058
:040E97000000000057
:040E98000000000056
:040E99000000000055
:040E9A000000000054
:040E9B000000000053
:040E9C000000000052
:040E9D000000000051
:040E9E000000000050
:040E9F00000000004F
:040EA000000000004E
:040EA100000000004D
:040EA200000000004C
:040EA300000000004B
:040EA400000000004A
:040EA5000000000049
:040EA6000000000048
:040EA7000000000047
:040EA8000000000046
:040EA9000000000045
:040EAA000000000044
:040EAB000000000043
:040EAC000000000042
:040EAD000000000041
:040EAE000000000040
:040EAF00000000003F
:040EB000000000003E
:040EB100000000003D
:040EB200000000003C
:040EB300000000003B
:040EB400000000003A
:040EB5000000000039
:040EB6000000000038
:040EB7000000000037
:040EB8000000000036
:040EB9000000000035
:040EBA000000000034
:040EBB000000000033
:040EBC000000000032
:040EBD000000000031
:040EBE000000000030
:040EBF00000000002F
:040EC000000000002E
:040EC100000000002D
:040EC200000000002C
:040EC300000000002B
:040EC400000000002A
:040EC5000000000029
:040EC6000000000028
:040EC7000000000027
:040EC8000000000026
:040EC9000000000025
:040ECA000000000024
:040ECB000000000023
:040ECC000000000022
:040ECD000000000021
:040ECE000000000020
:040ECF00000000001F
:040ED000000000001E
:040ED100000000001D
:040ED200000000001C
:040ED300000000001B
:040ED400000000001A
:040ED5000000000019
:040ED6000000000018
:040ED7000000000017
:040ED8000000000016
:040ED9000000000015
:040EDA000000000014
:040EDB000000000013
:040EDC000000000012
:040EDD000000000011
:040EDE000000000010
:040EDF00000000000F
:040EE000000000000E
:040EE100000000000D
:040EE200000000000C
:040EE300000000000B
:040EE400000000000A
:040EE5000000000009
:040EE6000000000008
:040EE7000000000007
:040EE8000000000006
:040EE9000000000005
:040EEA000000000004
:040EEB000000000003
:040EEC000000000002
:040EED000000000001
:040EEE000000000000
:040EEF0000000000FF
:040EF00000000000FE
:040EF10000000000FD
:040EF20000000000FC
:040EF30000000000FB
:040EF40000000000FA
:040EF50000000000F9
:040EF60000000000F8
:040EF70000000000F7
:040EF80000000000F6
:040EF90000000000F5
:040EFA0000000000F4
:040EFB0000000000F3
:040EFC0000000000F2
:040EFD0000000000F1
:040EFE0000000000F0
:040EFF0000000000EF
:040F000000000000ED
:040F010000000000EC
:040F020000000000EB
:040F030000000000EA
:040F040000000000E9
:040F050000000000E8
:040F060000000000E7
:040F070000000000E6
:040F080000000000E5
:040F090000000000E4
:040F0A0000000000E3
:040F0B0000000000E2
:040F0C0000000000E1
:040F0D0000000000E0
:040F0E0000000000DF
:040F0F0000000000DE
:040F100000000000DD
:040F110000000000DC
:040F120000000000DB
:040F130000000000DA
:040F140000000000D9
:040F150000000000D8
:040F160000000000D7
:040F170000000000D6
:040F180000000000D5
:040F190000000000D4
:040F1A0000000000D3
:040F1B0000000000D2
:040F1C0000000000D1
:040F1D0000000000D0
:040F1E0000000000CF
:040F1F0000000000CE
:040F200000000000CD
:040F210000000000CC
:040F220000000000CB
:040F230000000000CA
:040F240000000000C9
:040F250000000000C8
:040F260000000000C7
:040F270000000000C6
:040F280000000000C5
:040F290000000000C4
:040F2A0000000000C3
:040F2B0000000000C2
:040F2C0000000000C1
:040F2D0000000000C0
:040F2E0000000000BF
:040F2F0000000000BE
:040F300000000000BD
:040F310000000000BC
:040F320000000000BB
:040F330000000000BA
:040F340000000000B9
:040F350000000000B8
:040F360000000000B7
:040F370000000000B6
:040F380000000000B5
:040F390000000000B4
:040F3A0000000000B3
:040F3B0000000000B2
:040F3C0000000000B1
:040F3D0000000000B0
:040F3E0000000000AF
:040F3F0000000000AE
:040F400000000000AD
:040F410000000000AC
:040F420000000000AB
:040F430000000000AA
:040F440000000000A9
:040F450000000000A8
:040F460000000000A7
:040F470000000000A6
:040F480000000000A5
:040F490000000000A4
:040F4A0000000000A3
:040F4B0000000000A2
:040F4C0000000000A1
:040F4D0000000000A0
:040F4E00000000009F
:040F4F00000000009E
:040F5000000000009D
:040F5100000000009C
:040F5200000000009B
:040F5300000000009A
:040F54000000000099
:040F55000000000098
:040F56000000000097
:040F57000000000096
:040F58000000000095
:040F59000000000094
:040F5A000000000093
:040F5B000000000092
:040F5C000000000091
:040F5D000000000090
:040F5E00000000008F
:040F5F00000000008E
:040F6000000000008D
:040F6100000000008C
:040F6200000000008B
:040F6300000000008A
:040F64000000000089
:040F65000000000088
:040F66000000000087
:040F67000000000086
:040F68000000000085
:040F69000000000084
:040F6A000000000083
:040F6B000000000082
:040F6C000000000081
:040F6D000000000080
:040F6E00000000007F
:040F6F00000000007E
:040F7000000000007D
:040F7100000000007C
:040F7200000000007B
:040F7300000000007A
:040F74000000000079
:040F75000000000078
:040F76000000000077
:040F77000000000076
:040F78000000000075
:040F79000000000074
:040F7A000000000073
:040F7B000000000072
:040F7C000000000071
:040F7D000000000070
:040F7E00000000006F
:040F7F00000000006E
:040F8000000000006D
:040F8100000000006C
:040F8200000000006B
:040F8300000000006A
:040F84000000000069
:040F85000000000068
:040F86000000000067
:040F87000000000066
:040F88000000000065
:040F89000000000064
:040F8A000000000063
:040F8B000000000062
:040F8C000000000061
:040F8D000000000060
:040F8E00000000005F
:040F8F00000000005E
:040F9000000000005D
:040F9100000000005C
:040F9200000000005B
:040F9300000000005A
:040F94000000000059
:040F95000000000058
:040F96000000000057
:040F97000000000056
:040F98000000000055
:040F99000000000054
:040F9A000000000053
:040F9B000000000052
:040F9C000000000051
:040F9D000000000050
:040F9E00000000004F
:040F9F00000000004E
:040FA000000000004D
:040FA100000000004C
:040FA200000000004B
:040FA300000000004A
:040FA4000000000049
:040FA5000000000048
:040FA6000000000047
:040FA7000000000046
:040FA8000000000045
:040FA9000000000044
:040FAA000000000043
:040FAB000000000042
:040FAC000000000041
:040FAD000000000040
:040FAE00000000003F
:040FAF00000000003E
:040FB000000000003D
:040FB100000000003C
:040FB200000000003B
:040FB300000000003A
:040FB4000000000039
:040FB5000000000038
:040FB6000000000037
:040FB7000000000036
:040FB8000000000035
:040FB9000000000034
:040FBA000000000033
:040FBB000000000032
:040FBC000000000031
:040FBD000000000030
:040FBE00000000002F
:040FBF00000000002E
:040FC000000000002D
:040FC100000000002C
:040FC200000000002B
:040FC300000000002A
:040FC4000000000029
:040FC5000000000028
:040FC6000000000027
:040FC7000000000026
:040FC8000000000025
:040FC9000000000024
:040FCA000000000023
:040FCB000000000022
:040FCC000000000021
:040FCD000000000020
:040FCE00000000001F
:040FCF00000000001E
:040FD000000000001D
:040FD100000000001C
:040FD200000000001B
:040FD300000000001A
:040FD4000000000019
:040FD5000000000018
:040FD6000000000017
:040FD7000000000016
:040FD8000000000015
:040FD9000000000014
:040FDA000000000013
:040FDB000000000012
:040FDC000000000011
:040FDD000000000010
:040FDE00000000000F
:040FDF00000000000E
:040FE000000000000D
:040FE100000000000C
:040FE200000000000B
:040FE300000000000A
:040FE4000000000009
:040FE5000000000008
:040FE6000000000007
:040FE7000000000006
:040FE8000000000005
:040FE9000000000004
:040FEA000000000003
:040FEB000000000002
:040FEC000000000001
:040FED000000000000
:040FEE0000000000FF
:040FEF0000000000FE
:040FF00000000000FD
:040FF10000000000FC
:040FF20000000000FB
:040FF30000000000FA
:040FF40000000000F9
:040FF50000000000F8
:040FF60000000000F7
:040FF70000000000F6
:040FF80000000000F5
:040FF90000000000F4
:040FFA0000000000F3
:040FFB0000000000F2
:040FFC0000000000F1
:040FFD0000000000F0
:040FFE0000000000EF
:040FFF0000000000EE
:0410000000000000EC
:0410010000000000EB
:0410020000000000EA
:0410030000000000E9
:0410040000000000E8
:0410050000000000E7
:0410060000000000E6
:0410070000000000E5
:0410080000000000E4
:0410090000000000E3
:04100A0000000000E2
:04100B0000000000E1
:04100C0000000000E0
:04100D0000000000DF
:04100E0000000000DE
:04100F0000000000DD
:0410100000000000DC
:0410110000000000DB
:0410120000000000DA
:0410130000000000D9
:0410140000000000D8
:0410150000000000D7
:0410160000000000D6
:0410170000000000D5
:0410180000000000D4
:0410190000000000D3
:04101A0000000000D2
:04101B0000000000D1
:04101C0000000000D0
:04101D0000000000CF
:04101E0000000000CE
:04101F0000000000CD
:0410200000000000CC
:0410210000000000CB
:0410220000000000CA
:0410230000000000C9
:0410240000000000C8
:0410250000000000C7
:0410260000000000C6
:0410270000000000C5
:0410280000000000C4
:0410290000000000C3
:04102A0000000000C2
:04102B0000000000C1
:04102C0000000000C0
:04102D0000000000BF
:04102E0000000000BE
:04102F0000000000BD
:0410300000000000BC
:0410310000000000BB
:0410320000000000BA
:0410330000000000B9
:0410340000000000B8
:0410350000000000B7
:0410360000000000B6
:0410370000000000B5
:0410380000000000B4
:0410390000000000B3
:04103A0000000000B2
:04103B0000000000B1
:04103C0000000000B0
:04103D0000000000AF
:04103E0000000000AE
:04103F0000000000AD
:0410400000000000AC
:0410410000000000AB
:0410420000000000AA
:0410430000000000A9
:0410440000000000A8
:0410450000000000A7
:0410460000000000A6
:0410470000000000A5
:0410480000000000A4
:0410490000000000A3
:04104A0000000000A2
:04104B0000000000A1
:04104C0000000000A0
:04104D00000000009F
:04104E00000000009E
:04104F00000000009D
:04105000000000009C
:04105100000000009B
:04105200000000009A
:041053000000000099
:041054000000000098
:041055000000000097
:041056000000000096
:041057000000000095
:041058000000000094
:041059000000000093
:04105A000000000092
:04105B000000000091
:04105C000000000090
:04105D00000000008F
:04105E00000000008E
:04105F00000000008D
:04106000000000008C
:04106100000000008B
:04106200000000008A
:041063000000000089
:041064000000000088
:041065000000000087
:041066000000000086
:041067000000000085
:041068000000000084
:041069000000000083
:04106A000000000082
:04106B000000000081
:04106C000000000080
:04106D00000000007F
:04106E00000000007E
:04106F00000000007D
:04107000000000007C
:04107100000000007B
:04107200000000007A
:041073000000000079
:041074000000000078
:041075000000000077
:041076000000000076
:041077000000000075
:041078000000000074
:041079000000000073
:04107A000000000072
:04107B000000000071
:04107C000000000070
:04107D00000000006F
:04107E00000000006E
:04107F00000000006D
:04108000000000006C
:04108100000000006B
:04108200000000006A
:041083000000000069
:041084000000000068
:041085000000000067
:041086000000000066
:041087000000000065
:041088000000000064
:041089000000000063
:04108A000000000062
:04108B000000000061
:04108C000000000060
:04108D00000000005F
:04108E00000000005E
:04108F00000000005D
:04109000000000005C
:04109100000000005B
:04109200000000005A
:041093000000000059
:041094000000000058
:041095000000000057
:041096000000000056
:041097000000000055
:041098000000000054
:041099000000000053
:04109A000000000052
:04109B000000000051
:04109C000000000050
:04109D00000000004F
:04109E00000000004E
:04109F00000000004D
:0410A000000000004C
:0410A100000000004B
:0410A200000000004A
:0410A3000000000049
:0410A4000000000048
:0410A5000000000047
:0410A6000000000046
:0410A7000000000045
:0410A8000000000044
:0410A9000000000043
:0410AA000000000042
:0410AB000000000041
:0410AC000000000040
:0410AD00000000003F
:0410AE00000000003E
:0410AF00000000003D
:0410B000000000003C
:0410B100000000003B
:0410B200000000003A
:0410B3000000000039
:0410B4000000000038
:0410B5000000000037
:0410B6000000000036
:0410B7000000000035
:0410B8000000000034
:0410B9000000000033
:0410BA000000000032
:0410BB000000000031
:0410BC000000000030
:0410BD00000000002F
:0410BE00000000002E
:0410BF00000000002D
:0410C000000000002C
:0410C100000000002B
:0410C200000000002A
:0410C3000000000029
:0410C4000000000028
:0410C5000000000027
:0410C6000000000026
:0410C7000000000025
:0410C8000000000024
:0410C9000000000023
:0410CA000000000022
:0410CB000000000021
:0410CC000000000020
:0410CD00000000001F
:0410CE00000000001E
:0410CF00000000001D
:0410D000000000001C
:0410D100000000001B
:0410D200000000001A
:0410D3000000000019
:0410D4000000000018
:0410D5000000000017
:0410D6000000000016
:0410D7000000000015
:0410D8000000000014
:0410D9000000000013
:0410DA000000000012
:0410DB000000000011
:0410DC000000000010
:0410DD00000000000F
:0410DE00000000000E
:0410DF00000000000D
:0410E000000000000C
:0410E100000000000B
:0410E200000000000A
:0410E3000000000009
:0410E4000000000008
:0410E5000000000007
:0410E6000000000006
:0410E7000000000005
:0410E8000000000004
:0410E9000000000003
:0410EA000000000002
:0410EB000000000001
:0410EC000000000000
:0410ED0000000000FF
:0410EE0000000000FE
:0410EF0000000000FD
:0410F00000000000FC
:0410F10000000000FB
:0410F20000000000FA
:0410F30000000000F9
:0410F40000000000F8
:0410F50000000000F7
:0410F60000000000F6
:0410F70000000000F5
:0410F80000000000F4
:0410F90000000000F3
:0410FA0000000000F2
:0410FB0000000000F1
:0410FC0000000000F0
:0410FD0000000000EF
:0410FE0000000000EE
:0410FF0000000000ED
:0411000000000000EB
:0411010000000000EA
:0411020000000000E9
:0411030000000000E8
:0411040000000000E7
:0411050000000000E6
:0411060000000000E5
:0411070000000000E4
:0411080000000000E3
:0411090000000000E2
:04110A0000000000E1
:04110B0000000000E0
:04110C0000000000DF
:04110D0000000000DE
:04110E0000000000DD
:04110F0000000000DC
:0411100000000000DB
:0411110000000000DA
:0411120000000000D9
:0411130000000000D8
:0411140000000000D7
:0411150000000000D6
:0411160000000000D5
:0411170000000000D4
:0411180000000000D3
:0411190000000000D2
:04111A0000000000D1
:04111B0000000000D0
:04111C0000000000CF
:04111D0000000000CE
:04111E0000000000CD
:04111F0000000000CC
:0411200000000000CB
:0411210000000000CA
:0411220000000000C9
:0411230000000000C8
:0411240000000000C7
:0411250000000000C6
:0411260000000000C5
:0411270000000000C4
:0411280000000000C3
:0411290000000000C2
:04112A0000000000C1
:04112B0000000000C0
:04112C0000000000BF
:04112D0000000000BE
:04112E0000000000BD
:04112F0000000000BC
:0411300000000000BB
:0411310000000000BA
:0411320000000000B9
:0411330000000000B8
:0411340000000000B7
:0411350000000000B6
:0411360000000000B5
:0411370000000000B4
:0411380000000000B3
:0411390000000000B2
:04113A0000000000B1
:04113B0000000000B0
:04113C0000000000AF
:04113D0000000000AE
:04113E0000000000AD
:04113F0000000000AC
:0411400000000000AB
:0411410000000000AA
:0411420000000000A9
:0411430000000000A8
:0411440000000000A7
:0411450000000000A6
:0411460000000000A5
:0411470000000000A4
:0411480000000000A3
:0411490000000000A2
:04114A0000000000A1
:04114B0000000000A0
:04114C00000000009F
:04114D00000000009E
:04114E00000000009D
:04114F00000000009C
:04115000000000009B
:04115100000000009A
:041152000000000099
:041153000000000098
:041154000000000097
:041155000000000096
:041156000000000095
:041157000000000094
:041158000000000093
:041159000000000092
:04115A000000000091
:04115B000000000090
:04115C00000000008F
:04115D00000000008E
:04115E00000000008D
:04115F00000000008C
:04116000000000008B
:04116100000000008A
:041162000000000089
:041163000000000088
:041164000000000087
:041165000000000086
:041166000000000085
:041167000000000084
:041168000000000083
:041169000000000082
:04116A000000000081
:04116B000000000080
:04116C00000000007F
:04116D00000000007E
:04116E00000000007D
:04116F00000000007C
:04117000000000007B
:04117100000000007A
:041172000000000079
:041173000000000078
:041174000000000077
:041175000000000076
:041176000000000075
:041177000000000074
:041178000000000073
:041179000000000072
:04117A000000000071
:04117B000000000070
:04117C00000000006F
:04117D00000000006E
:04117E00000000006D
:04117F00000000006C
:04118000000000006B
:04118100000000006A
:041182000000000069
:041183000000000068
:041184000000000067
:041185000000000066
:041186000000000065
:041187000000000064
:041188000000000063
:041189000000000062
:04118A000000000061
:04118B000000000060
:04118C00000000005F
:04118D00000000005E
:04118E00000000005D
:04118F00000000005C
:04119000000000005B
:04119100000000005A
:041192000000000059
:041193000000000058
:041194000000000057
:041195000000000056
:041196000000000055
:041197000000000054
:041198000000000053
:041199000000000052
:04119A000000000051
:04119B000000000050
:04119C00000000004F
:04119D00000000004E
:04119E00000000004D
:04119F00000000004C
:0411A000000000004B
:0411A100000000004A
:0411A2000000000049
:0411A3000000000048
:0411A4000000000047
:0411A5000000000046
:0411A6000000000045
:0411A7000000000044
:0411A8000000000043
:0411A9000000000042
:0411AA000000000041
:0411AB000000000040
:0411AC00000000003F
:0411AD00000000003E
:0411AE00000000003D
:0411AF00000000003C
:0411B000000000003B
:0411B100000000003A
:0411B2000000000039
:0411B3000000000038
:0411B4000000000037
:0411B5000000000036
:0411B6000000000035
:0411B7000000000034
:0411B8000000000033
:0411B9000000000032
:0411BA000000000031
:0411BB000000000030
:0411BC00000000002F
:0411BD00000000002E
:0411BE00000000002D
:0411BF00000000002C
:0411C000000000002B
:0411C100000000002A
:0411C2000000000029
:0411C3000000000028
:0411C4000000000027
:0411C5000000000026
:0411C6000000000025
:0411C7000000000024
:0411C8000000000023
:0411C9000000000022
:0411CA000000000021
:0411CB000000000020
:0411CC00000000001F
:0411CD00000000001E
:0411CE00000000001D
:0411CF00000000001C
:0411D000000000001B
:0411D100000000001A
:0411D2000000000019
:0411D3000000000018
:0411D4000000000017
:0411D5000000000016
:0411D6000000000015
:0411D7000000000014
:0411D8000000000013
:0411D9000000000012
:0411DA000000000011
:0411DB000000000010
:0411DC00000000000F
:0411DD00000000000E
:0411DE00000000000D
:0411DF00000000000C
:0411E000000000000B
:0411E100000000000A
:0411E2000000000009
:0411E3000000000008
:0411E4000000000007
:0411E5000000000006
:0411E6000000000005
:0411E7000000000004
:0411E8000000000003
:0411E9000000000002
:0411EA000000000001
:0411EB000000000000
:0411EC0000000000FF
:0411ED0000000000FE
:0411EE0000000000FD
:0411EF0000000000FC
:0411F00000000000FB
:0411F10000000000FA
:0411F20000000000F9
:0411F30000000000F8
:0411F40000000000F7
:0411F50000000000F6
:0411F60000000000F5
:0411F70000000000F4
:0411F80000000000F3
:0411F90000000000F2
:0411FA0000000000F1
:0411FB0000000000F0
:0411FC0000000000EF
:0411FD0000000000EE
:0411FE0000000000ED
:0411FF0000000000EC
:0412000000000000EA
:0412010000000000E9
:0412020000000000E8
:0412030000000000E7
:0412040000000000E6
:0412050000000000E5
:0412060000000000E4
:0412070000000000E3
:0412080000000000E2
:0412090000000000E1
:04120A0000000000E0
:04120B0000000000DF
:04120C0000000000DE
:04120D0000000000DD
:04120E0000000000DC
:04120F0000000000DB
:0412100000000000DA
:0412110000000000D9
:0412120000000000D8
:0412130000000000D7
:0412140000000000D6
:0412150000000000D5
:0412160000000000D4
:0412170000000000D3
:0412180000000000D2
:0412190000000000D1
:04121A0000000000D0
:04121B0000000000CF
:04121C0000000000CE
:04121D0000000000CD
:04121E0000000000CC
:04121F0000000000CB
:0412200000000000CA
:0412210000000000C9
:0412220000000000C8
:0412230000000000C7
:0412240000000000C6
:0412250000000000C5
:0412260000000000C4
:0412270000000000C3
:0412280000000000C2
:0412290000000000C1
:04122A0000000000C0
:04122B0000000000BF
:04122C0000000000BE
:04122D0000000000BD
:04122E0000000000BC
:04122F0000000000BB
:0412300000000000BA
:0412310000000000B9
:0412320000000000B8
:0412330000000000B7
:0412340000000000B6
:0412350000000000B5
:0412360000000000B4
:0412370000000000B3
:0412380000000000B2
:0412390000000000B1
:04123A0000000000B0
:04123B0000000000AF
:04123C0000000000AE
:04123D0000000000AD
:04123E0000000000AC
:04123F0000000000AB
:0412400000000000AA
:0412410000000000A9
:0412420000000000A8
:0412430000000000A7
:0412440000000000A6
:0412450000000000A5
:0412460000000000A4
:0412470000000000A3
:0412480000000000A2
:0412490000000000A1
:04124A0000000000A0
:04124B00000000009F
:04124C00000000009E
:04124D00000000009D
:04124E00000000009C
:04124F00000000009B
:04125000000000009A
:041251000000000099
:041252000000000098
:041253000000000097
:041254000000000096
:041255000000000095
:041256000000000094
:041257000000000093
:041258000000000092
:041259000000000091
:04125A000000000090
:04125B00000000008F
:04125C00000000008E
:04125D00000000008D
:04125E00000000008C
:04125F00000000008B
:04126000000000008A
:041261000000000089
:041262000000000088
:041263000000000087
:041264000000000086
:041265000000000085
:041266000000000084
:041267000000000083
:041268000000000082
:041269000000000081
:04126A000000000080
:04126B00000000007F
:04126C00000000007E
:04126D00000000007D
:04126E00000000007C
:04126F00000000007B
:04127000000000007A
:041271000000000079
:041272000000000078
:041273000000000077
:041274000000000076
:041275000000000075
:041276000000000074
:041277000000000073
:041278000000000072
:041279000000000071
:04127A000000000070
:04127B00000000006F
:04127C00000000006E
:04127D00000000006D
:04127E00000000006C
:04127F00000000006B
:04128000000000006A
:041281000000000069
:041282000000000068
:041283000000000067
:041284000000000066
:041285000000000065
:041286000000000064
:041287000000000063
:041288000000000062
:041289000000000061
:04128A000000000060
:04128B00000000005F
:04128C00000000005E
:04128D00000000005D
:04128E00000000005C
:04128F00000000005B
:04129000000000005A
:041291000000000059
:041292000000000058
:041293000000000057
:041294000000000056
:041295000000000055
:041296000000000054
:041297000000000053
:041298000000000052
:041299000000000051
:04129A000000000050
:04129B00000000004F
:04129C00000000004E
:04129D00000000004D
:04129E00000000004C
:04129F00000000004B
:0412A000000000004A
:0412A1000000000049
:0412A2000000000048
:0412A3000000000047
:0412A4000000000046
:0412A5000000000045
:0412A6000000000044
:0412A7000000000043
:0412A8000000000042
:0412A9000000000041
:0412AA000000000040
:0412AB00000000003F
:0412AC00000000003E
:0412AD00000000003D
:0412AE00000000003C
:0412AF00000000003B
:0412B000000000003A
:0412B1000000000039
:0412B2000000000038
:0412B3000000000037
:0412B4000000000036
:0412B5000000000035
:0412B6000000000034
:0412B7000000000033
:0412B8000000000032
:0412B9000000000031
:0412BA000000000030
:0412BB00000000002F
:0412BC00000000002E
:0412BD00000000002D
:0412BE00000000002C
:0412BF00000000002B
:0412C000000000002A
:0412C1000000000029
:0412C2000000000028
:0412C3000000000027
:0412C4000000000026
:0412C5000000000025
:0412C6000000000024
:0412C7000000000023
:0412C8000000000022
:0412C9000000000021
:0412CA000000000020
:0412CB00000000001F
:0412CC00000000001E
:0412CD00000000001D
:0412CE00000000001C
:0412CF00000000001B
:0412D000000000001A
:0412D1000000000019
:0412D2000000000018
:0412D3000000000017
:0412D4000000000016
:0412D5000000000015
:0412D6000000000014
:0412D7000000000013
:0412D8000000000012
:0412D9000000000011
:0412DA000000000010
:0412DB00000000000F
:0412DC00000000000E
:0412DD00000000000D
:0412DE00000000000C
:0412DF00000000000B
:0412E000000000000A
:0412E1000000000009
:0412E2000000000008
:0412E3000000000007
:0412E4000000000006
:0412E5000000000005
:0412E6000000000004
:0412E7000000000003
:0412E8000000000002
:0412E9000000000001
:0412EA000000000000
:0412EB0000000000FF
:0412EC0000000000FE
:0412ED0000000000FD
:0412EE0000000000FC
:0412EF0000000000FB
:0412F00000000000FA
:0412F10000000000F9
:0412F20000000000F8
:0412F30000000000F7
:0412F40000000000F6
:0412F50000000000F5
:0412F60000000000F4
:0412F70000000000F3
:0412F80000000000F2
:0412F90000000000F1
:0412FA0000000000F0
:0412FB0000000000EF
:0412FC0000000000EE
:0412FD0000000000ED
:0412FE0000000000EC
:0412FF0000000000EB
:0413000000000000E9
:0413010000000000E8
:0413020000000000E7
:0413030000000000E6
:0413040000000000E5
:0413050000000000E4
:0413060000000000E3
:0413070000000000E2
:0413080000000000E1
:0413090000000000E0
:04130A0000000000DF
:04130B0000000000DE
:04130C0000000000DD
:04130D0000000000DC
:04130E0000000000DB
:04130F0000000000DA
:0413100000000000D9
:0413110000000000D8
:0413120000000000D7
:0413130000000000D6
:0413140000000000D5
:0413150000000000D4
:0413160000000000D3
:0413170000000000D2
:0413180000000000D1
:0413190000000000D0
:04131A0000000000CF
:04131B0000000000CE
:04131C0000000000CD
:04131D0000000000CC
:04131E0000000000CB
:04131F0000000000CA
:0413200000000000C9
:0413210000000000C8
:0413220000000000C7
:0413230000000000C6
:0413240000000000C5
:0413250000000000C4
:0413260000000000C3
:0413270000000000C2
:0413280000000000C1
:0413290000000000C0
:04132A0000000000BF
:04132B0000000000BE
:04132C0000000000BD
:04132D0000000000BC
:04132E0000000000BB
:04132F0000000000BA
:0413300000000000B9
:0413310000000000B8
:0413320000000000B7
:0413330000000000B6
:0413340000000000B5
:0413350000000000B4
:0413360000000000B3
:0413370000000000B2
:0413380000000000B1
:0413390000000000B0
:04133A0000000000AF
:04133B0000000000AE
:04133C0000000000AD
:04133D0000000000AC
:04133E0000000000AB
:04133F0000000000AA
:0413400000000000A9
:0413410000000000A8
:0413420000000000A7
:0413430000000000A6
:0413440000000000A5
:0413450000000000A4
:0413460000000000A3
:0413470000000000A2
:0413480000000000A1
:0413490000000000A0
:04134A00000000009F
:04134B00000000009E
:04134C00000000009D
:04134D00000000009C
:04134E00000000009B
:04134F00000000009A
:041350000000000099
:041351000000000098
:041352000000000097
:041353000000000096
:041354000000000095
:041355000000000094
:041356000000000093
:041357000000000092
:041358000000000091
:041359000000000090
:04135A00000000008F
:04135B00000000008E
:04135C00000000008D
:04135D00000000008C
:04135E00000000008B
:04135F00000000008A
:041360000000000089
:041361000000000088
:041362000000000087
:041363000000000086
:041364000000000085
:041365000000000084
:041366000000000083
:041367000000000082
:041368000000000081
:041369000000000080
:04136A00000000007F
:04136B00000000007E
:04136C00000000007D
:04136D00000000007C
:04136E00000000007B
:04136F00000000007A
:041370000000000079
:041371000000000078
:041372000000000077
:041373000000000076
:041374000000000075
:041375000000000074
:041376000000000073
:041377000000000072
:041378000000000071
:041379000000000070
:04137A00000000006F
:04137B00000000006E
:04137C00000000006D
:04137D00000000006C
:04137E00000000006B
:04137F00000000006A
:041380000000000069
:041381000000000068
:041382000000000067
:041383000000000066
:041384000000000065
:041385000000000064
:041386000000000063
:041387000000000062
:041388000000000061
:041389000000000060
:04138A00000000005F
:04138B00000000005E
:04138C00000000005D
:04138D00000000005C
:04138E00000000005B
:04138F00000000005A
:041390000000000059
:041391000000000058
:041392000000000057
:041393000000000056
:041394000000000055
:041395000000000054
:041396000000000053
:041397000000000052
:041398000000000051
:041399000000000050
:04139A00000000004F
:04139B00000000004E
:04139C00000000004D
:04139D00000000004C
:04139E00000000004B
:04139F00000000004A
:0413A0000000000049
:0413A1000000000048
:0413A2000000000047
:0413A3000000000046
:0413A4000000000045
:0413A5000000000044
:0413A6000000000043
:0413A7000000000042
:0413A8000000000041
:0413A9000000000040
:0413AA00000000003F
:0413AB00000000003E
:0413AC00000000003D
:0413AD00000000003C
:0413AE00000000003B
:0413AF00000000003A
:0413B0000000000039
:0413B1000000000038
:0413B2000000000037
:0413B3000000000036
:0413B4000000000035
:0413B5000000000034
:0413B6000000000033
:0413B7000000000032
:0413B8000000000031
:0413B9000000000030
:0413BA00000000002F
:0413BB00000000002E
:0413BC00000000002D
:0413BD00000000002C
:0413BE00000000002B
:0413BF00000000002A
:0413C0000000000029
:0413C1000000000028
:0413C2000000000027
:0413C3000000000026
:0413C4000000000025
:0413C5000000000024
:0413C6000000000023
:0413C7000000000022
:0413C8000000000021
:0413C9000000000020
:0413CA00000000001F
:0413CB00000000001E
:0413CC00000000001D
:0413CD00000000001C
:0413CE00000000001B
:0413CF00000000001A
:0413D0000000000019
:0413D1000000000018
:0413D2000000000017
:0413D3000000000016
:0413D4000000000015
:0413D5000000000014
:0413D6000000000013
:0413D7000000000012
:0413D8000000000011
:0413D9000000000010
:0413DA00000000000F
:0413DB00000000000E
:0413DC00000000000D
:0413DD00000000000C
:0413DE00000000000B
:0413DF00000000000A
:0413E0000000000009
:0413E1000000000008
:0413E2000000000007
:0413E3000000000006
:0413E4000000000005
:0413E5000000000004
:0413E6000000000003
:0413E7000000000002
:0413E8000000000001
:0413E9000000000000
:0413EA0000000000FF
:0413EB0000000000FE
:0413EC0000000000FD
:0413ED0000000000FC
:0413EE0000000000FB
:0413EF0000000000FA
:0413F00000000000F9
:0413F10000000000F8
:0413F20000000000F7
:0413F30000000000F6
:0413F40000000000F5
:0413F50000000000F4
:0413F60000000000F3
:0413F70000000000F2
:0413F80000000000F1
:0413F90000000000F0
:0413FA0000000000EF
:0413FB0000000000EE
:0413FC0000000000ED
:0413FD0000000000EC
:0413FE0000000000EB
:0413FF0000000000EA
:0414000000000000E8
:0414010000000000E7
:0414020000000000E6
:0414030000000000E5
:0414040000000000E4
:0414050000000000E3
:0414060000000000E2
:0414070000000000E1
:0414080000000000E0
:0414090000000000DF
:04140A0000000000DE
:04140B0000000000DD
:04140C0000000000DC
:04140D0000000000DB
:04140E0000000000DA
:04140F0000000000D9
:0414100000000000D8
:0414110000000000D7
:0414120000000000D6
:0414130000000000D5
:0414140000000000D4
:0414150000000000D3
:0414160000000000D2
:0414170000000000D1
:0414180000000000D0
:0414190000000000CF
:04141A0000000000CE
:04141B0000000000CD
:04141C0000000000CC
:04141D0000000000CB
:04141E0000000000CA
:04141F0000000000C9
:0414200000000000C8
:0414210000000000C7
:0414220000000000C6
:0414230000000000C5
:0414240000000000C4
:0414250000000000C3
:0414260000000000C2
:0414270000000000C1
:0414280000000000C0
:0414290000000000BF
:04142A0000000000BE
:04142B0000000000BD
:04142C0000000000BC
:04142D0000000000BB
:04142E0000000000BA
:04142F0000000000B9
:0414300000000000B8
:0414310000000000B7
:0414320000000000B6
:0414330000000000B5
:0414340000000000B4
:0414350000000000B3
:0414360000000000B2
:0414370000000000B1
:0414380000000000B0
:0414390000000000AF
:04143A0000000000AE
:04143B0000000000AD
:04143C0000000000AC
:04143D0000000000AB
:04143E0000000000AA
:04143F0000000000A9
:0414400000000000A8
:0414410000000000A7
:0414420000000000A6
:0414430000000000A5
:0414440000000000A4
:0414450000000000A3
:0414460000000000A2
:0414470000000000A1
:0414480000000000A0
:04144900000000009F
:04144A00000000009E
:04144B00000000009D
:04144C00000000009C
:04144D00000000009B
:04144E00000000009A
:04144F000000000099
:041450000000000098
:041451000000000097
:041452000000000096
:041453000000000095
:041454000000000094
:041455000000000093
:041456000000000092
:041457000000000091
:041458000000000090
:04145900000000008F
:04145A00000000008E
:04145B00000000008D
:04145C00000000008C
:04145D00000000008B
:04145E00000000008A
:04145F000000000089
:041460000000000088
:041461000000000087
:041462000000000086
:041463000000000085
:041464000000000084
:041465000000000083
:041466000000000082
:041467000000000081
:041468000000000080
:04146900000000007F
:04146A00000000007E
:04146B00000000007D
:04146C00000000007C
:04146D00000000007B
:04146E00000000007A
:04146F000000000079
:041470000000000078
:041471000000000077
:041472000000000076
:041473000000000075
:041474000000000074
:041475000000000073
:041476000000000072
:041477000000000071
:041478000000000070
:04147900000000006F
:04147A00000000006E
:04147B00000000006D
:04147C00000000006C
:04147D00000000006B
:04147E00000000006A
:04147F000000000069
:041480000000000068
:041481000000000067
:041482000000000066
:041483000000000065
:041484000000000064
:041485000000000063
:041486000000000062
:041487000000000061
:041488000000000060
:04148900000000005F
:04148A00000000005E
:04148B00000000005D
:04148C00000000005C
:04148D00000000005B
:04148E00000000005A
:04148F000000000059
:041490000000000058
:041491000000000057
:041492000000000056
:041493000000000055
:041494000000000054
:041495000000000053
:041496000000000052
:041497000000000051
:041498000000000050
:04149900000000004F
:04149A00000000004E
:04149B00000000004D
:04149C00000000004C
:04149D00000000004B
:04149E00000000004A
:04149F000000000049
:0414A0000000000048
:0414A1000000000047
:0414A2000000000046
:0414A3000000000045
:0414A4000000000044
:0414A5000000000043
:0414A6000000000042
:0414A7000000000041
:0414A8000000000040
:0414A900000000003F
:0414AA00000000003E
:0414AB00000000003D
:0414AC00000000003C
:0414AD00000000003B
:0414AE00000000003A
:0414AF000000000039
:0414B0000000000038
:0414B1000000000037
:0414B2000000000036
:0414B3000000000035
:0414B4000000000034
:0414B5000000000033
:0414B6000000000032
:0414B7000000000031
:0414B8000000000030
:0414B900000000002F
:0414BA00000000002E
:0414BB00000000002D
:0414BC00000000002C
:0414BD00000000002B
:0414BE00000000002A
:0414BF000000000029
:0414C0000000000028
:0414C1000000000027
:0414C2000000000026
:0414C3000000000025
:0414C4000000000024
:0414C5000000000023
:0414C6000000000022
:0414C7000000000021
:0414C8000000000020
:0414C900000000001F
:0414CA00000000001E
:0414CB00000000001D
:0414CC00000000001C
:0414CD00000000001B
:0414CE00000000001A
:0414CF000000000019
:0414D0000000000018
:0414D1000000000017
:0414D2000000000016
:0414D3000000000015
:0414D4000000000014
:0414D5000000000013
:0414D6000000000012
:0414D7000000000011
:0414D8000000000010
:0414D900000000000F
:0414DA00000000000E
:0414DB00000000000D
:0414DC00000000000C
:0414DD00000000000B
:0414DE00000000000A
:0414DF000000000009
:0414E0000000000008
:0414E1000000000007
:0414E2000000000006
:0414E3000000000005
:0414E4000000000004
:0414E5000000000003
:0414E6000000000002
:0414E7000000000001
:0414E8000000000000
:0414E90000000000FF
:0414EA0000000000FE
:0414EB0000000000FD
:0414EC0000000000FC
:0414ED0000000000FB
:0414EE0000000000FA
:0414EF0000000000F9
:0414F00000000000F8
:0414F10000000000F7
:0414F20000000000F6
:0414F30000000000F5
:0414F40000000000F4
:0414F50000000000F3
:0414F60000000000F2
:0414F70000000000F1
:0414F80000000000F0
:0414F90000000000EF
:0414FA0000000000EE
:0414FB0000000000ED
:0414FC0000000000EC
:0414FD0000000000EB
:0414FE0000000000EA
:0414FF0000000000E9
:0415000000000000E7
:0415010000000000E6
:0415020000000000E5
:0415030000000000E4
:0415040000000000E3
:0415050000000000E2
:0415060000000000E1
:0415070000000000E0
:0415080000000000DF
:0415090000000000DE
:04150A0000000000DD
:04150B0000000000DC
:04150C0000000000DB
:04150D0000000000DA
:04150E0000000000D9
:04150F0000000000D8
:0415100000000000D7
:0415110000000000D6
:0415120000000000D5
:0415130000000000D4
:0415140000000000D3
:0415150000000000D2
:0415160000000000D1
:0415170000000000D0
:0415180000000000CF
:0415190000000000CE
:04151A0000000000CD
:04151B0000000000CC
:04151C0000000000CB
:04151D0000000000CA
:04151E0000000000C9
:04151F0000000000C8
:0415200000000000C7
:0415210000000000C6
:0415220000000000C5
:0415230000000000C4
:0415240000000000C3
:0415250000000000C2
:0415260000000000C1
:0415270000000000C0
:0415280000000000BF
:0415290000000000BE
:04152A0000000000BD
:04152B0000000000BC
:04152C0000000000BB
:04152D0000000000BA
:04152E0000000000B9
:04152F0000000000B8
:0415300000000000B7
:0415310000000000B6
:0415320000000000B5
:0415330000000000B4
:0415340000000000B3
:0415350000000000B2
:0415360000000000B1
:0415370000000000B0
:0415380000000000AF
:0415390000000000AE
:04153A0000000000AD
:04153B0000000000AC
:04153C0000000000AB
:04153D0000000000AA
:04153E0000000000A9
:04153F0000000000A8
:0415400000000000A7
:0415410000000000A6
:0415420000000000A5
:0415430000000000A4
:0415440000000000A3
:0415450000000000A2
:0415460000000000A1
:0415470000000000A0
:04154800000000009F
:04154900000000009E
:04154A00000000009D
:04154B00000000009C
:04154C00000000009B
:04154D00000000009A
:04154E000000000099
:04154F000000000098
:041550000000000097
:041551000000000096
:041552000000000095
:041553000000000094
:041554000000000093
:041555000000000092
:041556000000000091
:041557000000000090
:04155800000000008F
:04155900000000008E
:04155A00000000008D
:04155B00000000008C
:04155C00000000008B
:04155D00000000008A
:04155E000000000089
:04155F000000000088
:041560000000000087
:041561000000000086
:041562000000000085
:041563000000000084
:041564000000000083
:041565000000000082
:041566000000000081
:041567000000000080
:04156800000000007F
:04156900000000007E
:04156A00000000007D
:04156B00000000007C
:04156C00000000007B
:04156D00000000007A
:04156E000000000079
:04156F000000000078
:041570000000000077
:041571000000000076
:041572000000000075
:041573000000000074
:041574000000000073
:041575000000000072
:041576000000000071
:041577000000000070
:04157800000000006F
:04157900000000006E
:04157A00000000006D
:04157B00000000006C
:04157C00000000006B
:04157D00000000006A
:04157E000000000069
:04157F000000000068
:041580000000000067
:041581000000000066
:041582000000000065
:041583000000000064
:041584000000000063
:041585000000000062
:041586000000000061
:041587000000000060
:04158800000000005F
:04158900000000005E
:04158A00000000005D
:04158B00000000005C
:04158C00000000005B
:04158D00000000005A
:04158E000000000059
:04158F000000000058
:041590000000000057
:041591000000000056
:041592000000000055
:041593000000000054
:041594000000000053
:041595000000000052
:041596000000000051
:041597000000000050
:04159800000000004F
:04159900000000004E
:04159A00000000004D
:04159B00000000004C
:04159C00000000004B
:04159D00000000004A
:04159E000000000049
:04159F000000000048
:0415A0000000000047
:0415A1000000000046
:0415A2000000000045
:0415A3000000000044
:0415A4000000000043
:0415A5000000000042
:0415A6000000000041
:0415A7000000000040
:0415A800000000003F
:0415A900000000003E
:0415AA00000000003D
:0415AB00000000003C
:0415AC00000000003B
:0415AD00000000003A
:0415AE000000000039
:0415AF000000000038
:0415B0000000000037
:0415B1000000000036
:0415B2000000000035
:0415B3000000000034
:0415B4000000000033
:0415B5000000000032
:0415B6000000000031
:0415B7000000000030
:0415B800000000002F
:0415B900000000002E
:0415BA00000000002D
:0415BB00000000002C
:0415BC00000000002B
:0415BD00000000002A
:0415BE000000000029
:0415BF000000000028
:0415C0000000000027
:0415C1000000000026
:0415C2000000000025
:0415C3000000000024
:0415C4000000000023
:0415C5000000000022
:0415C6000000000021
:0415C7000000000020
:0415C800000000001F
:0415C900000000001E
:0415CA00000000001D
:0415CB00000000001C
:0415CC00000000001B
:0415CD00000000001A
:0415CE000000000019
:0415CF000000000018
:0415D0000000000017
:0415D1000000000016
:0415D2000000000015
:0415D3000000000014
:0415D4000000000013
:0415D5000000000012
:0415D6000000000011
:0415D7000000000010
:0415D800000000000F
:0415D900000000000E
:0415DA00000000000D
:0415DB00000000000C
:0415DC00000000000B
:0415DD00000000000A
:0415DE000000000009
:0415DF000000000008
:0415E0000000000007
:0415E1000000000006
:0415E2000000000005
:0415E3000000000004
:0415E4000000000003
:0415E5000000000002
:0415E6000000000001
:0415E7000000000000
:0415E80000000000FF
:0415E90000000000FE
:0415EA0000000000FD
:0415EB0000000000FC
:0415EC0000000000FB
:0415ED0000000000FA
:0415EE0000000000F9
:0415EF0000000000F8
:0415F00000000000F7
:0415F10000000000F6
:0415F20000000000F5
:0415F30000000000F4
:0415F40000000000F3
:0415F50000000000F2
:0415F60000000000F1
:0415F70000000000F0
:0415F80000000000EF
:0415F90000000000EE
:0415FA0000000000ED
:0415FB0000000000EC
:0415FC0000000000EB
:0415FD0000000000EA
:0415FE0000000000E9
:0415FF0000000000E8
:0416000000000000E6
:0416010000000000E5
:0416020000000000E4
:0416030000000000E3
:0416040000000000E2
:0416050000000000E1
:0416060000000000E0
:0416070000000000DF
:0416080000000000DE
:0416090000000000DD
:04160A0000000000DC
:04160B0000000000DB
:04160C0000000000DA
:04160D0000000000D9
:04160E0000000000D8
:04160F0000000000D7
:0416100000000000D6
:0416110000000000D5
:0416120000000000D4
:0416130000000000D3
:0416140000000000D2
:0416150000000000D1
:0416160000000000D0
:0416170000000000CF
:0416180000000000CE
:0416190000000000CD
:04161A0000000000CC
:04161B0000000000CB
:04161C0000000000CA
:04161D0000000000C9
:04161E0000000000C8
:04161F0000000000C7
:0416200000000000C6
:0416210000000000C5
:0416220000000000C4
:0416230000000000C3
:0416240000000000C2
:0416250000000000C1
:0416260000000000C0
:0416270000000000BF
:0416280000000000BE
:0416290000000000BD
:04162A0000000000BC
:04162B0000000000BB
:04162C0000000000BA
:04162D0000000000B9
:04162E0000000000B8
:04162F0000000000B7
:0416300000000000B6
:0416310000000000B5
:0416320000000000B4
:0416330000000000B3
:0416340000000000B2
:0416350000000000B1
:0416360000000000B0
:0416370000000000AF
:0416380000000000AE
:0416390000000000AD
:04163A0000000000AC
:04163B0000000000AB
:04163C0000000000AA
:04163D0000000000A9
:04163E0000000000A8
:04163F0000000000A7
:0416400000000000A6
:0416410000000000A5
:0416420000000000A4
:0416430000000000A3
:0416440000000000A2
:0416450000000000A1
:0416460000000000A0
:04164700000000009F
:04164800000000009E
:04164900000000009D
:04164A00000000009C
:04164B00000000009B
:04164C00000000009A
:04164D000000000099
:04164E000000000098
:04164F000000000097
:041650000000000096
:041651000000000095
:041652000000000094
:041653000000000093
:041654000000000092
:041655000000000091
:041656000000000090
:04165700000000008F
:04165800000000008E
:04165900000000008D
:04165A00000000008C
:04165B00000000008B
:04165C00000000008A
:04165D000000000089
:04165E000000000088
:04165F000000000087
:041660000000000086
:041661000000000085
:041662000000000084
:041663000000000083
:041664000000000082
:041665000000000081
:041666000000000080
:04166700000000007F
:04166800000000007E
:04166900000000007D
:04166A00000000007C
:04166B00000000007B
:04166C00000000007A
:04166D000000000079
:04166E000000000078
:04166F000000000077
:041670000000000076
:041671000000000075
:041672000000000074
:041673000000000073
:041674000000000072
:041675000000000071
:041676000000000070
:04167700000000006F
:04167800000000006E
:04167900000000006D
:04167A00000000006C
:04167B00000000006B
:04167C00000000006A
:04167D000000000069
:04167E000000000068
:04167F000000000067
:041680000000000066
:041681000000000065
:041682000000000064
:041683000000000063
:041684000000000062
:041685000000000061
:041686000000000060
:04168700000000005F
:04168800000000005E
:04168900000000005D
:04168A00000000005C
:04168B00000000005B
:04168C00000000005A
:04168D000000000059
:04168E000000000058
:04168F000000000057
:041690000000000056
:041691000000000055
:041692000000000054
:041693000000000053
:041694000000000052
:041695000000000051
:041696000000000050
:04169700000000004F
:04169800000000004E
:04169900000000004D
:04169A00000000004C
:04169B00000000004B
:04169C00000000004A
:04169D000000000049
:04169E000000000048
:04169F000000000047
:0416A0000000000046
:0416A1000000000045
:0416A2000000000044
:0416A3000000000043
:0416A4000000000042
:0416A5000000000041
:0416A6000000000040
:0416A700000000003F
:0416A800000000003E
:0416A900000000003D
:0416AA00000000003C
:0416AB00000000003B
:0416AC00000000003A
:0416AD000000000039
:0416AE000000000038
:0416AF000000000037
:0416B0000000000036
:0416B1000000000035
:0416B2000000000034
:0416B3000000000033
:0416B4000000000032
:0416B5000000000031
:0416B6000000000030
:0416B700000000002F
:0416B800000000002E
:0416B900000000002D
:0416BA00000000002C
:0416BB00000000002B
:0416BC00000000002A
:0416BD000000000029
:0416BE000000000028
:0416BF000000000027
:0416C0000000000026
:0416C1000000000025
:0416C2000000000024
:0416C3000000000023
:0416C4000000000022
:0416C5000000000021
:0416C6000000000020
:0416C700000000001F
:0416C800000000001E
:0416C900000000001D
:0416CA00000000001C
:0416CB00000000001B
:0416CC00000000001A
:0416CD000000000019
:0416CE000000000018
:0416CF000000000017
:0416D0000000000016
:0416D1000000000015
:0416D2000000000014
:0416D3000000000013
:0416D4000000000012
:0416D5000000000011
:0416D6000000000010
:0416D700000000000F
:0416D800000000000E
:0416D900000000000D
:0416DA00000000000C
:0416DB00000000000B
:0416DC00000000000A
:0416DD000000000009
:0416DE000000000008
:0416DF000000000007
:0416E0000000000006
:0416E1000000000005
:0416E2000000000004
:0416E3000000000003
:0416E4000000000002
:0416E5000000000001
:0416E6000000000000
:0416E70000000000FF
:0416E80000000000FE
:0416E90000000000FD
:0416EA0000000000FC
:0416EB0000000000FB
:0416EC0000000000FA
:0416ED0000000000F9
:0416EE0000000000F8
:0416EF0000000000F7
:0416F00000000000F6
:0416F10000000000F5
:0416F20000000000F4
:0416F30000000000F3
:0416F40000000000F2
:0416F50000000000F1
:0416F60000000000F0
:0416F70000000000EF
:0416F80000000000EE
:0416F90000000000ED
:0416FA0000000000EC
:0416FB0000000000EB
:0416FC0000000000EA
:0416FD0000000000E9
:0416FE0000000000E8
:0416FF0000000000E7
:0417000000000000E5
:0417010000000000E4
:0417020000000000E3
:0417030000000000E2
:0417040000000000E1
:0417050000000000E0
:0417060000000000DF
:0417070000000000DE
:0417080000000000DD
:0417090000000000DC
:04170A0000000000DB
:04170B0000000000DA
:04170C0000000000D9
:04170D0000000000D8
:04170E0000000000D7
:04170F0000000000D6
:0417100000000000D5
:0417110000000000D4
:0417120000000000D3
:0417130000000000D2
:0417140000000000D1
:0417150000000000D0
:0417160000000000CF
:0417170000000000CE
:0417180000000000CD
:0417190000000000CC
:04171A0000000000CB
:04171B0000000000CA
:04171C0000000000C9
:04171D0000000000C8
:04171E0000000000C7
:04171F0000000000C6
:0417200000000000C5
:0417210000000000C4
:0417220000000000C3
:0417230000000000C2
:0417240000000000C1
:0417250000000000C0
:0417260000000000BF
:0417270000000000BE
:0417280000000000BD
:0417290000000000BC
:04172A0000000000BB
:04172B0000000000BA
:04172C0000000000B9
:04172D0000000000B8
:04172E0000000000B7
:04172F0000000000B6
:0417300000000000B5
:0417310000000000B4
:0417320000000000B3
:0417330000000000B2
:0417340000000000B1
:0417350000000000B0
:0417360000000000AF
:0417370000000000AE
:0417380000000000AD
:0417390000000000AC
:04173A0000000000AB
:04173B0000000000AA
:04173C0000000000A9
:04173D0000000000A8
:04173E0000000000A7
:04173F0000000000A6
:0417400000000000A5
:0417410000000000A4
:0417420000000000A3
:0417430000000000A2
:0417440000000000A1
:0417450000000000A0
:04174600000000009F
:04174700000000009E
:04174800000000009D
:04174900000000009C
:04174A00000000009B
:04174B00000000009A
:04174C000000000099
:04174D000000000098
:04174E000000000097
:04174F000000000096
:041750000000000095
:041751000000000094
:041752000000000093
:041753000000000092
:041754000000000091
:041755000000000090
:04175600000000008F
:04175700000000008E
:04175800000000008D
:04175900000000008C
:04175A00000000008B
:04175B00000000008A
:04175C000000000089
:04175D000000000088
:04175E000000000087
:04175F000000000086
:041760000000000085
:041761000000000084
:041762000000000083
:041763000000000082
:041764000000000081
:041765000000000080
:04176600000000007F
:04176700000000007E
:04176800000000007D
:04176900000000007C
:04176A00000000007B
:04176B00000000007A
:04176C000000000079
:04176D000000000078
:04176E000000000077
:04176F000000000076
:041770000000000075
:041771000000000074
:041772000000000073
:041773000000000072
:041774000000000071
:041775000000000070
:04177600000000006F
:04177700000000006E
:04177800000000006D
:04177900000000006C
:04177A00000000006B
:04177B00000000006A
:04177C000000000069
:04177D000000000068
:04177E000000000067
:04177F000000000066
:041780000000000065
:041781000000000064
:041782000000000063
:041783000000000062
:041784000000000061
:041785000000000060
:04178600000000005F
:04178700000000005E
:04178800000000005D
:04178900000000005C
:04178A00000000005B
:04178B00000000005A
:04178C000000000059
:04178D000000000058
:04178E000000000057
:04178F000000000056
:041790000000000055
:041791000000000054
:041792000000000053
:041793000000000052
:041794000000000051
:041795000000000050
:04179600000000004F
:04179700000000004E
:04179800000000004D
:04179900000000004C
:04179A00000000004B
:04179B00000000004A
:04179C000000000049
:04179D000000000048
:04179E000000000047
:04179F000000000046
:0417A0000000000045
:0417A1000000000044
:0417A2000000000043
:0417A3000000000042
:0417A4000000000041
:0417A5000000000040
:0417A600000000003F
:0417A700000000003E
:0417A800000000003D
:0417A900000000003C
:0417AA00000000003B
:0417AB00000000003A
:0417AC000000000039
:0417AD000000000038
:0417AE000000000037
:0417AF000000000036
:0417B0000000000035
:0417B1000000000034
:0417B2000000000033
:0417B3000000000032
:0417B4000000000031
:0417B5000000000030
:0417B600000000002F
:0417B700000000002E
:0417B800000000002D
:0417B900000000002C
:0417BA00000000002B
:0417BB00000000002A
:0417BC000000000029
:0417BD000000000028
:0417BE000000000027
:0417BF000000000026
:0417C0000000000025
:0417C1000000000024
:0417C2000000000023
:0417C3000000000022
:0417C4000000000021
:0417C5000000000020
:0417C600000000001F
:0417C700000000001E
:0417C800000000001D
:0417C900000000001C
:0417CA00000000001B
:0417CB00000000001A
:0417CC000000000019
:0417CD000000000018
:0417CE000000000017
:0417CF000000000016
:0417D0000000000015
:0417D1000000000014
:0417D2000000000013
:0417D3000000000012
:0417D4000000000011
:0417D5000000000010
:0417D600000000000F
:0417D700000000000E
:0417D800000000000D
:0417D900000000000C
:0417DA00000000000B
:0417DB00000000000A
:0417DC000000000009
:0417DD000000000008
:0417DE000000000007
:0417DF000000000006
:0417E0000000000005
:0417E1000000000004
:0417E2000000000003
:0417E3000000000002
:0417E4000000000001
:0417E5000000000000
:0417E60000000000FF
:0417E70000000000FE
:0417E80000000000FD
:0417E90000000000FC
:0417EA0000000000FB
:0417EB0000000000FA
:0417EC0000000000F9
:0417ED0000000000F8
:0417EE0000000000F7
:0417EF0000000000F6
:0417F00000000000F5
:0417F10000000000F4
:0417F20000000000F3
:0417F30000000000F2
:0417F40000000000F1
:0417F50000000000F0
:0417F60000000000EF
:0417F70000000000EE
:0417F80000000000ED
:0417F90000000000EC
:0417FA0000000000EB
:0417FB0000000000EA
:0417FC0000000000E9
:0417FD0000000000E8
:0417FE0000000000E7
:0417FF0000000000E6
:0418000000000000E4
:0418010000000000E3
:0418020000000000E2
:0418030000000000E1
:0418040000000000E0
:0418050000000000DF
:0418060000000000DE
:0418070000000000DD
:0418080000000000DC
:0418090000000000DB
:04180A0000000000DA
:04180B0000000000D9
:04180C0000000000D8
:04180D0000000000D7
:04180E0000000000D6
:04180F0000000000D5
:0418100000000000D4
:0418110000000000D3
:0418120000000000D2
:0418130000000000D1
:0418140000000000D0
:0418150000000000CF
:0418160000000000CE
:0418170000000000CD
:0418180000000000CC
:0418190000000000CB
:04181A0000000000CA
:04181B0000000000C9
:04181C0000000000C8
:04181D0000000000C7
:04181E0000000000C6
:04181F0000000000C5
:0418200000000000C4
:0418210000000000C3
:0418220000000000C2
:0418230000000000C1
:0418240000000000C0
:0418250000000000BF
:0418260000000000BE
:0418270000000000BD
:0418280000000000BC
:0418290000000000BB
:04182A0000000000BA
:04182B0000000000B9
:04182C0000000000B8
:04182D0000000000B7
:04182E0000000000B6
:04182F0000000000B5
:0418300000000000B4
:0418310000000000B3
:0418320000000000B2
:0418330000000000B1
:0418340000000000B0
:0418350000000000AF
:0418360000000000AE
:0418370000000000AD
:0418380000000000AC
:0418390000000000AB
:04183A0000000000AA
:04183B0000000000A9
:04183C0000000000A8
:04183D0000000000A7
:04183E0000000000A6
:04183F0000000000A5
:0418400000000000A4
:0418410000000000A3
:0418420000000000A2
:0418430000000000A1
:0418440000000000A0
:04184500000000009F
:04184600000000009E
:04184700000000009D
:04184800000000009C
:04184900000000009B
:04184A00000000009A
:04184B000000000099
:04184C000000000098
:04184D000000000097
:04184E000000000096
:04184F000000000095
:041850000000000094
:041851000000000093
:041852000000000092
:041853000000000091
:041854000000000090
:04185500000000008F
:04185600000000008E
:04185700000000008D
:04185800000000008C
:04185900000000008B
:04185A00000000008A
:04185B000000000089
:04185C000000000088
:04185D000000000087
:04185E000000000086
:04185F000000000085
:041860000000000084
:041861000000000083
:041862000000000082
:041863000000000081
:041864000000000080
:04186500000000007F
:04186600000000007E
:04186700000000007D
:04186800000000007C
:04186900000000007B
:04186A00000000007A
:04186B000000000079
:04186C000000000078
:04186D000000000077
:04186E000000000076
:04186F000000000075
:041870000000000074
:041871000000000073
:041872000000000072
:041873000000000071
:041874000000000070
:04187500000000006F
:04187600000000006E
:04187700000000006D
:04187800000000006C
:04187900000000006B
:04187A00000000006A
:04187B000000000069
:04187C000000000068
:04187D000000000067
:04187E000000000066
:04187F000000000065
:041880000000000064
:041881000000000063
:041882000000000062
:041883000000000061
:041884000000000060
:04188500000000005F
:04188600000000005E
:04188700000000005D
:04188800000000005C
:04188900000000005B
:04188A00000000005A
:04188B000000000059
:04188C000000000058
:04188D000000000057
:04188E000000000056
:04188F000000000055
:041890000000000054
:041891000000000053
:041892000000000052
:041893000000000051
:041894000000000050
:04189500000000004F
:04189600000000004E
:04189700000000004D
:04189800000000004C
:04189900000000004B
:04189A00000000004A
:04189B000000000049
:04189C000000000048
:04189D000000000047
:04189E000000000046
:04189F000000000045
:0418A0000000000044
:0418A1000000000043
:0418A2000000000042
:0418A3000000000041
:0418A4000000000040
:0418A500000000003F
:0418A600000000003E
:0418A700000000003D
:0418A800000000003C
:0418A900000000003B
:0418AA00000000003A
:0418AB000000000039
:0418AC000000000038
:0418AD000000000037
:0418AE000000000036
:0418AF000000000035
:0418B0000000000034
:0418B1000000000033
:0418B2000000000032
:0418B3000000000031
:0418B4000000000030
:0418B500000000002F
:0418B600000000002E
:0418B700000000002D
:0418B800000000002C
:0418B900000000002B
:0418BA00000000002A
:0418BB000000000029
:0418BC000000000028
:0418BD000000000027
:0418BE000000000026
:0418BF000000000025
:0418C0000000000024
:0418C1000000000023
:0418C2000000000022
:0418C3000000000021
:0418C4000000000020
:0418C500000000001F
:0418C600000000001E
:0418C700000000001D
:0418C800000000001C
:0418C900000000001B
:0418CA00000000001A
:0418CB000000000019
:0418CC000000000018
:0418CD000000000017
:0418CE000000000016
:0418CF000000000015
:0418D0000000000014
:0418D1000000000013
:0418D2000000000012
:0418D3000000000011
:0418D4000000000010
:0418D500000000000F
:0418D600000000000E
:0418D700000000000D
:0418D800000000000C
:0418D900000000000B
:0418DA00000000000A
:0418DB000000000009
:0418DC000000000008
:0418DD000000000007
:0418DE000000000006
:0418DF000000000005
:0418E0000000000004
:0418E1000000000003
:0418E2000000000002
:0418E3000000000001
:0418E4000000000000
:0418E50000000000FF
:0418E60000000000FE
:0418E70000000000FD
:0418E80000000000FC
:0418E90000000000FB
:0418EA0000000000FA
:0418EB0000000000F9
:0418EC0000000000F8
:0418ED0000000000F7
:0418EE0000000000F6
:0418EF0000000000F5
:0418F00000000000F4
:0418F10000000000F3
:0418F20000000000F2
:0418F30000000000F1
:0418F40000000000F0
:0418F50000000000EF
:0418F60000000000EE
:0418F70000000000ED
:0418F80000000000EC
:0418F90000000000EB
:0418FA0000000000EA
:0418FB0000000000E9
:0418FC0000000000E8
:0418FD0000000000E7
:0418FE0000000000E6
:0418FF0000000000E5
:0419000000000000E3
:0419010000000000E2
:0419020000000000E1
:0419030000000000E0
:0419040000000000DF
:0419050000000000DE
:0419060000000000DD
:0419070000000000DC
:0419080000000000DB
:0419090000000000DA
:04190A0000000000D9
:04190B0000000000D8
:04190C0000000000D7
:04190D0000000000D6
:04190E0000000000D5
:04190F0000000000D4
:0419100000000000D3
:0419110000000000D2
:0419120000000000D1
:0419130000000000D0
:0419140000000000CF
:0419150000000000CE
:0419160000000000CD
:0419170000000000CC
:0419180000000000CB
:0419190000000000CA
:04191A0000000000C9
:04191B0000000000C8
:04191C0000000000C7
:04191D0000000000C6
:04191E0000000000C5
:04191F0000000000C4
:0419200000000000C3
:0419210000000000C2
:0419220000000000C1
:0419230000000000C0
:0419240000000000BF
:0419250000000000BE
:0419260000000000BD
:0419270000000000BC
:0419280000000000BB
:0419290000000000BA
:04192A0000000000B9
:04192B0000000000B8
:04192C0000000000B7
:04192D0000000000B6
:04192E0000000000B5
:04192F0000000000B4
:0419300000000000B3
:0419310000000000B2
:0419320000000000B1
:0419330000000000B0
:0419340000000000AF
:0419350000000000AE
:0419360000000000AD
:0419370000000000AC
:0419380000000000AB
:0419390000000000AA
:04193A0000000000A9
:04193B0000000000A8
:04193C0000000000A7
:04193D0000000000A6
:04193E0000000000A5
:04193F0000000000A4
:0419400000000000A3
:0419410000000000A2
:0419420000000000A1
:0419430000000000A0
:04194400000000009F
:04194500000000009E
:04194600000000009D
:04194700000000009C
:04194800000000009B
:04194900000000009A
:04194A000000000099
:04194B000000000098
:04194C000000000097
:04194D000000000096
:04194E000000000095
:04194F000000000094
:041950000000000093
:041951000000000092
:041952000000000091
:041953000000000090
:04195400000000008F
:04195500000000008E
:04195600000000008D
:04195700000000008C
:04195800000000008B
:04195900000000008A
:04195A000000000089
:04195B000000000088
:04195C000000000087
:04195D000000000086
:04195E000000000085
:04195F000000000084
:041960000000000083
:041961000000000082
:041962000000000081
:041963000000000080
:04196400000000007F
:04196500000000007E
:04196600000000007D
:04196700000000007C
:04196800000000007B
:04196900000000007A
:04196A000000000079
:04196B000000000078
:04196C000000000077
:04196D000000000076
:04196E000000000075
:04196F000000000074
:041970000000000073
:041971000000000072
:041972000000000071
:041973000000000070
:04197400000000006F
:04197500000000006E
:04197600000000006D
:04197700000000006C
:04197800000000006B
:04197900000000006A
:04197A000000000069
:04197B000000000068
:04197C000000000067
:04197D000000000066
:04197E000000000065
:04197F000000000064
:041980000000000063
:041981000000000062
:041982000000000061
:041983000000000060
:04198400000000005F
:04198500000000005E
:04198600000000005D
:04198700000000005C
:04198800000000005B
:04198900000000005A
:04198A000000000059
:04198B000000000058
:04198C000000000057
:04198D000000000056
:04198E000000000055
:04198F000000000054
:041990000000000053
:041991000000000052
:041992000000000051
:041993000000000050
:04199400000000004F
:04199500000000004E
:04199600000000004D
:04199700000000004C
:04199800000000004B
:04199900000000004A
:04199A000000000049
:04199B000000000048
:04199C000000000047
:04199D000000000046
:04199E000000000045
:04199F000000000044
:0419A0000000000043
:0419A1000000000042
:0419A2000000000041
:0419A3000000000040
:0419A400000000003F
:0419A500000000003E
:0419A600000000003D
:0419A700000000003C
:0419A800000000003B
:0419A900000000003A
:0419AA000000000039
:0419AB000000000038
:0419AC000000000037
:0419AD000000000036
:0419AE000000000035
:0419AF000000000034
:0419B0000000000033
:0419B1000000000032
:0419B2000000000031
:0419B3000000000030
:0419B400000000002F
:0419B500000000002E
:0419B600000000002D
:0419B700000000002C
:0419B800000000002B
:0419B900000000002A
:0419BA000000000029
:0419BB000000000028
:0419BC000000000027
:0419BD000000000026
:0419BE000000000025
:0419BF000000000024
:0419C0000000000023
:0419C1000000000022
:0419C2000000000021
:0419C3000000000020
:0419C400000000001F
:0419C500000000001E
:0419C600000000001D
:0419C700000000001C
:0419C800000000001B
:0419C900000000001A
:0419CA000000000019
:0419CB000000000018
:0419CC000000000017
:0419CD000000000016
:0419CE000000000015
:0419CF000000000014
:0419D0000000000013
:0419D1000000000012
:0419D2000000000011
:0419D3000000000010
:0419D400000000000F
:0419D500000000000E
:0419D600000000000D
:0419D700000000000C
:0419D800000000000B
:0419D900000000000A
:0419DA000000000009
:0419DB000000000008
:0419DC000000000007
:0419DD000000000006
:0419DE000000000005
:0419DF000000000004
:0419E0000000000003
:0419E1000000000002
:0419E2000000000001
:0419E3000000000000
:0419E40000000000FF
:0419E50000000000FE
:0419E60000000000FD
:0419E70000000000FC
:0419E80000000000FB
:0419E90000000000FA
:0419EA0000000000F9
:0419EB0000000000F8
:0419EC0000000000F7
:0419ED0000000000F6
:0419EE0000000000F5
:0419EF0000000000F4
:0419F00000000000F3
:0419F10000000000F2
:0419F20000000000F1
:0419F30000000000F0
:0419F40000000000EF
:0419F50000000000EE
:0419F60000000000ED
:0419F70000000000EC
:0419F80000000000EB
:0419F90000000000EA
:0419FA0000000000E9
:0419FB0000000000E8
:0419FC0000000000E7
:0419FD0000000000E6
:0419FE0000000000E5
:0419FF0000000000E4
:041A000000000000E2
:041A010000000000E1
:041A020000000000E0
:041A030000000000DF
:041A040000000000DE
:041A050000000000DD
:041A060000000000DC
:041A070000000000DB
:041A080000000000DA
:041A090000000000D9
:041A0A0000000000D8
:041A0B0000000000D7
:041A0C0000000000D6
:041A0D0000000000D5
:041A0E0000000000D4
:041A0F0000000000D3
:041A100000000000D2
:041A110000000000D1
:041A120000000000D0
:041A130000000000CF
:041A140000000000CE
:041A150000000000CD
:041A160000000000CC
:041A170000000000CB
:041A180000000000CA
:041A190000000000C9
:041A1A0000000000C8
:041A1B0000000000C7
:041A1C0000000000C6
:041A1D0000000000C5
:041A1E0000000000C4
:041A1F0000000000C3
:041A200000000000C2
:041A210000000000C1
:041A220000000000C0
:041A230000000000BF
:041A240000000000BE
:041A250000000000BD
:041A260000000000BC
:041A270000000000BB
:041A280000000000BA
:041A290000000000B9
:041A2A0000000000B8
:041A2B0000000000B7
:041A2C0000000000B6
:041A2D0000000000B5
:041A2E0000000000B4
:041A2F0000000000B3
:041A300000000000B2
:041A310000000000B1
:041A320000000000B0
:041A330000000000AF
:041A340000000000AE
:041A350000000000AD
:041A360000000000AC
:041A370000000000AB
:041A380000000000AA
:041A390000000000A9
:041A3A0000000000A8
:041A3B0000000000A7
:041A3C0000000000A6
:041A3D0000000000A5
:041A3E0000000000A4
:041A3F0000000000A3
:041A400000000000A2
:041A410000000000A1
:041A420000000000A0
:041A4300000000009F
:041A4400000000009E
:041A4500000000009D
:041A4600000000009C
:041A4700000000009B
:041A4800000000009A
:041A49000000000099
:041A4A000000000098
:041A4B000000000097
:041A4C000000000096
:041A4D000000000095
:041A4E000000000094
:041A4F000000000093
:041A50000000000092
:041A51000000000091
:041A52000000000090
:041A5300000000008F
:041A5400000000008E
:041A5500000000008D
:041A5600000000008C
:041A5700000000008B
:041A5800000000008A
:041A59000000000089
:041A5A000000000088
:041A5B000000000087
:041A5C000000000086
:041A5D000000000085
:041A5E000000000084
:041A5F000000000083
:041A60000000000082
:041A61000000000081
:041A62000000000080
:041A6300000000007F
:041A6400000000007E
:041A6500000000007D
:041A6600000000007C
:041A6700000000007B
:041A6800000000007A
:041A69000000000079
:041A6A000000000078
:041A6B000000000077
:041A6C000000000076
:041A6D000000000075
:041A6E000000000074
:041A6F000000000073
:041A70000000000072
:041A71000000000071
:041A72000000000070
:041A7300000000006F
:041A7400000000006E
:041A7500000000006D
:041A7600000000006C
:041A7700000000006B
:041A7800000000006A
:041A79000000000069
:041A7A000000000068
:041A7B000000000067
:041A7C000000000066
:041A7D000000000065
:041A7E000000000064
:041A7F000000000063
:041A80000000000062
:041A81000000000061
:041A82000000000060
:041A8300000000005F
:041A8400000000005E
:041A8500000000005D
:041A8600000000005C
:041A8700000000005B
:041A8800000000005A
:041A89000000000059
:041A8A000000000058
:041A8B000000000057
:041A8C000000000056
:041A8D000000000055
:041A8E000000000054
:041A8F000000000053
:041A90000000000052
:041A91000000000051
:041A92000000000050
:041A9300000000004F
:041A9400000000004E
:041A9500000000004D
:041A9600000000004C
:041A9700000000004B
:041A9800000000004A
:041A99000000000049
:041A9A000000000048
:041A9B000000000047
:041A9C000000000046
:041A9D000000000045
:041A9E000000000044
:041A9F000000000043
:041AA0000000000042
:041AA1000000000041
:041AA2000000000040
:041AA300000000003F
:041AA400000000003E
:041AA500000000003D
:041AA600000000003C
:041AA700000000003B
:041AA800000000003A
:041AA9000000000039
:041AAA000000000038
:041AAB000000000037
:041AAC000000000036
:041AAD000000000035
:041AAE000000000034
:041AAF000000000033
:041AB0000000000032
:041AB1000000000031
:041AB2000000000030
:041AB300000000002F
:041AB400000000002E
:041AB500000000002D
:041AB600000000002C
:041AB700000000002B
:041AB800000000002A
:041AB9000000000029
:041ABA000000000028
:041ABB000000000027
:041ABC000000000026
:041ABD000000000025
:041ABE000000000024
:041ABF000000000023
:041AC0000000000022
:041AC1000000000021
:041AC2000000000020
:041AC300000000001F
:041AC400000000001E
:041AC500000000001D
:041AC600000000001C
:041AC700000000001B
:041AC800000000001A
:041AC9000000000019
:041ACA000000000018
:041ACB000000000017
:041ACC000000000016
:041ACD000000000015
:041ACE000000000014
:041ACF000000000013
:041AD0000000000012
:041AD1000000000011
:041AD2000000000010
:041AD300000000000F
:041AD400000000000E
:041AD500000000000D
:041AD600000000000C
:041AD700000000000B
:041AD800000000000A
:041AD9000000000009
:041ADA000000000008
:041ADB000000000007
:041ADC000000000006
:041ADD000000000005
:041ADE000000000004
:041ADF000000000003
:041AE0000000000002
:041AE1000000000001
:041AE2000000000000
:041AE30000000000FF
:041AE40000000000FE
:041AE50000000000FD
:041AE60000000000FC
:041AE70000000000FB
:041AE80000000000FA
:041AE90000000000F9
:041AEA0000000000F8
:041AEB0000000000F7
:041AEC0000000000F6
:041AED0000000000F5
:041AEE0000000000F4
:041AEF0000000000F3
:041AF00000000000F2
:041AF10000000000F1
:041AF20000000000F0
:041AF30000000000EF
:041AF40000000000EE
:041AF50000000000ED
:041AF60000000000EC
:041AF70000000000EB
:041AF80000000000EA
:041AF90000000000E9
:041AFA0000000000E8
:041AFB0000000000E7
:041AFC0000000000E6
:041AFD0000000000E5
:041AFE0000000000E4
:041AFF0000000000E3
:041B000000000000E1
:041B010000000000E0
:041B020000000000DF
:041B030000000000DE
:041B040000000000DD
:041B050000000000DC
:041B060000000000DB
:041B070000000000DA
:041B080000000000D9
:041B090000000000D8
:041B0A0000000000D7
:041B0B0000000000D6
:041B0C0000000000D5
:041B0D0000000000D4
:041B0E0000000000D3
:041B0F0000000000D2
:041B100000000000D1
:041B110000000000D0
:041B120000000000CF
:041B130000000000CE
:041B140000000000CD
:041B150000000000CC
:041B160000000000CB
:041B170000000000CA
:041B180000000000C9
:041B190000000000C8
:041B1A0000000000C7
:041B1B0000000000C6
:041B1C0000000000C5
:041B1D0000000000C4
:041B1E0000000000C3
:041B1F0000000000C2
:041B200000000000C1
:041B210000000000C0
:041B220000000000BF
:041B230000000000BE
:041B240000000000BD
:041B250000000000BC
:041B260000000000BB
:041B270000000000BA
:041B280000000000B9
:041B290000000000B8
:041B2A0000000000B7
:041B2B0000000000B6
:041B2C0000000000B5
:041B2D0000000000B4
:041B2E0000000000B3
:041B2F0000000000B2
:041B300000000000B1
:041B310000000000B0
:041B320000000000AF
:041B330000000000AE
:041B340000000000AD
:041B350000000000AC
:041B360000000000AB
:041B370000000000AA
:041B380000000000A9
:041B390000000000A8
:041B3A0000000000A7
:041B3B0000000000A6
:041B3C0000000000A5
:041B3D0000000000A4
:041B3E0000000000A3
:041B3F0000000000A2
:041B400000000000A1
:041B410000000000A0
:041B4200000000009F
:041B4300000000009E
:041B4400000000009D
:041B4500000000009C
:041B4600000000009B
:041B4700000000009A
:041B48000000000099
:041B49000000000098
:041B4A000000000097
:041B4B000000000096
:041B4C000000000095
:041B4D000000000094
:041B4E000000000093
:041B4F000000000092
:041B50000000000091
:041B51000000000090
:041B5200000000008F
:041B5300000000008E
:041B5400000000008D
:041B5500000000008C
:041B5600000000008B
:041B5700000000008A
:041B58000000000089
:041B59000000000088
:041B5A000000000087
:041B5B000000000086
:041B5C000000000085
:041B5D000000000084
:041B5E000000000083
:041B5F000000000082
:041B60000000000081
:041B61000000000080
:041B6200000000007F
:041B6300000000007E
:041B6400000000007D
:041B6500000000007C
:041B6600000000007B
:041B6700000000007A
:041B68000000000079
:041B69000000000078
:041B6A000000000077
:041B6B000000000076
:041B6C000000000075
:041B6D000000000074
:041B6E000000000073
:041B6F000000000072
:041B70000000000071
:041B71000000000070
:041B7200000000006F
:041B7300000000006E
:041B7400000000006D
:041B7500000000006C
:041B7600000000006B
:041B7700000000006A
:041B78000000000069
:041B79000000000068
:041B7A000000000067
:041B7B000000000066
:041B7C000000000065
:041B7D000000000064
:041B7E000000000063
:041B7F000000000062
:041B80000000000061
:041B81000000000060
:041B8200000000005F
:041B8300000000005E
:041B8400000000005D
:041B8500000000005C
:041B8600000000005B
:041B8700000000005A
:041B88000000000059
:041B89000000000058
:041B8A000000000057
:041B8B000000000056
:041B8C000000000055
:041B8D000000000054
:041B8E000000000053
:041B8F000000000052
:041B90000000000051
:041B91000000000050
:041B9200000000004F
:041B9300000000004E
:041B9400000000004D
:041B9500000000004C
:041B9600000000004B
:041B9700000000004A
:041B98000000000049
:041B99000000000048
:041B9A000000000047
:041B9B000000000046
:041B9C000000000045
:041B9D000000000044
:041B9E000000000043
:041B9F000000000042
:041BA0000000000041
:041BA1000000000040
:041BA200000000003F
:041BA300000000003E
:041BA400000000003D
:041BA500000000003C
:041BA600000000003B
:041BA700000000003A
:041BA8000000000039
:041BA9000000000038
:041BAA000000000037
:041BAB000000000036
:041BAC000000000035
:041BAD000000000034
:041BAE000000000033
:041BAF000000000032
:041BB0000000000031
:041BB1000000000030
:041BB200000000002F
:041BB300000000002E
:041BB400000000002D
:041BB500000000002C
:041BB600000000002B
:041BB700000000002A
:041BB8000000000029
:041BB9000000000028
:041BBA000000000027
:041BBB000000000026
:041BBC000000000025
:041BBD000000000024
:041BBE000000000023
:041BBF000000000022
:041BC0000000000021
:041BC1000000000020
:041BC200000000001F
:041BC300000000001E
:041BC400000000001D
:041BC500000000001C
:041BC600000000001B
:041BC700000000001A
:041BC8000000000019
:041BC9000000000018
:041BCA000000000017
:041BCB000000000016
:041BCC000000000015
:041BCD000000000014
:041BCE000000000013
:041BCF000000000012
:041BD0000000000011
:041BD1000000000010
:041BD200000000000F
:041BD300000000000E
:041BD400000000000D
:041BD500000000000C
:041BD600000000000B
:041BD700000000000A
:041BD8000000000009
:041BD9000000000008
:041BDA000000000007
:041BDB000000000006
:041BDC000000000005
:041BDD000000000004
:041BDE000000000003
:041BDF000000000002
:041BE0000000000001
:041BE1000000000000
:041BE20000000000FF
:041BE30000000000FE
:041BE40000000000FD
:041BE50000000000FC
:041BE60000000000FB
:041BE70000000000FA
:041BE80000000000F9
:041BE90000000000F8
:041BEA0000000000F7
:041BEB0000000000F6
:041BEC0000000000F5
:041BED0000000000F4
:041BEE0000000000F3
:041BEF0000000000F2
:041BF00000000000F1
:041BF10000000000F0
:041BF20000000000EF
:041BF30000000000EE
:041BF40000000000ED
:041BF50000000000EC
:041BF60000000000EB
:041BF70000000000EA
:041BF80000000000E9
:041BF90000000000E8
:041BFA0000000000E7
:041BFB0000000000E6
:041BFC0000000000E5
:041BFD0000000000E4
:041BFE0000000000E3
:041BFF0000000000E2
:041C000000000000E0
:041C010000000000DF
:041C020000000000DE
:041C030000000000DD
:041C040000000000DC
:041C050000000000DB
:041C060000000000DA
:041C070000000000D9
:041C080000000000D8
:041C090000000000D7
:041C0A0000000000D6
:041C0B0000000000D5
:041C0C0000000000D4
:041C0D0000000000D3
:041C0E0000000000D2
:041C0F0000000000D1
:041C100000000000D0
:041C110000000000CF
:041C120000000000CE
:041C130000000000CD
:041C140000000000CC
:041C150000000000CB
:041C160000000000CA
:041C170000000000C9
:041C180000000000C8
:041C190000000000C7
:041C1A0000000000C6
:041C1B0000000000C5
:041C1C0000000000C4
:041C1D0000000000C3
:041C1E0000000000C2
:041C1F0000000000C1
:041C200000000000C0
:041C210000000000BF
:041C220000000000BE
:041C230000000000BD
:041C240000000000BC
:041C250000000000BB
:041C260000000000BA
:041C270000000000B9
:041C280000000000B8
:041C290000000000B7
:041C2A0000000000B6
:041C2B0000000000B5
:041C2C0000000000B4
:041C2D0000000000B3
:041C2E0000000000B2
:041C2F0000000000B1
:041C300000000000B0
:041C310000000000AF
:041C320000000000AE
:041C330000000000AD
:041C340000000000AC
:041C350000000000AB
:041C360000000000AA
:041C370000000000A9
:041C380000000000A8
:041C390000000000A7
:041C3A0000000000A6
:041C3B0000000000A5
:041C3C0000000000A4
:041C3D0000000000A3
:041C3E0000000000A2
:041C3F0000000000A1
:041C400000000000A0
:041C4100000000009F
:041C4200000000009E
:041C4300000000009D
:041C4400000000009C
:041C4500000000009B
:041C4600000000009A
:041C47000000000099
:041C48000000000098
:041C49000000000097
:041C4A000000000096
:041C4B000000000095
:041C4C000000000094
:041C4D000000000093
:041C4E000000000092
:041C4F000000000091
:041C50000000000090
:041C5100000000008F
:041C5200000000008E
:041C5300000000008D
:041C5400000000008C
:041C5500000000008B
:041C5600000000008A
:041C57000000000089
:041C58000000000088
:041C59000000000087
:041C5A000000000086
:041C5B000000000085
:041C5C000000000084
:041C5D000000000083
:041C5E000000000082
:041C5F000000000081
:041C60000000000080
:041C6100000000007F
:041C6200000000007E
:041C6300000000007D
:041C6400000000007C
:041C6500000000007B
:041C6600000000007A
:041C67000000000079
:041C68000000000078
:041C69000000000077
:041C6A000000000076
:041C6B000000000075
:041C6C000000000074
:041C6D000000000073
:041C6E000000000072
:041C6F000000000071
:041C70000000000070
:041C7100000000006F
:041C7200000000006E
:041C7300000000006D
:041C7400000000006C
:041C7500000000006B
:041C7600000000006A
:041C77000000000069
:041C78000000000068
:041C79000000000067
:041C7A000000000066
:041C7B000000000065
:041C7C000000000064
:041C7D000000000063
:041C7E000000000062
:041C7F000000000061
:041C80000000000060
:041C8100000000005F
:041C8200000000005E
:041C8300000000005D
:041C8400000000005C
:041C8500000000005B
:041C8600000000005A
:041C87000000000059
:041C88000000000058
:041C89000000000057
:041C8A000000000056
:041C8B000000000055
:041C8C000000000054
:041C8D000000000053
:041C8E000000000052
:041C8F000000000051
:041C90000000000050
:041C9100000000004F
:041C9200000000004E
:041C9300000000004D
:041C9400000000004C
:041C9500000000004B
:041C9600000000004A
:041C97000000000049
:041C98000000000048
:041C99000000000047
:041C9A000000000046
:041C9B000000000045
:041C9C000000000044
:041C9D000000000043
:041C9E000000000042
:041C9F000000000041
:041CA0000000000040
:041CA100000000003F
:041CA200000000003E
:041CA300000000003D
:041CA400000000003C
:041CA500000000003B
:041CA600000000003A
:041CA7000000000039
:041CA8000000000038
:041CA9000000000037
:041CAA000000000036
:041CAB000000000035
:041CAC000000000034
:041CAD000000000033
:041CAE000000000032
:041CAF000000000031
:041CB0000000000030
:041CB100000000002F
:041CB200000000002E
:041CB300000000002D
:041CB400000000002C
:041CB500000000002B
:041CB600000000002A
:041CB7000000000029
:041CB8000000000028
:041CB9000000000027
:041CBA000000000026
:041CBB000000000025
:041CBC000000000024
:041CBD000000000023
:041CBE000000000022
:041CBF000000000021
:041CC0000000000020
:041CC100000000001F
:041CC200000000001E
:041CC300000000001D
:041CC400000000001C
:041CC500000000001B
:041CC600000000001A
:041CC7000000000019
:041CC8000000000018
:041CC9000000000017
:041CCA000000000016
:041CCB000000000015
:041CCC000000000014
:041CCD000000000013
:041CCE000000000012
:041CCF000000000011
:041CD0000000000010
:041CD100000000000F
:041CD200000000000E
:041CD300000000000D
:041CD400000000000C
:041CD500000000000B
:041CD600000000000A
:041CD7000000000009
:041CD8000000000008
:041CD9000000000007
:041CDA000000000006
:041CDB000000000005
:041CDC000000000004
:041CDD000000000003
:041CDE000000000002
:041CDF000000000001
:041CE0000000000000
:041CE10000000000FF
:041CE20000000000FE
:041CE30000000000FD
:041CE40000000000FC
:041CE50000000000FB
:041CE60000000000FA
:041CE70000000000F9
:041CE80000000000F8
:041CE90000000000F7
:041CEA0000000000F6
:041CEB0000000000F5
:041CEC0000000000F4
:041CED0000000000F3
:041CEE0000000000F2
:041CEF0000000000F1
:041CF00000000000F0
:041CF10000000000EF
:041CF20000000000EE
:041CF30000000000ED
:041CF40000000000EC
:041CF50000000000EB
:041CF60000000000EA
:041CF70000000000E9
:041CF80000000000E8
:041CF90000000000E7
:041CFA0000000000E6
:041CFB0000000000E5
:041CFC0000000000E4
:041CFD0000000000E3
:041CFE0000000000E2
:041CFF0000000000E1
:041D000000000000DF
:041D010000000000DE
:041D020000000000DD
:041D030000000000DC
:041D040000000000DB
:041D050000000000DA
:041D060000000000D9
:041D070000000000D8
:041D080000000000D7
:041D090000000000D6
:041D0A0000000000D5
:041D0B0000000000D4
:041D0C0000000000D3
:041D0D0000000000D2
:041D0E0000000000D1
:041D0F0000000000D0
:041D100000000000CF
:041D110000000000CE
:041D120000000000CD
:041D130000000000CC
:041D140000000000CB
:041D150000000000CA
:041D160000000000C9
:041D170000000000C8
:041D180000000000C7
:041D190000000000C6
:041D1A0000000000C5
:041D1B0000000000C4
:041D1C0000000000C3
:041D1D0000000000C2
:041D1E0000000000C1
:041D1F0000000000C0
:041D200000000000BF
:041D210000000000BE
:041D220000000000BD
:041D230000000000BC
:041D240000000000BB
:041D250000000000BA
:041D260000000000B9
:041D270000000000B8
:041D280000000000B7
:041D290000000000B6
:041D2A0000000000B5
:041D2B0000000000B4
:041D2C0000000000B3
:041D2D0000000000B2
:041D2E0000000000B1
:041D2F0000000000B0
:041D300000000000AF
:041D310000000000AE
:041D320000000000AD
:041D330000000000AC
:041D340000000000AB
:041D350000000000AA
:041D360000000000A9
:041D370000000000A8
:041D380000000000A7
:041D390000000000A6
:041D3A0000000000A5
:041D3B0000000000A4
:041D3C0000000000A3
:041D3D0000000000A2
:041D3E0000000000A1
:041D3F0000000000A0
:041D4000000000009F
:041D4100000000009E
:041D4200000000009D
:041D4300000000009C
:041D4400000000009B
:041D4500000000009A
:041D46000000000099
:041D47000000000098
:041D48000000000097
:041D49000000000096
:041D4A000000000095
:041D4B000000000094
:041D4C000000000093
:041D4D000000000092
:041D4E000000000091
:041D4F000000000090
:041D5000000000008F
:041D5100000000008E
:041D5200000000008D
:041D5300000000008C
:041D5400000000008B
:041D5500000000008A
:041D56000000000089
:041D57000000000088
:041D58000000000087
:041D59000000000086
:041D5A000000000085
:041D5B000000000084
:041D5C000000000083
:041D5D000000000082
:041D5E000000000081
:041D5F000000000080
:041D6000000000007F
:041D6100000000007E
:041D6200000000007D
:041D6300000000007C
:041D6400000000007B
:041D6500000000007A
:041D66000000000079
:041D67000000000078
:041D68000000000077
:041D69000000000076
:041D6A000000000075
:041D6B000000000074
:041D6C000000000073
:041D6D000000000072
:041D6E000000000071
:041D6F000000000070
:041D7000000000006F
:041D7100000000006E
:041D7200000000006D
:041D7300000000006C
:041D7400000000006B
:041D7500000000006A
:041D76000000000069
:041D77000000000068
:041D78000000000067
:041D79000000000066
:041D7A000000000065
:041D7B000000000064
:041D7C000000000063
:041D7D000000000062
:041D7E000000000061
:041D7F000000000060
:041D8000000000005F
:041D8100000000005E
:041D8200000000005D
:041D8300000000005C
:041D8400000000005B
:041D8500000000005A
:041D86000000000059
:041D87000000000058
:041D88000000000057
:041D89000000000056
:041D8A000000000055
:041D8B000000000054
:041D8C000000000053
:041D8D000000000052
:041D8E000000000051
:041D8F000000000050
:041D9000000000004F
:041D9100000000004E
:041D9200000000004D
:041D9300000000004C
:041D9400000000004B
:041D9500000000004A
:041D96000000000049
:041D97000000000048
:041D98000000000047
:041D99000000000046
:041D9A000000000045
:041D9B000000000044
:041D9C000000000043
:041D9D000000000042
:041D9E000000000041
:041D9F000000000040
:041DA000000000003F
:041DA100000000003E
:041DA200000000003D
:041DA300000000003C
:041DA400000000003B
:041DA500000000003A
:041DA6000000000039
:041DA7000000000038
:041DA8000000000037
:041DA9000000000036
:041DAA000000000035
:041DAB000000000034
:041DAC000000000033
:041DAD000000000032
:041DAE000000000031
:041DAF000000000030
:041DB000000000002F
:041DB100000000002E
:041DB200000000002D
:041DB300000000002C
:041DB400000000002B
:041DB500000000002A
:041DB6000000000029
:041DB7000000000028
:041DB8000000000027
:041DB9000000000026
:041DBA000000000025
:041DBB000000000024
:041DBC000000000023
:041DBD000000000022
:041DBE000000000021
:041DBF000000000020
:041DC000000000001F
:041DC100000000001E
:041DC200000000001D
:041DC300000000001C
:041DC400000000001B
:041DC500000000001A
:041DC6000000000019
:041DC7000000000018
:041DC8000000000017
:041DC9000000000016
:041DCA000000000015
:041DCB000000000014
:041DCC000000000013
:041DCD000000000012
:041DCE000000000011
:041DCF000000000010
:041DD000000000000F
:041DD100000000000E
:041DD200000000000D
:041DD300000000000C
:041DD400000000000B
:041DD500000000000A
:041DD6000000000009
:041DD7000000000008
:041DD8000000000007
:041DD9000000000006
:041DDA000000000005
:041DDB000000000004
:041DDC000000000003
:041DDD000000000002
:041DDE000000000001
:041DDF000000000000
:041DE00000000000FF
:041DE10000000000FE
:041DE20000000000FD
:041DE30000000000FC
:041DE40000000000FB
:041DE50000000000FA
:041DE60000000000F9
:041DE70000000000F8
:041DE80000000000F7
:041DE90000000000F6
:041DEA0000000000F5
:041DEB0000000000F4
:041DEC0000000000F3
:041DED0000000000F2
:041DEE0000000000F1
:041DEF0000000000F0
:041DF00000000000EF
:041DF10000000000EE
:041DF20000000000ED
:041DF30000000000EC
:041DF40000000000EB
:041DF50000000000EA
:041DF60000000000E9
:041DF70000000000E8
:041DF80000000000E7
:041DF90000000000E6
:041DFA0000000000E5
:041DFB0000000000E4
:041DFC0000000000E3
:041DFD0000000000E2
:041DFE0000000000E1
:041DFF0000000000E0
:041E000000000000DE
:041E010000000000DD
:041E020000000000DC
:041E030000000000DB
:041E040000000000DA
:041E050000000000D9
:041E060000000000D8
:041E070000000000D7
:041E080000000000D6
:041E090000000000D5
:041E0A0000000000D4
:041E0B0000000000D3
:041E0C0000000000D2
:041E0D0000000000D1
:041E0E0000000000D0
:041E0F0000000000CF
:041E100000000000CE
:041E110000000000CD
:041E120000000000CC
:041E130000000000CB
:041E140000000000CA
:041E150000000000C9
:041E160000000000C8
:041E170000000000C7
:041E180000000000C6
:041E190000000000C5
:041E1A0000000000C4
:041E1B0000000000C3
:041E1C0000000000C2
:041E1D0000000000C1
:041E1E0000000000C0
:041E1F0000000000BF
:041E200000000000BE
:041E210000000000BD
:041E220000000000BC
:041E230000000000BB
:041E240000000000BA
:041E250000000000B9
:041E260000000000B8
:041E270000000000B7
:041E280000000000B6
:041E290000000000B5
:041E2A0000000000B4
:041E2B0000000000B3
:041E2C0000000000B2
:041E2D0000000000B1
:041E2E0000000000B0
:041E2F0000000000AF
:041E300000000000AE
:041E310000000000AD
:041E320000000000AC
:041E330000000000AB
:041E340000000000AA
:041E350000000000A9
:041E360000000000A8
:041E370000000000A7
:041E380000000000A6
:041E390000000000A5
:041E3A0000000000A4
:041E3B0000000000A3
:041E3C0000000000A2
:041E3D0000000000A1
:041E3E0000000000A0
:041E3F00000000009F
:041E4000000000009E
:041E4100000000009D
:041E4200000000009C
:041E4300000000009B
:041E4400000000009A
:041E45000000000099
:041E46000000000098
:041E47000000000097
:041E48000000000096
:041E49000000000095
:041E4A000000000094
:041E4B000000000093
:041E4C000000000092
:041E4D000000000091
:041E4E000000000090
:041E4F00000000008F
:041E5000000000008E
:041E5100000000008D
:041E5200000000008C
:041E5300000000008B
:041E5400000000008A
:041E55000000000089
:041E56000000000088
:041E57000000000087
:041E58000000000086
:041E59000000000085
:041E5A000000000084
:041E5B000000000083
:041E5C000000000082
:041E5D000000000081
:041E5E000000000080
:041E5F00000000007F
:041E6000000000007E
:041E6100000000007D
:041E6200000000007C
:041E6300000000007B
:041E6400000000007A
:041E65000000000079
:041E66000000000078
:041E67000000000077
:041E68000000000076
:041E69000000000075
:041E6A000000000074
:041E6B000000000073
:041E6C000000000072
:041E6D000000000071
:041E6E000000000070
:041E6F00000000006F
:041E7000000000006E
:041E7100000000006D
:041E7200000000006C
:041E7300000000006B
:041E7400000000006A
:041E75000000000069
:041E76000000000068
:041E77000000000067
:041E78000000000066
:041E79000000000065
:041E7A000000000064
:041E7B000000000063
:041E7C000000000062
:041E7D000000000061
:041E7E000000000060
:041E7F00000000005F
:041E8000000000005E
:041E8100000000005D
:041E8200000000005C
:041E8300000000005B
:041E8400000000005A
:041E85000000000059
:041E86000000000058
:041E87000000000057
:041E88000000000056
:041E89000000000055
:041E8A000000000054
:041E8B000000000053
:041E8C000000000052
:041E8D000000000051
:041E8E000000000050
:041E8F00000000004F
:041E9000000000004E
:041E9100000000004D
:041E9200000000004C
:041E9300000000004B
:041E9400000000004A
:041E95000000000049
:041E96000000000048
:041E97000000000047
:041E98000000000046
:041E99000000000045
:041E9A000000000044
:041E9B000000000043
:041E9C000000000042
:041E9D000000000041
:041E9E000000000040
:041E9F00000000003F
:041EA000000000003E
:041EA100000000003D
:041EA200000000003C
:041EA300000000003B
:041EA400000000003A
:041EA5000000000039
:041EA6000000000038
:041EA7000000000037
:041EA8000000000036
:041EA9000000000035
:041EAA000000000034
:041EAB000000000033
:041EAC000000000032
:041EAD000000000031
:041EAE000000000030
:041EAF00000000002F
:041EB000000000002E
:041EB100000000002D
:041EB200000000002C
:041EB300000000002B
:041EB400000000002A
:041EB5000000000029
:041EB6000000000028
:041EB7000000000027
:041EB8000000000026
:041EB9000000000025
:041EBA000000000024
:041EBB000000000023
:041EBC000000000022
:041EBD000000000021
:041EBE000000000020
:041EBF00000000001F
:041EC000000000001E
:041EC100000000001D
:041EC200000000001C
:041EC300000000001B
:041EC400000000001A
:041EC5000000000019
:041EC6000000000018
:041EC7000000000017
:041EC8000000000016
:041EC9000000000015
:041ECA000000000014
:041ECB000000000013
:041ECC000000000012
:041ECD000000000011
:041ECE000000000010
:041ECF00000000000F
:041ED000000000000E
:041ED100000000000D
:041ED200000000000C
:041ED300000000000B
:041ED400000000000A
:041ED5000000000009
:041ED6000000000008
:041ED7000000000007
:041ED8000000000006
:041ED9000000000005
:041EDA000000000004
:041EDB000000000003
:041EDC000000000002
:041EDD000000000001
:041EDE000000000000
:041EDF0000000000FF
:041EE00000000000FE
:041EE10000000000FD
:041EE20000000000FC
:041EE30000000000FB
:041EE40000000000FA
:041EE50000000000F9
:041EE60000000000F8
:041EE70000000000F7
:041EE80000000000F6
:041EE90000000000F5
:041EEA0000000000F4
:041EEB0000000000F3
:041EEC0000000000F2
:041EED0000000000F1
:041EEE0000000000F0
:041EEF0000000000EF
:041EF00000000000EE
:041EF10000000000ED
:041EF20000000000EC
:041EF30000000000EB
:041EF40000000000EA
:041EF50000000000E9
:041EF60000000000E8
:041EF70000000000E7
:041EF80000000000E6
:041EF90000000000E5
:041EFA0000000000E4
:041EFB0000000000E3
:041EFC0000000000E2
:041EFD0000000000E1
:041EFE0000000000E0
:041EFF0000000000DF
:041F000000000000DD
:041F010000000000DC
:041F020000000000DB
:041F030000000000DA
:041F040000000000D9
:041F050000000000D8
:041F060000000000D7
:041F070000000000D6
:041F080000000000D5
:041F090000000000D4
:041F0A0000000000D3
:041F0B0000000000D2
:041F0C0000000000D1
:041F0D0000000000D0
:041F0E0000000000CF
:041F0F0000000000CE
:041F100000000000CD
:041F110000000000CC
:041F120000000000CB
:041F130000000000CA
:041F140000000000C9
:041F150000000000C8
:041F160000000000C7
:041F170000000000C6
:041F180000000000C5
:041F190000000000C4
:041F1A0000000000C3
:041F1B0000000000C2
:041F1C0000000000C1
:041F1D0000000000C0
:041F1E0000000000BF
:041F1F0000000000BE
:041F200000000000BD
:041F210000000000BC
:041F220000000000BB
:041F230000000000BA
:041F240000000000B9
:041F250000000000B8
:041F260000000000B7
:041F270000000000B6
:041F280000000000B5
:041F290000000000B4
:041F2A0000000000B3
:041F2B0000000000B2
:041F2C0000000000B1
:041F2D0000000000B0
:041F2E0000000000AF
:041F2F0000000000AE
:041F300000000000AD
:041F310000000000AC
:041F320000000000AB
:041F330000000000AA
:041F340000000000A9
:041F350000000000A8
:041F360000000000A7
:041F370000000000A6
:041F380000000000A5
:041F390000000000A4
:041F3A0000000000A3
:041F3B0000000000A2
:041F3C0000000000A1
:041F3D0000000000A0
:041F3E00000000009F
:041F3F00000000009E
:041F4000000000009D
:041F4100000000009C
:041F4200000000009B
:041F4300000000009A
:041F44000000000099
:041F45000000000098
:041F46000000000097
:041F47000000000096
:041F48000000000095
:041F49000000000094
:041F4A000000000093
:041F4B000000000092
:041F4C000000000091
:041F4D000000000090
:041F4E00000000008F
:041F4F00000000008E
:041F5000000000008D
:041F5100000000008C
:041F5200000000008B
:041F5300000000008A
:041F54000000000089
:041F55000000000088
:041F56000000000087
:041F57000000000086
:041F58000000000085
:041F59000000000084
:041F5A000000000083
:041F5B000000000082
:041F5C000000000081
:041F5D000000000080
:041F5E00000000007F
:041F5F00000000007E
:041F6000000000007D
:041F6100000000007C
:041F6200000000007B
:041F6300000000007A
:041F64000000000079
:041F65000000000078
:041F66000000000077
:041F67000000000076
:041F68000000000075
:041F69000000000074
:041F6A000000000073
:041F6B000000000072
:041F6C000000000071
:041F6D000000000070
:041F6E00000000006F
:041F6F00000000006E
:041F7000000000006D
:041F7100000000006C
:041F7200000000006B
:041F7300000000006A
:041F74000000000069
:041F75000000000068
:041F76000000000067
:041F77000000000066
:041F78000000000065
:041F79000000000064
:041F7A000000000063
:041F7B000000000062
:041F7C000000000061
:041F7D000000000060
:041F7E00000000005F
:041F7F00000000005E
:041F8000000000005D
:041F8100000000005C
:041F8200000000005B
:041F8300000000005A
:041F84000000000059
:041F85000000000058
:041F86000000000057
:041F87000000000056
:041F88000000000055
:041F89000000000054
:041F8A000000000053
:041F8B000000000052
:041F8C000000000051
:041F8D000000000050
:041F8E00000000004F
:041F8F00000000004E
:041F9000000000004D
:041F9100000000004C
:041F9200000000004B
:041F9300000000004A
:041F94000000000049
:041F95000000000048
:041F96000000000047
:041F97000000000046
:041F98000000000045
:041F99000000000044
:041F9A000000000043
:041F9B000000000042
:041F9C000000000041
:041F9D000000000040
:041F9E00000000003F
:041F9F00000000003E
:041FA000000000003D
:041FA100000000003C
:041FA200000000003B
:041FA300000000003A
:041FA4000000000039
:041FA5000000000038
:041FA6000000000037
:041FA7000000000036
:041FA8000000000035
:041FA9000000000034
:041FAA000000000033
:041FAB000000000032
:041FAC000000000031
:041FAD000000000030
:041FAE00000000002F
:041FAF00000000002E
:041FB000000000002D
:041FB100000000002C
:041FB200000000002B
:041FB300000000002A
:041FB4000000000029
:041FB5000000000028
:041FB6000000000027
:041FB7000000000026
:041FB8000000000025
:041FB9000000000024
:041FBA000000000023
:041FBB000000000022
:041FBC000000000021
:041FBD000000000020
:041FBE00000000001F
:041FBF00000000001E
:041FC000000000001D
:041FC100000000001C
:041FC200000000001B
:041FC300000000001A
:041FC4000000000019
:041FC5000000000018
:041FC6000000000017
:041FC7000000000016
:041FC8000000000015
:041FC9000000000014
:041FCA000000000013
:041FCB000000000012
:041FCC000000000011
:041FCD000000000010
:041FCE00000000000F
:041FCF00000000000E
:041FD000000000000D
:041FD100000000000C
:041FD200000000000B
:041FD300000000000A
:041FD4000000000009
:041FD5000000000008
:041FD6000000000007
:041FD7000000000006
:041FD8000000000005
:041FD9000000000004
:041FDA000000000003
:041FDB000000000002
:041FDC000000000001
:041FDD000000000000
:041FDE0000000000FF
:041FDF0000000000FE
:041FE00000000000FD
:041FE10000000000FC
:041FE20000000000FB
:041FE30000000000FA
:041FE40000000000F9
:041FE50000000000F8
:041FE60000000000F7
:041FE70000000000F6
:041FE80000000000F5
:041FE90000000000F4
:041FEA0000000000F3
:041FEB0000000000F2
:041FEC0000000000F1
:041FED0000000000F0
:041FEE0000000000EF
:041FEF0000000000EE
:041FF00000000000ED
:041FF10000000000EC
:041FF20000000000EB
:041FF30000000000EA
:041FF40000000000E9
:041FF50000000000E8
:041FF60000000000E7
:041FF70000000000E6
:041FF80000000000E5
:041FF90000000000E4
:041FFA0000000000E3
:041FFB0000000000E2
:041FFC0000000000E1
:041FFD0000000000E0
:041FFE0000000000DF
:041FFF0000000000DE
:0420000000000000DC
:0420010000000000DB
:0420020000000000DA
:0420030000000000D9
:0420040000000000D8
:0420050000000000D7
:0420060000000000D6
:0420070000000000D5
:0420080000000000D4
:0420090000000000D3
:04200A0000000000D2
:04200B0000000000D1
:04200C0000000000D0
:04200D0000000000CF
:04200E0000000000CE
:04200F0000000000CD
:0420100000000000CC
:0420110000000000CB
:0420120000000000CA
:0420130000000000C9
:0420140000000000C8
:0420150000000000C7
:0420160000000000C6
:0420170000000000C5
:0420180000000000C4
:0420190000000000C3
:04201A0000000000C2
:04201B0000000000C1
:04201C0000000000C0
:04201D0000000000BF
:04201E0000000000BE
:04201F0000000000BD
:0420200000000000BC
:0420210000000000BB
:0420220000000000BA
:0420230000000000B9
:0420240000000000B8
:0420250000000000B7
:0420260000000000B6
:0420270000000000B5
:0420280000000000B4
:0420290000000000B3
:04202A0000000000B2
:04202B0000000000B1
:04202C0000000000B0
:04202D0000000000AF
:04202E0000000000AE
:04202F0000000000AD
:0420300000000000AC
:0420310000000000AB
:0420320000000000AA
:0420330000000000A9
:0420340000000000A8
:0420350000000000A7
:0420360000000000A6
:0420370000000000A5
:0420380000000000A4
:0420390000000000A3
:04203A0000000000A2
:04203B0000000000A1
:04203C0000000000A0
:04203D00000000009F
:04203E00000000009E
:04203F00000000009D
:04204000000000009C
:04204100000000009B
:04204200000000009A
:042043000000000099
:042044000000000098
:042045000000000097
:042046000000000096
:042047000000000095
:042048000000000094
:042049000000000093
:04204A000000000092
:04204B000000000091
:04204C000000000090
:04204D00000000008F
:04204E00000000008E
:04204F00000000008D
:04205000000000008C
:04205100000000008B
:04205200000000008A
:042053000000000089
:042054000000000088
:042055000000000087
:042056000000000086
:042057000000000085
:042058000000000084
:042059000000000083
:04205A000000000082
:04205B000000000081
:04205C000000000080
:04205D00000000007F
:04205E00000000007E
:04205F00000000007D
:04206000000000007C
:04206100000000007B
:04206200000000007A
:042063000000000079
:042064000000000078
:042065000000000077
:042066000000000076
:042067000000000075
:042068000000000074
:042069000000000073
:04206A000000000072
:04206B000000000071
:04206C000000000070
:04206D00000000006F
:04206E00000000006E
:04206F00000000006D
:04207000000000006C
:04207100000000006B
:04207200000000006A
:042073000000000069
:042074000000000068
:042075000000000067
:042076000000000066
:042077000000000065
:042078000000000064
:042079000000000063
:04207A000000000062
:04207B000000000061
:04207C000000000060
:04207D00000000005F
:04207E00000000005E
:04207F00000000005D
:04208000000000005C
:04208100000000005B
:04208200000000005A
:042083000000000059
:042084000000000058
:042085000000000057
:042086000000000056
:042087000000000055
:042088000000000054
:042089000000000053
:04208A000000000052
:04208B000000000051
:04208C000000000050
:04208D00000000004F
:04208E00000000004E
:04208F00000000004D
:04209000000000004C
:04209100000000004B
:04209200000000004A
:042093000000000049
:042094000000000048
:042095000000000047
:042096000000000046
:042097000000000045
:042098000000000044
:042099000000000043
:04209A000000000042
:04209B000000000041
:04209C000000000040
:04209D00000000003F
:04209E00000000003E
:04209F00000000003D
:0420A000000000003C
:0420A100000000003B
:0420A200000000003A
:0420A3000000000039
:0420A4000000000038
:0420A5000000000037
:0420A6000000000036
:0420A7000000000035
:0420A8000000000034
:0420A9000000000033
:0420AA000000000032
:0420AB000000000031
:0420AC000000000030
:0420AD00000000002F
:0420AE00000000002E
:0420AF00000000002D
:0420B000000000002C
:0420B100000000002B
:0420B200000000002A
:0420B3000000000029
:0420B4000000000028
:0420B5000000000027
:0420B6000000000026
:0420B7000000000025
:0420B8000000000024
:0420B9000000000023
:0420BA000000000022
:0420BB000000000021
:0420BC000000000020
:0420BD00000000001F
:0420BE00000000001E
:0420BF00000000001D
:0420C000000000001C
:0420C100000000001B
:0420C200000000001A
:0420C3000000000019
:0420C4000000000018
:0420C5000000000017
:0420C6000000000016
:0420C7000000000015
:0420C8000000000014
:0420C9000000000013
:0420CA000000000012
:0420CB000000000011
:0420CC000000000010
:0420CD00000000000F
:0420CE00000000000E
:0420CF00000000000D
:0420D000000000000C
:0420D100000000000B
:0420D200000000000A
:0420D3000000000009
:0420D4000000000008
:0420D5000000000007
:0420D6000000000006
:0420D7000000000005
:0420D8000000000004
:0420D9000000000003
:0420DA000000000002
:0420DB000000000001
:0420DC000000000000
:0420DD0000000000FF
:0420DE0000000000FE
:0420DF0000000000FD
:0420E00000000000FC
:0420E10000000000FB
:0420E20000000000FA
:0420E30000000000F9
:0420E40000000000F8
:0420E50000000000F7
:0420E60000000000F6
:0420E70000000000F5
:0420E80000000000F4
:0420E90000000000F3
:0420EA0000000000F2
:0420EB0000000000F1
:0420EC0000000000F0
:0420ED0000000000EF
:0420EE0000000000EE
:0420EF0000000000ED
:0420F00000000000EC
:0420F10000000000EB
:0420F20000000000EA
:0420F30000000000E9
:0420F40000000000E8
:0420F50000000000E7
:0420F60000000000E6
:0420F70000000000E5
:0420F80000000000E4
:0420F90000000000E3
:0420FA0000000000E2
:0420FB0000000000E1
:0420FC0000000000E0
:0420FD0000000000DF
:0420FE0000000000DE
:0420FF0000000000DD
:0421000000000000DB
:0421010000000000DA
:0421020000000000D9
:0421030000000000D8
:0421040000000000D7
:0421050000000000D6
:0421060000000000D5
:0421070000000000D4
:0421080000000000D3
:0421090000000000D2
:04210A0000000000D1
:04210B0000000000D0
:04210C0000000000CF
:04210D0000000000CE
:04210E0000000000CD
:04210F0000000000CC
:0421100000000000CB
:0421110000000000CA
:0421120000000000C9
:0421130000000000C8
:0421140000000000C7
:0421150000000000C6
:0421160000000000C5
:0421170000000000C4
:0421180000000000C3
:0421190000000000C2
:04211A0000000000C1
:04211B0000000000C0
:04211C0000000000BF
:04211D0000000000BE
:04211E0000000000BD
:04211F0000000000BC
:0421200000000000BB
:0421210000000000BA
:0421220000000000B9
:0421230000000000B8
:0421240000000000B7
:0421250000000000B6
:0421260000000000B5
:0421270000000000B4
:0421280000000000B3
:0421290000000000B2
:04212A0000000000B1
:04212B0000000000B0
:04212C0000000000AF
:04212D0000000000AE
:04212E0000000000AD
:04212F0000000000AC
:0421300000000000AB
:0421310000000000AA
:0421320000000000A9
:0421330000000000A8
:0421340000000000A7
:0421350000000000A6
:0421360000000000A5
:0421370000000000A4
:0421380000000000A3
:0421390000000000A2
:04213A0000000000A1
:04213B0000000000A0
:04213C00000000009F
:04213D00000000009E
:04213E00000000009D
:04213F00000000009C
:04214000000000009B
:04214100000000009A
:042142000000000099
:042143000000000098
:042144000000000097
:042145000000000096
:042146000000000095
:042147000000000094
:042148000000000093
:042149000000000092
:04214A000000000091
:04214B000000000090
:04214C00000000008F
:04214D00000000008E
:04214E00000000008D
:04214F00000000008C
:04215000000000008B
:04215100000000008A
:042152000000000089
:042153000000000088
:042154000000000087
:042155000000000086
:042156000000000085
:042157000000000084
:042158000000000083
:042159000000000082
:04215A000000000081
:04215B000000000080
:04215C00000000007F
:04215D00000000007E
:04215E00000000007D
:04215F00000000007C
:04216000000000007B
:04216100000000007A
:042162000000000079
:042163000000000078
:042164000000000077
:042165000000000076
:042166000000000075
:042167000000000074
:042168000000000073
:042169000000000072
:04216A000000000071
:04216B000000000070
:04216C00000000006F
:04216D00000000006E
:04216E00000000006D
:04216F00000000006C
:04217000000000006B
:04217100000000006A
:042172000000000069
:042173000000000068
:042174000000000067
:042175000000000066
:042176000000000065
:042177000000000064
:042178000000000063
:042179000000000062
:04217A000000000061
:04217B000000000060
:04217C00000000005F
:04217D00000000005E
:04217E00000000005D
:04217F00000000005C
:04218000000000005B
:04218100000000005A
:042182000000000059
:042183000000000058
:042184000000000057
:042185000000000056
:042186000000000055
:042187000000000054
:042188000000000053
:042189000000000052
:04218A000000000051
:04218B000000000050
:04218C00000000004F
:04218D00000000004E
:04218E00000000004D
:04218F00000000004C
:04219000000000004B
:04219100000000004A
:042192000000000049
:042193000000000048
:042194000000000047
:042195000000000046
:042196000000000045
:042197000000000044
:042198000000000043
:042199000000000042
:04219A000000000041
:04219B000000000040
:04219C00000000003F
:04219D00000000003E
:04219E00000000003D
:04219F00000000003C
:0421A000000000003B
:0421A100000000003A
:0421A2000000000039
:0421A3000000000038
:0421A4000000000037
:0421A5000000000036
:0421A6000000000035
:0421A7000000000034
:0421A8000000000033
:0421A9000000000032
:0421AA000000000031
:0421AB000000000030
:0421AC00000000002F
:0421AD00000000002E
:0421AE00000000002D
:0421AF00000000002C
:0421B000000000002B
:0421B100000000002A
:0421B2000000000029
:0421B3000000000028
:0421B4000000000027
:0421B5000000000026
:0421B6000000000025
:0421B7000000000024
:0421B8000000000023
:0421B9000000000022
:0421BA000000000021
:0421BB000000000020
:0421BC00000000001F
:0421BD00000000001E
:0421BE00000000001D
:0421BF00000000001C
:0421C000000000001B
:0421C100000000001A
:0421C2000000000019
:0421C3000000000018
:0421C4000000000017
:0421C5000000000016
:0421C6000000000015
:0421C7000000000014
:0421C8000000000013
:0421C9000000000012
:0421CA000000000011
:0421CB000000000010
:0421CC00000000000F
:0421CD00000000000E
:0421CE00000000000D
:0421CF00000000000C
:0421D000000000000B
:0421D100000000000A
:0421D2000000000009
:0421D3000000000008
:0421D4000000000007
:0421D5000000000006
:0421D6000000000005
:0421D7000000000004
:0421D8000000000003
:0421D9000000000002
:0421DA000000000001
:0421DB000000000000
:0421DC0000000000FF
:0421DD0000000000FE
:0421DE0000000000FD
:0421DF0000000000FC
:0421E00000000000FB
:0421E10000000000FA
:0421E20000000000F9
:0421E30000000000F8
:0421E40000000000F7
:0421E50000000000F6
:0421E60000000000F5
:0421E70000000000F4
:0421E80000000000F3
:0421E90000000000F2
:0421EA0000000000F1
:0421EB0000000000F0
:0421EC0000000000EF
:0421ED0000000000EE
:0421EE0000000000ED
:0421EF0000000000EC
:0421F00000000000EB
:0421F10000000000EA
:0421F20000000000E9
:0421F30000000000E8
:0421F40000000000E7
:0421F50000000000E6
:0421F60000000000E5
:0421F70000000000E4
:0421F80000000000E3
:0421F90000000000E2
:0421FA0000000000E1
:0421FB0000000000E0
:0421FC0000000000DF
:0421FD0000000000DE
:0421FE0000000000DD
:0421FF0000000000DC
:0422000000000000DA
:0422010000000000D9
:0422020000000000D8
:0422030000000000D7
:0422040000000000D6
:0422050000000000D5
:0422060000000000D4
:0422070000000000D3
:0422080000000000D2
:0422090000000000D1
:04220A0000000000D0
:04220B0000000000CF
:04220C0000000000CE
:04220D0000000000CD
:04220E0000000000CC
:04220F0000000000CB
:0422100000000000CA
:0422110000000000C9
:0422120000000000C8
:0422130000000000C7
:0422140000000000C6
:0422150000000000C5
:0422160000000000C4
:0422170000000000C3
:0422180000000000C2
:0422190000000000C1
:04221A0000000000C0
:04221B0000000000BF
:04221C0000000000BE
:04221D0000000000BD
:04221E0000000000BC
:04221F0000000000BB
:0422200000000000BA
:0422210000000000B9
:0422220000000000B8
:0422230000000000B7
:0422240000000000B6
:0422250000000000B5
:0422260000000000B4
:0422270000000000B3
:0422280000000000B2
:0422290000000000B1
:04222A0000000000B0
:04222B0000000000AF
:04222C0000000000AE
:04222D0000000000AD
:04222E0000000000AC
:04222F0000000000AB
:0422300000000000AA
:0422310000000000A9
:0422320000000000A8
:0422330000000000A7
:0422340000000000A6
:0422350000000000A5
:0422360000000000A4
:0422370000000000A3
:0422380000000000A2
:0422390000000000A1
:04223A0000000000A0
:04223B00000000009F
:04223C00000000009E
:04223D00000000009D
:04223E00000000009C
:04223F00000000009B
:04224000000000009A
:042241000000000099
:042242000000000098
:042243000000000097
:042244000000000096
:042245000000000095
:042246000000000094
:042247000000000093
:042248000000000092
:042249000000000091
:04224A000000000090
:04224B00000000008F
:04224C00000000008E
:04224D00000000008D
:04224E00000000008C
:04224F00000000008B
:04225000000000008A
:042251000000000089
:042252000000000088
:042253000000000087
:042254000000000086
:042255000000000085
:042256000000000084
:042257000000000083
:042258000000000082
:042259000000000081
:04225A000000000080
:04225B00000000007F
:04225C00000000007E
:04225D00000000007D
:04225E00000000007C
:04225F00000000007B
:04226000000000007A
:042261000000000079
:042262000000000078
:042263000000000077
:042264000000000076
:042265000000000075
:042266000000000074
:042267000000000073
:042268000000000072
:042269000000000071
:04226A000000000070
:04226B00000000006F
:04226C00000000006E
:04226D00000000006D
:04226E00000000006C
:04226F00000000006B
:04227000000000006A
:042271000000000069
:042272000000000068
:042273000000000067
:042274000000000066
:042275000000000065
:042276000000000064
:042277000000000063
:042278000000000062
:042279000000000061
:04227A000000000060
:04227B00000000005F
:04227C00000000005E
:04227D00000000005D
:04227E00000000005C
:04227F00000000005B
:04228000000000005A
:042281000000000059
:042282000000000058
:042283000000000057
:042284000000000056
:042285000000000055
:042286000000000054
:042287000000000053
:042288000000000052
:042289000000000051
:04228A000000000050
:04228B00000000004F
:04228C00000000004E
:04228D00000000004D
:04228E00000000004C
:04228F00000000004B
:04229000000000004A
:042291000000000049
:042292000000000048
:042293000000000047
:042294000000000046
:042295000000000045
:042296000000000044
:042297000000000043
:042298000000000042
:042299000000000041
:04229A000000000040
:04229B00000000003F
:04229C00000000003E
:04229D00000000003D
:04229E00000000003C
:04229F00000000003B
:0422A000000000003A
:0422A1000000000039
:0422A2000000000038
:0422A3000000000037
:0422A4000000000036
:0422A5000000000035
:0422A6000000000034
:0422A7000000000033
:0422A8000000000032
:0422A9000000000031
:0422AA000000000030
:0422AB00000000002F
:0422AC00000000002E
:0422AD00000000002D
:0422AE00000000002C
:0422AF00000000002B
:0422B000000000002A
:0422B1000000000029
:0422B2000000000028
:0422B3000000000027
:0422B4000000000026
:0422B5000000000025
:0422B6000000000024
:0422B7000000000023
:0422B8000000000022
:0422B9000000000021
:0422BA000000000020
:0422BB00000000001F
:0422BC00000000001E
:0422BD00000000001D
:0422BE00000000001C
:0422BF00000000001B
:0422C000000000001A
:0422C1000000000019
:0422C2000000000018
:0422C3000000000017
:0422C4000000000016
:0422C5000000000015
:0422C6000000000014
:0422C7000000000013
:0422C8000000000012
:0422C9000000000011
:0422CA000000000010
:0422CB00000000000F
:0422CC00000000000E
:0422CD00000000000D
:0422CE00000000000C
:0422CF00000000000B
:0422D000000000000A
:0422D1000000000009
:0422D2000000000008
:0422D3000000000007
:0422D4000000000006
:0422D5000000000005
:0422D6000000000004
:0422D7000000000003
:0422D8000000000002
:0422D9000000000001
:0422DA000000000000
:0422DB0000000000FF
:0422DC0000000000FE
:0422DD0000000000FD
:0422DE0000000000FC
:0422DF0000000000FB
:0422E00000000000FA
:0422E10000000000F9
:0422E20000000000F8
:0422E30000000000F7
:0422E40000000000F6
:0422E50000000000F5
:0422E60000000000F4
:0422E70000000000F3
:0422E80000000000F2
:0422E90000000000F1
:0422EA0000000000F0
:0422EB0000000000EF
:0422EC0000000000EE
:0422ED0000000000ED
:0422EE0000000000EC
:0422EF0000000000EB
:0422F00000000000EA
:0422F10000000000E9
:0422F20000000000E8
:0422F30000000000E7
:0422F40000000000E6
:0422F50000000000E5
:0422F60000000000E4
:0422F70000000000E3
:0422F80000000000E2
:0422F90000000000E1
:0422FA0000000000E0
:0422FB0000000000DF
:0422FC0000000000DE
:0422FD0000000000DD
:0422FE0000000000DC
:0422FF0000000000DB
:0423000000000000D9
:0423010000000000D8
:0423020000000000D7
:0423030000000000D6
:0423040000000000D5
:0423050000000000D4
:0423060000000000D3
:0423070000000000D2
:0423080000000000D1
:0423090000000000D0
:04230A0000000000CF
:04230B0000000000CE
:04230C0000000000CD
:04230D0000000000CC
:04230E0000000000CB
:04230F0000000000CA
:0423100000000000C9
:0423110000000000C8
:0423120000000000C7
:0423130000000000C6
:0423140000000000C5
:0423150000000000C4
:0423160000000000C3
:0423170000000000C2
:0423180000000000C1
:0423190000000000C0
:04231A0000000000BF
:04231B0000000000BE
:04231C0000000000BD
:04231D0000000000BC
:04231E0000000000BB
:04231F0000000000BA
:0423200000000000B9
:0423210000000000B8
:0423220000000000B7
:0423230000000000B6
:0423240000000000B5
:0423250000000000B4
:0423260000000000B3
:0423270000000000B2
:0423280000000000B1
:0423290000000000B0
:04232A0000000000AF
:04232B0000000000AE
:04232C0000000000AD
:04232D0000000000AC
:04232E0000000000AB
:04232F0000000000AA
:0423300000000000A9
:0423310000000000A8
:0423320000000000A7
:0423330000000000A6
:0423340000000000A5
:0423350000000000A4
:0423360000000000A3
:0423370000000000A2
:0423380000000000A1
:0423390000000000A0
:04233A00000000009F
:04233B00000000009E
:04233C00000000009D
:04233D00000000009C
:04233E00000000009B
:04233F00000000009A
:042340000000000099
:042341000000000098
:042342000000000097
:042343000000000096
:042344000000000095
:042345000000000094
:042346000000000093
:042347000000000092
:042348000000000091
:042349000000000090
:04234A00000000008F
:04234B00000000008E
:04234C00000000008D
:04234D00000000008C
:04234E00000000008B
:04234F00000000008A
:042350000000000089
:042351000000000088
:042352000000000087
:042353000000000086
:042354000000000085
:042355000000000084
:042356000000000083
:042357000000000082
:042358000000000081
:042359000000000080
:04235A00000000007F
:04235B00000000007E
:04235C00000000007D
:04235D00000000007C
:04235E00000000007B
:04235F00000000007A
:042360000000000079
:042361000000000078
:042362000000000077
:042363000000000076
:042364000000000075
:042365000000000074
:042366000000000073
:042367000000000072
:042368000000000071
:042369000000000070
:04236A00000000006F
:04236B00000000006E
:04236C00000000006D
:04236D00000000006C
:04236E00000000006B
:04236F00000000006A
:042370000000000069
:042371000000000068
:042372000000000067
:042373000000000066
:042374000000000065
:042375000000000064
:042376000000000063
:042377000000000062
:042378000000000061
:042379000000000060
:04237A00000000005F
:04237B00000000005E
:04237C00000000005D
:04237D00000000005C
:04237E00000000005B
:04237F00000000005A
:042380000000000059
:042381000000000058
:042382000000000057
:042383000000000056
:042384000000000055
:042385000000000054
:042386000000000053
:042387000000000052
:042388000000000051
:042389000000000050
:04238A00000000004F
:04238B00000000004E
:04238C00000000004D
:04238D00000000004C
:04238E00000000004B
:04238F00000000004A
:042390000000000049
:042391000000000048
:042392000000000047
:042393000000000046
:042394000000000045
:042395000000000044
:042396000000000043
:042397000000000042
:042398000000000041
:042399000000000040
:04239A00000000003F
:04239B00000000003E
:04239C00000000003D
:04239D00000000003C
:04239E00000000003B
:04239F00000000003A
:0423A0000000000039
:0423A1000000000038
:0423A2000000000037
:0423A3000000000036
:0423A4000000000035
:0423A5000000000034
:0423A6000000000033
:0423A7000000000032
:0423A8000000000031
:0423A9000000000030
:0423AA00000000002F
:0423AB00000000002E
:0423AC00000000002D
:0423AD00000000002C
:0423AE00000000002B
:0423AF00000000002A
:0423B0000000000029
:0423B1000000000028
:0423B2000000000027
:0423B3000000000026
:0423B4000000000025
:0423B5000000000024
:0423B6000000000023
:0423B7000000000022
:0423B8000000000021
:0423B9000000000020
:0423BA00000000001F
:0423BB00000000001E
:0423BC00000000001D
:0423BD00000000001C
:0423BE00000000001B
:0423BF00000000001A
:0423C0000000000019
:0423C1000000000018
:0423C2000000000017
:0423C3000000000016
:0423C4000000000015
:0423C5000000000014
:0423C6000000000013
:0423C7000000000012
:0423C8000000000011
:0423C9000000000010
:0423CA00000000000F
:0423CB00000000000E
:0423CC00000000000D
:0423CD00000000000C
:0423CE00000000000B
:0423CF00000000000A
:0423D0000000000009
:0423D1000000000008
:0423D2000000000007
:0423D3000000000006
:0423D4000000000005
:0423D5000000000004
:0423D6000000000003
:0423D7000000000002
:0423D8000000000001
:0423D9000000000000
:0423DA0000000000FF
:0423DB0000000000FE
:0423DC0000000000FD
:0423DD0000000000FC
:0423DE0000000000FB
:0423DF0000000000FA
:0423E00000000000F9
:0423E10000000000F8
:0423E20000000000F7
:0423E30000000000F6
:0423E40000000000F5
:0423E50000000000F4
:0423E60000000000F3
:0423E70000000000F2
:0423E80000000000F1
:0423E90000000000F0
:0423EA0000000000EF
:0423EB0000000000EE
:0423EC0000000000ED
:0423ED0000000000EC
:0423EE0000000000EB
:0423EF0000000000EA
:0423F00000000000E9
:0423F10000000000E8
:0423F20000000000E7
:0423F30000000000E6
:0423F40000000000E5
:0423F50000000000E4
:0423F60000000000E3
:0423F70000000000E2
:0423F80000000000E1
:0423F90000000000E0
:0423FA0000000000DF
:0423FB0000000000DE
:0423FC0000000000DD
:0423FD0000000000DC
:0423FE0000000000DB
:0423FF0000000000DA
:0424000000000000D8
:0424010000000000D7
:0424020000000000D6
:0424030000000000D5
:0424040000000000D4
:0424050000000000D3
:0424060000000000D2
:0424070000000000D1
:0424080000000000D0
:0424090000000000CF
:04240A0000000000CE
:04240B0000000000CD
:04240C0000000000CC
:04240D0000000000CB
:04240E0000000000CA
:04240F0000000000C9
:0424100000000000C8
:0424110000000000C7
:0424120000000000C6
:0424130000000000C5
:0424140000000000C4
:0424150000000000C3
:0424160000000000C2
:0424170000000000C1
:0424180000000000C0
:0424190000000000BF
:04241A0000000000BE
:04241B0000000000BD
:04241C0000000000BC
:04241D0000000000BB
:04241E0000000000BA
:04241F0000000000B9
:0424200000000000B8
:0424210000000000B7
:0424220000000000B6
:0424230000000000B5
:0424240000000000B4
:0424250000000000B3
:0424260000000000B2
:0424270000000000B1
:0424280000000000B0
:0424290000000000AF
:04242A0000000000AE
:04242B0000000000AD
:04242C0000000000AC
:04242D0000000000AB
:04242E0000000000AA
:04242F0000000000A9
:0424300000000000A8
:0424310000000000A7
:0424320000000000A6
:0424330000000000A5
:0424340000000000A4
:0424350000000000A3
:0424360000000000A2
:0424370000000000A1
:0424380000000000A0
:04243900000000009F
:04243A00000000009E
:04243B00000000009D
:04243C00000000009C
:04243D00000000009B
:04243E00000000009A
:04243F000000000099
:042440000000000098
:042441000000000097
:042442000000000096
:042443000000000095
:042444000000000094
:042445000000000093
:042446000000000092
:042447000000000091
:042448000000000090
:04244900000000008F
:04244A00000000008E
:04244B00000000008D
:04244C00000000008C
:04244D00000000008B
:04244E00000000008A
:04244F000000000089
:042450000000000088
:042451000000000087
:042452000000000086
:042453000000000085
:042454000000000084
:042455000000000083
:042456000000000082
:042457000000000081
:042458000000000080
:04245900000000007F
:04245A00000000007E
:04245B00000000007D
:04245C00000000007C
:04245D00000000007B
:04245E00000000007A
:04245F000000000079
:042460000000000078
:042461000000000077
:042462000000000076
:042463000000000075
:042464000000000074
:042465000000000073
:042466000000000072
:042467000000000071
:042468000000000070
:04246900000000006F
:04246A00000000006E
:04246B00000000006D
:04246C00000000006C
:04246D00000000006B
:04246E00000000006A
:04246F000000000069
:042470000000000068
:042471000000000067
:042472000000000066
:042473000000000065
:042474000000000064
:042475000000000063
:042476000000000062
:042477000000000061
:042478000000000060
:04247900000000005F
:04247A00000000005E
:04247B00000000005D
:04247C00000000005C
:04247D00000000005B
:04247E00000000005A
:04247F000000000059
:042480000000000058
:042481000000000057
:042482000000000056
:042483000000000055
:042484000000000054
:042485000000000053
:042486000000000052
:042487000000000051
:042488000000000050
:04248900000000004F
:04248A00000000004E
:04248B00000000004D
:04248C00000000004C
:04248D00000000004B
:04248E00000000004A
:04248F000000000049
:042490000000000048
:042491000000000047
:042492000000000046
:042493000000000045
:042494000000000044
:042495000000000043
:042496000000000042
:042497000000000041
:042498000000000040
:04249900000000003F
:04249A00000000003E
:04249B00000000003D
:04249C00000000003C
:04249D00000000003B
:04249E00000000003A
:04249F000000000039
:0424A0000000000038
:0424A1000000000037
:0424A2000000000036
:0424A3000000000035
:0424A4000000000034
:0424A5000000000033
:0424A6000000000032
:0424A7000000000031
:0424A8000000000030
:0424A900000000002F
:0424AA00000000002E
:0424AB00000000002D
:0424AC00000000002C
:0424AD00000000002B
:0424AE00000000002A
:0424AF000000000029
:0424B0000000000028
:0424B1000000000027
:0424B2000000000026
:0424B3000000000025
:0424B4000000000024
:0424B5000000000023
:0424B6000000000022
:0424B7000000000021
:0424B8000000000020
:0424B900000000001F
:0424BA00000000001E
:0424BB00000000001D
:0424BC00000000001C
:0424BD00000000001B
:0424BE00000000001A
:0424BF000000000019
:0424C0000000000018
:0424C1000000000017
:0424C2000000000016
:0424C3000000000015
:0424C4000000000014
:0424C5000000000013
:0424C6000000000012
:0424C7000000000011
:0424C8000000000010
:0424C900000000000F
:0424CA00000000000E
:0424CB00000000000D
:0424CC00000000000C
:0424CD00000000000B
:0424CE00000000000A
:0424CF000000000009
:0424D0000000000008
:0424D1000000000007
:0424D2000000000006
:0424D3000000000005
:0424D4000000000004
:0424D5000000000003
:0424D6000000000002
:0424D7000000000001
:0424D8000000000000
:0424D90000000000FF
:0424DA0000000000FE
:0424DB0000000000FD
:0424DC0000000000FC
:0424DD0000000000FB
:0424DE0000000000FA
:0424DF0000000000F9
:0424E00000000000F8
:0424E10000000000F7
:0424E20000000000F6
:0424E30000000000F5
:0424E40000000000F4
:0424E50000000000F3
:0424E60000000000F2
:0424E70000000000F1
:0424E80000000000F0
:0424E90000000000EF
:0424EA0000000000EE
:0424EB0000000000ED
:0424EC0000000000EC
:0424ED0000000000EB
:0424EE0000000000EA
:0424EF0000000000E9
:0424F00000000000E8
:0424F10000000000E7
:0424F20000000000E6
:0424F30000000000E5
:0424F40000000000E4
:0424F50000000000E3
:0424F60000000000E2
:0424F70000000000E1
:0424F80000000000E0
:0424F90000000000DF
:0424FA0000000000DE
:0424FB0000000000DD
:0424FC0000000000DC
:0424FD0000000000DB
:0424FE0000000000DA
:0424FF0000000000D9
:0425000000000000D7
:0425010000000000D6
:0425020000000000D5
:0425030000000000D4
:0425040000000000D3
:0425050000000000D2
:0425060000000000D1
:0425070000000000D0
:0425080000000000CF
:0425090000000000CE
:04250A0000000000CD
:04250B0000000000CC
:04250C0000000000CB
:04250D0000000000CA
:04250E0000000000C9
:04250F0000000000C8
:0425100000000000C7
:0425110000000000C6
:0425120000000000C5
:0425130000000000C4
:0425140000000000C3
:0425150000000000C2
:0425160000000000C1
:0425170000000000C0
:0425180000000000BF
:0425190000000000BE
:04251A0000000000BD
:04251B0000000000BC
:04251C0000000000BB
:04251D0000000000BA
:04251E0000000000B9
:04251F0000000000B8
:0425200000000000B7
:0425210000000000B6
:0425220000000000B5
:0425230000000000B4
:0425240000000000B3
:0425250000000000B2
:0425260000000000B1
:0425270000000000B0
:0425280000000000AF
:0425290000000000AE
:04252A0000000000AD
:04252B0000000000AC
:04252C0000000000AB
:04252D0000000000AA
:04252E0000000000A9
:04252F0000000000A8
:0425300000000000A7
:0425310000000000A6
:0425320000000000A5
:0425330000000000A4
:0425340000000000A3
:0425350000000000A2
:0425360000000000A1
:0425370000000000A0
:04253800000000009F
:04253900000000009E
:04253A00000000009D
:04253B00000000009C
:04253C00000000009B
:04253D00000000009A
:04253E000000000099
:04253F000000000098
:042540000000000097
:042541000000000096
:042542000000000095
:042543000000000094
:042544000000000093
:042545000000000092
:042546000000000091
:042547000000000090
:04254800000000008F
:04254900000000008E
:04254A00000000008D
:04254B00000000008C
:04254C00000000008B
:04254D00000000008A
:04254E000000000089
:04254F000000000088
:042550000000000087
:042551000000000086
:042552000000000085
:042553000000000084
:042554000000000083
:042555000000000082
:042556000000000081
:042557000000000080
:04255800000000007F
:04255900000000007E
:04255A00000000007D
:04255B00000000007C
:04255C00000000007B
:04255D00000000007A
:04255E000000000079
:04255F000000000078
:042560000000000077
:042561000000000076
:042562000000000075
:042563000000000074
:042564000000000073
:042565000000000072
:042566000000000071
:042567000000000070
:04256800000000006F
:04256900000000006E
:04256A00000000006D
:04256B00000000006C
:04256C00000000006B
:04256D00000000006A
:04256E000000000069
:04256F000000000068
:042570000000000067
:042571000000000066
:042572000000000065
:042573000000000064
:042574000000000063
:042575000000000062
:042576000000000061
:042577000000000060
:04257800000000005F
:04257900000000005E
:04257A00000000005D
:04257B00000000005C
:04257C00000000005B
:04257D00000000005A
:04257E000000000059
:04257F000000000058
:042580000000000057
:042581000000000056
:042582000000000055
:042583000000000054
:042584000000000053
:042585000000000052
:042586000000000051
:042587000000000050
:04258800000000004F
:04258900000000004E
:04258A00000000004D
:04258B00000000004C
:04258C00000000004B
:04258D00000000004A
:04258E000000000049
:04258F000000000048
:042590000000000047
:042591000000000046
:042592000000000045
:042593000000000044
:042594000000000043
:042595000000000042
:042596000000000041
:042597000000000040
:04259800000000003F
:04259900000000003E
:04259A00000000003D
:04259B00000000003C
:04259C00000000003B
:04259D00000000003A
:04259E000000000039
:04259F000000000038
:0425A0000000000037
:0425A1000000000036
:0425A2000000000035
:0425A3000000000034
:0425A4000000000033
:0425A5000000000032
:0425A6000000000031
:0425A7000000000030
:0425A800000000002F
:0425A900000000002E
:0425AA00000000002D
:0425AB00000000002C
:0425AC00000000002B
:0425AD00000000002A
:0425AE000000000029
:0425AF000000000028
:0425B0000000000027
:0425B1000000000026
:0425B2000000000025
:0425B3000000000024
:0425B4000000000023
:0425B5000000000022
:0425B6000000000021
:0425B7000000000020
:0425B800000000001F
:0425B900000000001E
:0425BA00000000001D
:0425BB00000000001C
:0425BC00000000001B
:0425BD00000000001A
:0425BE000000000019
:0425BF000000000018
:0425C0000000000017
:0425C1000000000016
:0425C2000000000015
:0425C3000000000014
:0425C4000000000013
:0425C5000000000012
:0425C6000000000011
:0425C7000000000010
:0425C800000000000F
:0425C900000000000E
:0425CA00000000000D
:0425CB00000000000C
:0425CC00000000000B
:0425CD00000000000A
:0425CE000000000009
:0425CF000000000008
:0425D0000000000007
:0425D1000000000006
:0425D2000000000005
:0425D3000000000004
:0425D4000000000003
:0425D5000000000002
:0425D6000000000001
:0425D7000000000000
:0425D80000000000FF
:0425D90000000000FE
:0425DA0000000000FD
:0425DB0000000000FC
:0425DC0000000000FB
:0425DD0000000000FA
:0425DE0000000000F9
:0425DF0000000000F8
:0425E00000000000F7
:0425E10000000000F6
:0425E20000000000F5
:0425E30000000000F4
:0425E40000000000F3
:0425E50000000000F2
:0425E60000000000F1
:0425E70000000000F0
:0425E80000000000EF
:0425E90000000000EE
:0425EA0000000000ED
:0425EB0000000000EC
:0425EC0000000000EB
:0425ED0000000000EA
:0425EE0000000000E9
:0425EF0000000000E8
:0425F00000000000E7
:0425F10000000000E6
:0425F20000000000E5
:0425F30000000000E4
:0425F40000000000E3
:0425F50000000000E2
:0425F60000000000E1
:0425F70000000000E0
:0425F80000000000DF
:0425F90000000000DE
:0425FA0000000000DD
:0425FB0000000000DC
:0425FC0000000000DB
:0425FD0000000000DA
:0425FE0000000000D9
:0425FF0000000000D8
:0426000000000000D6
:0426010000000000D5
:0426020000000000D4
:0426030000000000D3
:0426040000000000D2
:0426050000000000D1
:0426060000000000D0
:0426070000000000CF
:0426080000000000CE
:0426090000000000CD
:04260A0000000000CC
:04260B0000000000CB
:04260C0000000000CA
:04260D0000000000C9
:04260E0000000000C8
:04260F0000000000C7
:0426100000000000C6
:0426110000000000C5
:0426120000000000C4
:0426130000000000C3
:0426140000000000C2
:0426150000000000C1
:0426160000000000C0
:0426170000000000BF
:0426180000000000BE
:0426190000000000BD
:04261A0000000000BC
:04261B0000000000BB
:04261C0000000000BA
:04261D0000000000B9
:04261E0000000000B8
:04261F0000000000B7
:0426200000000000B6
:0426210000000000B5
:0426220000000000B4
:0426230000000000B3
:0426240000000000B2
:0426250000000000B1
:0426260000000000B0
:0426270000000000AF
:0426280000000000AE
:0426290000000000AD
:04262A0000000000AC
:04262B0000000000AB
:04262C0000000000AA
:04262D0000000000A9
:04262E0000000000A8
:04262F0000000000A7
:0426300000000000A6
:0426310000000000A5
:0426320000000000A4
:0426330000000000A3
:0426340000000000A2
:0426350000000000A1
:0426360000000000A0
:04263700000000009F
:04263800000000009E
:04263900000000009D
:04263A00000000009C
:04263B00000000009B
:04263C00000000009A
:04263D000000000099
:04263E000000000098
:04263F000000000097
:042640000000000096
:042641000000000095
:042642000000000094
:042643000000000093
:042644000000000092
:042645000000000091
:042646000000000090
:04264700000000008F
:04264800000000008E
:04264900000000008D
:04264A00000000008C
:04264B00000000008B
:04264C00000000008A
:04264D000000000089
:04264E000000000088
:04264F000000000087
:042650000000000086
:042651000000000085
:042652000000000084
:042653000000000083
:042654000000000082
:042655000000000081
:042656000000000080
:04265700000000007F
:04265800000000007E
:04265900000000007D
:04265A00000000007C
:04265B00000000007B
:04265C00000000007A
:04265D000000000079
:04265E000000000078
:04265F000000000077
:042660000000000076
:042661000000000075
:042662000000000074
:042663000000000073
:042664000000000072
:042665000000000071
:042666000000000070
:04266700000000006F
:04266800000000006E
:04266900000000006D
:04266A00000000006C
:04266B00000000006B
:04266C00000000006A
:04266D000000000069
:04266E000000000068
:04266F000000000067
:042670000000000066
:042671000000000065
:042672000000000064
:042673000000000063
:042674000000000062
:042675000000000061
:042676000000000060
:04267700000000005F
:04267800000000005E
:04267900000000005D
:04267A00000000005C
:04267B00000000005B
:04267C00000000005A
:04267D000000000059
:04267E000000000058
:04267F000000000057
:042680000000000056
:042681000000000055
:042682000000000054
:042683000000000053
:042684000000000052
:042685000000000051
:042686000000000050
:04268700000000004F
:04268800000000004E
:04268900000000004D
:04268A00000000004C
:04268B00000000004B
:04268C00000000004A
:04268D000000000049
:04268E000000000048
:04268F000000000047
:042690000000000046
:042691000000000045
:042692000000000044
:042693000000000043
:042694000000000042
:042695000000000041
:042696000000000040
:04269700000000003F
:04269800000000003E
:04269900000000003D
:04269A00000000003C
:04269B00000000003B
:04269C00000000003A
:04269D000000000039
:04269E000000000038
:04269F000000000037
:0426A0000000000036
:0426A1000000000035
:0426A2000000000034
:0426A3000000000033
:0426A4000000000032
:0426A5000000000031
:0426A6000000000030
:0426A700000000002F
:0426A800000000002E
:0426A900000000002D
:0426AA00000000002C
:0426AB00000000002B
:0426AC00000000002A
:0426AD000000000029
:0426AE000000000028
:0426AF000000000027
:0426B0000000000026
:0426B1000000000025
:0426B2000000000024
:0426B3000000000023
:0426B4000000000022
:0426B5000000000021
:0426B6000000000020
:0426B700000000001F
:0426B800000000001E
:0426B900000000001D
:0426BA00000000001C
:0426BB00000000001B
:0426BC00000000001A
:0426BD000000000019
:0426BE000000000018
:0426BF000000000017
:0426C0000000000016
:0426C1000000000015
:0426C2000000000014
:0426C3000000000013
:0426C4000000000012
:0426C5000000000011
:0426C6000000000010
:0426C700000000000F
:0426C800000000000E
:0426C900000000000D
:0426CA00000000000C
:0426CB00000000000B
:0426CC00000000000A
:0426CD000000000009
:0426CE000000000008
:0426CF000000000007
:0426D0000000000006
:0426D1000000000005
:0426D2000000000004
:0426D3000000000003
:0426D4000000000002
:0426D5000000000001
:0426D6000000000000
:0426D70000000000FF
:0426D80000000000FE
:0426D90000000000FD
:0426DA0000000000FC
:0426DB0000000000FB
:0426DC0000000000FA
:0426DD0000000000F9
:0426DE0000000000F8
:0426DF0000000000F7
:0426E00000000000F6
:0426E10000000000F5
:0426E20000000000F4
:0426E30000000000F3
:0426E40000000000F2
:0426E50000000000F1
:0426E60000000000F0
:0426E70000000000EF
:0426E80000000000EE
:0426E90000000000ED
:0426EA0000000000EC
:0426EB0000000000EB
:0426EC0000000000EA
:0426ED0000000000E9
:0426EE0000000000E8
:0426EF0000000000E7
:0426F00000000000E6
:0426F10000000000E5
:0426F20000000000E4
:0426F30000000000E3
:0426F40000000000E2
:0426F50000000000E1
:0426F60000000000E0
:0426F70000000000DF
:0426F80000000000DE
:0426F90000000000DD
:0426FA0000000000DC
:0426FB0000000000DB
:0426FC0000000000DA
:0426FD0000000000D9
:0426FE0000000000D8
:0426FF0000000000D7
:0427000000000000D5
:0427010000000000D4
:0427020000000000D3
:0427030000000000D2
:0427040000000000D1
:0427050000000000D0
:0427060000000000CF
:0427070000000000CE
:0427080000000000CD
:0427090000000000CC
:04270A0000000000CB
:04270B0000000000CA
:04270C0000000000C9
:04270D0000000000C8
:04270E0000000000C7
:04270F0000000000C6
